:020000040000FA
:100000000808080808080808080808080808080870
:100010000808080808080808080808080808080860
:100020000808080808080808080808080808080850
:100030000808080808080808080808080808080840
:020000040003F7
:020000040004F6
:1000000008080808080808080C0C0C0C0C0C0C0C50
:100010000C0C0C0C0C0C0C0C0C0C0C0C0C0C0C0C20
:100020000C0C0C0C0C0C0C0C0C0C0C0C0C0C0C0C10
:100030000C0C0C0C0C0C0C0C0C0C0C0C0C0C0C0C00
:1000400008080808080808080C0C0C0C0C0C0C0C10
:100050000C0C0C0C0C0C0C0C0C0C0C0C0C0C0C0CE0
:100060000C0C0C0C0C0C0C0C0C0C0C0C0C0C0C0CD0
:100070000C0C0C0C0C0C0C0C0C0C0C0C0C0C0C0CC0
:1000800008080808080808080C0C0C0C0C0C0C0CD0
:100090000C0C0C0C0C0C0C0C0C0C0C0C0C0C0C0CA0
:1000A0000C0C0C0C0C0C0C0C0C0C0C0C0C0C0C0C90
:1000B0000C0C0C0C0C0C0C0C0C0C0C0C0C0C0C0C80
:1000C00008080808080808080C0C0C0C0C0C0C0C90
:1000D0000C0C0C0C0C0C0C0C0C0C0C0C0C0C0C0C60
:1000E0000C0C0C0C0C0C0C0C0C0C0C0C0C0C0C0C50
:1000F0000C0C0C0C0C0C0C0C0C0C0C0C0C0C0C0C40
:1001000008080808080808080C0C0C0C0C0C0C0C4F
:100110000C0C0C0C0C0C0C0C0C0C0C0C0C0C0C0C1F
:100120000C0C0C0C0C0C0C0C0C0C0C0C0C0C0C0C0F
:100130000C0C0C0C0C0C0C0C0C0C0C0C0C0C0C0CFF
:1001400008080808080808080C0C0C0C0C0C0C0C0F
:100150000C0C0C0C0C0C0C0C0C0C0C0C0C0C0C0CDF
:100160000C0C0C0C0C0C0C0C0C0C0C0C0C0C0C0CCF
:100170000C0C0C0C0C0C0C0C0C0C0C0C0C0C0C0CBF
:1001800008080808080808080C0C0C0C0C0C0C0CCF
:100190000C0C0C0C0C0C0C0C0C0C0C0C0C0C0C0C9F
:1001A0000C0C0C0C0C0C0C0C0C0C0C0C0C0C0C0C8F
:1001B0000C0C0C0C0C0C0C0C0C0C0C0C0C0C0C0C7F
:1001C00008080808080808080C0C0C0C0C0C0C0C8F
:1001D0000C0C0C0C0C0C0C0C0C0C0C0C0C0C0C0C5F
:1001E0000C0C0C0C0C0C0C0C0C0C0C0C0C0C0C0C4F
:1001F0000C0C0C0C0C0C0C0C0C0C0C0C0C0C0C0C3F
:1002000008080808080808080C0C0C0C0C0C0C0C4E
:100210000C0C0C0C0C0C0C0C0C0C0C0C0C0C0C0C1E
:100220000C0C0C0C0C0C0C0C0C0C0C0C0C0C0C0C0E
:100230000C0C0C0C0C0C0C0C0C0C0C0C0C0C0C0CFE
:1002400008080808080808080C0C0C0C0C0C0C0C0E
:100250000C0C0C0C0C0C0C0C0C0C0C0C0C0C0C0CDE
:100260000C0C0C0C0C0C0C0C0C0C0C0C0C0C0C0CCE
:100270000C0C0C0C0C0C0C0C0C0C0C0C0C0C0C0CBE
:1002800008080808080808080C0C0C0C0C0C0C0CCE
:100290000C0C0C0C0C0C0C0C0C0C0C0C0C0C0C0C9E
:1002A0000C0C0C0C0C0C0C0C0C0C0C0C0C0C0C0C8E
:1002B0000C0C0C0C0C0C0C0C0C0C0C0C0C0C0C0C7E
:1002C00008080808080808080C0C0C0C0C0C0C0C8E
:1002D0000C0C0C0C0C0C0C0C0C0C0C0C0C0C0C0C5E
:1002E0000C0C0C0C0C0C0C0C0C0C0C0C0C0C0C0C4E
:1002F0000C0C0C0C0C0C0C0C0C0C0C0C0C0C0C0C3E
:1003000008080808080808080C0C0C0C0C0C0C0C4D
:100310000C0C0C0C0C0C0C0C0C0C0C0C0C0C0C0C1D
:100320000C0C0C0C0C0C0C0C0C0C0C0C0C0C0C0C0D
:100330000C0C0C0C0C0C0C0C0C0C0C0C0C0C0C0CFD
:1003400008080808080808080C0C0C0C0C0C0C0C0D
:100350000C0C0C0C0C0C0C0C0C0C0C0C0C0C0C0CDD
:100360000C0C0C0C0C0C0C0C0C0C0C0C0C0C0C0CCD
:100370000C0C0C0C0C0C0C0C0C0C0C0C0C0C0C0CBD
:1003800008080808080808080C0C0C0C0C0C0C0CCD
:100390000C0C0C0C0C0C0C0C0C0C0C0C0C0C0C0C9D
:1003A0000C0C0C0C0C0C0C0C0C0C0C0C0C0C0C0C8D
:1003B0000C0C0C0C0C0C0C0C0C0C0C0C0C0C0C0C7D
:1003C00008080808080808080C0C0C0C0C0C0C0C8D
:1003D0000C0C0C0C0C0C0C0C0C0C0C0C0C0C0C0C5D
:1003E0000C0C0C0C0C0C0C0C0C0C0C0C0C0C0C0C4D
:1003F0000C0C0C0C0C0C0C0C0C0C0C0C0C0C0C0C3D
:1004000008080808080808080C0C0C0C0C0C0C0C4C
:100410000C0C0C0C0C0C0C0C0C0C0C0C0C0C0C0C1C
:100420000C0C0C0C0C0C0C0C0C0C0C0C0C0C0C0C0C
:100430000C0C0C0C0C0C0C0C0C0C0C0C0C0C0C0CFC
:1004400008080808080808080C0C0C0C0C0C0C0C0C
:100450000C0C0C0C0C0C0C0C0C0C0C0C0C0C0C0CDC
:100460000C0C0C0C0C0C0C0C0C0C0C0C0C0C0C0CCC
:100470000C0C0C0C0C0C0C0C0C0C0C0C0C0C0C0CBC
:1004800008080808080808080C0C0C0C0C0C0C0CCC
:100490000C0C0C0C0C0C0C0C0C0C0C0C0C0C0C0C9C
:1004A0000C0C0C0C0C0C0C0C0C0C0C0C0C0C0C0C8C
:1004B0000C0C0C0C0C0C0C0C0C0C0C0C0C0C0C0C7C
:1004C00008080808080808080C0C0C0C0C0C0C0C8C
:1004D0000C0C0C0C0C0C0C0C0C0C0C0C0C0C0C0C5C
:1004E0000C0C0C0C0C0C0C0C0C0C0C0C0C0C0C0C4C
:1004F0000C0C0C0C0C0C0C0C0C0C0C0C0C0C0C0C3C
:1005000008080808080808080C0C0C0C0C0C0C0C4B
:100510000C0C0C0C0C0C0C0C0C0C0C0C0C0C0C0C1B
:100520000C0C0C0C0C0C0C0C0C0C0C0C0C0C0C0C0B
:100530000C0C0C0C0C0C0C0C0C0C0C0C0C0C0C0CFB
:1005400008080808080808080C0C0C0C0C0C0C0C0B
:100550000C0C0C0C0C0C0C0C0C0C0C0C0C0C0C0CDB
:100560000C0C0C0C0C0C0C0C0C0C0C0C0C0C0C0CCB
:100570000C0C0C0C0C0C0C0C0C0C0C0C0C0C0C0CBB
:1005800008080808080808080C0C0C0C0C0C0C0CCB
:100590000C0C0C0C0C0C0C0C0C0C0C0C0C0C0C0C9B
:1005A0000C0C0C0C0C0C0C0C0C0C0C0C0C0C0C0C8B
:1005B0000C0C0C0C0C0C0C0C0C0C0C0C0C0C0C0C7B
:1005C00008080808080808080C0C0C0C0C0C0C0C8B
:1005D0000C0C0C0C0C0C0C0C0C0C0C0C0C0C0C0C5B
:1005E0000C0C0C0C0C0C0C0C0C0C0C0C0C0C0C0C4B
:1005F0000C0C0C0C0C0C0C0C0C0C0C0C0C0C0C0C3B
:1006000008080808080808080C0C0C0C0C0C0C0C4A
:100610000C0C0C0C0C0C0C0C0C0C0C0C0C0C0C0C1A
:100620000C0C0C0C0C0C0C0C0C0C0C0C0C0C0C0C0A
:100630000C0C0C0C0C0C0C0C0C0C0C0C0C0C0C0CFA
:1006400008080808080808080C0C0C0C0C0C0C0C0A
:100650000C0C0C0C0C0C0C0C0C0C0C0C0C0C0C0CDA
:100660000C0C0C0C0C0C0C0C0C0C0C0C0C0C0C0CCA
:100670000C0C0C0C0C0C0C0C0C0C0C0C0C0C0C0CBA
:1006800008080808080808080C0C0C0C0C0C0C0CCA
:100690000C0C0C0C0C0C0C0C0C0C0C0C0C0C0C0C9A
:1006A0000C0C0C0C0C0C0C0C0C0C0C0C0C0C0C0C8A
:1006B0000C0C0C0C0C0C0C0C0C0C0C0C0C0C0C0C7A
:1006C00008080808080808080C0C0C0C0C0C0C0C8A
:1006D0000C0C0C0C0C0C0C0C0C0C0C0C0C0C0C0C5A
:1006E0000C0C0C0C0C0C0C0C0C0C0C0C0C0C0C0C4A
:1006F0000C0C0C0C0C0C0C0C0C0C0C0C0C0C0C0C3A
:1007000008080808080808080C0C0C0C0C0C0C0C49
:100710000C0C0C0C0C0C0C0C0C0C0C0C0C0C0C0C19
:100720000C0C0C0C0C0C0C0C0C0C0C0C0C0C0C0C09
:100730000C0C0C0C0C0C0C0C0C0C0C0C0C0C0C0CF9
:1007400008080808080808080C0C0C0C0C0C0C0C09
:100750000C0C0C0C0C0C0C0C0C0C0C0C0C0C0C0CD9
:100760000C0C0C0C0C0C0C0C0C0C0C0C0C0C0C0CC9
:100770000C0C0C0C0C0C0C0C0C0C0C0C0C0C0C0CB9
:1007800008080808080808080C0C0C0C0C0C0C0CC9
:100790000C0C0C0C0C0C0C0C0C0C0C0C0C0C0C0C99
:1007A0000C0C0C0C0C0C0C0C0C0C0C0C0C0C0C0C89
:1007B0000C0C0C0C0C0C0C0C0C0C0C0C0C0C0C0C79
:1007C00008080808080808080C0C0C0C0C0C0C0C89
:1007D0000C0C0C0C0C0C0C0C0C0C0C0C0C0C0C0C59
:1007E0000C0C0C0C0C0C0C0C0C0C0C0C0C0C0C0C49
:1007F0000C0C0C0C0C0C0C0C0C0C0C0C0C0C0C0C39
:1008000008080808080808080C0C0C0C0C0C0C0C48
:100810000C0C0C0C0C0C0C0C0C0C0C0C0C0C0C0C18
:100820000C0C0C0C0C0C0C0C0C0C0C0C0C0C0C0C08
:100830000C0C0C0C0C0C0C0C0C0C0C0C0C0C0C0CF8
:1008400008080808080808080C0C0C0C0C0C0C0C08
:100850000C0C0C0C0C0C0C0C0C0C0C0C0C0C0C0CD8
:100860000C0C0C0C0C0C0C0C0C0C0C0C0C0C0C0CC8
:100870000C0C0C0C0C0C0C0C0C0C0C0C0C0C0C0CB8
:1008800008080808080808080C0C0C0C0C0C0C0CC8
:100890000C0C0C0C0C0C0C0C0C0C0C0C0C0C0C0C98
:1008A0000C0C0C0C0C0C0C0C0C0C0C0C0C0C0C0C88
:1008B0000C0C0C0C0C0C0C0C0C0C0C0C0C0C0C0C78
:1008C00008080808080808080C0C0C0C0C0C0C0C88
:1008D0000C0C0C0C0C0C0C0C0C0C0C0C0C0C0C0C58
:1008E0000C0C0C0C0C0C0C0C0C0C0C0C0C0C0C0C48
:1008F0000C0C0C0C0C0C0C0C0C0C0C0C0C0C0C0C38
:1009000008080808080808080C0C0C0C0C0C0C0C47
:100910000C0C0C0C0C0C0C0C0C0C0C0C0C0C0C0C17
:100920000C0C0C0C0C0C0C0C0C0C0C0C0C0C0C0C07
:100930000C0C0C0C0C0C0C0C0C0C0C0C0C0C0C0CF7
:1009400008080808080808080C0C0C0C0C0C0C0C07
:100950000C0C0C0C0C0C0C0C0C0C0C0C0C0C0C0CD7
:100960000C0C0C0C0C0C0C0C0C0C0C0C0C0C0C0CC7
:100970000C0C0C0C0C0C0C0C0C0C0C0C0C0C0C0CB7
:1009800008080808080808080C0C0C0C0C0C0C0CC7
:100990000C0C0C0C0C0C0C0C0C0C0C0C0C0C0C0C97
:1009A0000C0C0C0C0C0C0C0C0C0C0C0C0C0C0C0C87
:1009B0000C0C0C0C0C0C0C0C0C0C0C0C0C0C0C0C77
:1009C00008080808080808080C0C0C0C0C0C0C0C87
:1009D0000C0C0C0C0C0C0C0C0C0C0C0C0C0C0C0C57
:1009E0000C0C0C0C0C0C0C0C0C0C0C0C0C0C0C0C47
:1009F0000C0C0C0C0C0C0C0C0C0C0C0C0C0C0C0C37
:100A000008080808080808080C0C0C0C0C0C0C0C46
:100A10000C0C0C0C0C0C0C0C0C0C0C0C0C0C0C0C16
:100A20000C0C0C0C0C0C0C0C0C0C0C0C0C0C0C0C06
:100A30000C0C0C0C0C0C0C0C0C0C0C0C0C0C0C0CF6
:100A400008080808080808080C0C0C0C0C0C0C0C06
:100A50000C0C0C0C0C0C0C0C0C0C0C0C0C0C0C0CD6
:100A60000C0C0C0C0C0C0C0C0C0C0C0C0C0C0C0CC6
:100A70000C0C0C0C0C0C0C0C0C0C0C0C0C0C0C0CB6
:100A800008080808080808080C0C0C0C0C0C0C0CC6
:100A90000C0C0C0C0C0C0C0C0C0C0C0C0C0C0C0C96
:100AA0000C0C0C0C0C0C0C0C0C0C0C0C0C0C0C0C86
:100AB0000C0C0C0C0C0C0C0C0C0C0C0C0C0C0C0C76
:100AC00008080808080808080C0C0C0C0C0C0C0C86
:100AD0000C0C0C0C0C0C0C0C0C0C0C0C0C0C0C0C56
:100AE0000C0C0C0C0C0C0C0C0C0C0C0C0C0C0C0C46
:100AF0000C0C0C0C0C0C0C0C0C0C0C0C0C0C0C0C36
:100B000008080808080808080C0C0C0C0C0C0C0C45
:100B10000C0C0C0C0C0C0C0C0C0C0C0C0C0C0C0C15
:100B20000C0C0C0C0C0C0C0C0C0C0C0C0C0C0C0C05
:100B30000C0C0C0C0C0C0C0C0C0C0C0C0C0C0C0CF5
:100B400008080808080808080C0C0C0C0C0C0C0C05
:100B50000C0C0C0C0C0C0C0C0C0C0C0C0C0C0C0CD5
:100B60000C0C0C0C0C0C0C0C0C0C0C0C0C0C0C0CC5
:100B70000C0C0C0C0C0C0C0C0C0C0C0C0C0C0C0CB5
:100B800008080808080808080C0C0C0C0C0C0C0CC5
:100B90000C0C0C0C0C0C0C0C0C0C0C0C0C0C0C0C95
:100BA0000C0C0C0C0C0C0C0C0C0C0C0C0C0C0C0C85
:100BB0000C0C0C0C0C0C0C0C0C0C0C0C0C0C0C0C75
:100BC00008080808080808080C0C0C0C0C0C0C0C85
:100BD0000C0C0C0C0C0C0C0C0C0C0C0C0C0C0C0C55
:100BE0000C0C0C0C0C0C0C0C0C0C0C0C0C0C0C0C45
:100BF0000C0C0C0C0C0C0C0C0C0C0C0C0C0C0C0C35
:100C000008080808080808080C0C0C0C0C0C0C0C44
:100C10000C0C0C0C0C0C0C0C0C0C0C0C0C0C0C0C14
:100C20000C0C0C0C0C0C0C0C0C0C0C0C0C0C0C0C04
:100C30000C0C0C0C0C0C0C0C0C0C0C0C0C0C0C0CF4
:100C400008080808080808080C0C0C0C0C0C0C0C04
:100C50000C0C0C0C0C0C0C0C0C0C0C0C0C0C0C0CD4
:100C60000C0C0C0C0C0C0C0C0C0C0C0C0C0C0C0CC4
:100C70000C0C0C0C0C0C0C0C0C0C0C0C0C0C0C0CB4
:100C800008080808080808080C0C0C0C0C0C0C0CC4
:100C90000C0C0C0C0C0C0C0C0C0C0C0C0C0C0C0C94
:100CA0000C0C0C0C0C0C0C0C0C0C0C0C0C0C0C0C84
:100CB0000C0C0C0C0C0C0C0C0C0C0C0C0C0C0C0C74
:100CC00008080808080808080C0C0C0C0C0C0C0C84
:100CD0000C0C0C0C0C0C0C0C0C0C0C0C0C0C0C0C54
:100CE0000C0C0C0C0C0C0C0C0C0C0C0C0C0C0C0C44
:100CF0000C0C0C0C0C0C0C0C0C0C0C0C0C0C0C0C34
:100D000008080808080808080C0C0C0C0C0C0C0C43
:100D10000C0C0C0C0C0C0C0C0C0C0C0C0C0C0C0C13
:100D20000C0C0C0C0C0C0C0C0C0C0C0C0C0C0C0C03
:100D30000C0C0C0C0C0C0C0C0C0C0C0C0C0C0C0CF3
:100D400008080808080808080C0C0C0C0C0C0C0C03
:100D50000C0C0C0C0C0C0C0C0C0C0C0C0C0C0C0CD3
:100D60000C0C0C0C0C0C0C0C0C0C0C0C0C0C0C0CC3
:100D70000C0C0C0C0C0C0C0C0C0C0C0C0C0C0C0CB3
:100D800008080808080808080C0C0C0C0C0C0C0CC3
:100D90000C0C0C0C0C0C0C0C0C0C0C0C0C0C0C0C93
:100DA0000C0C0C0C0C0C0C0C0C0C0C0C0C0C0C0C83
:100DB0000C0C0C0C0C0C0C0C0C0C0C0C0C0C0C0C73
:100DC00008080808080808080C0C0C0C0C0C0C0C83
:100DD0000C0C0C0C0C0C0C0C0C0C0C0C0C0C0C0C53
:100DE0000C0C0C0C0C0C0C0C0C0C0C0C0C0C0C0C43
:100DF0000C0C0C0C0C0C0C0C0C0C0C0C0C0C0C0C33
:100E000008080808080808080C0C0C0C0C0C0C0C42
:100E10000C0C0C0C0C0C0C0C0C0C0C0C0C0C0C0C12
:100E20000C0C0C0C0C0C0C0C0C0C0C0C0C0C0C0C02
:100E30000C0C0C0C0C0C0C0C0C0C0C0C0C0C0C0CF2
:100E400008080808080808080C0C0C0C0C0C0C0C02
:100E50000C0C0C0C0C0C0C0C0C0C0C0C0C0C0C0CD2
:100E60000C0C0C0C0C0C0C0C0C0C0C0C0C0C0C0CC2
:100E70000C0C0C0C0C0C0C0C0C0C0C0C0C0C0C0CB2
:100E800008080808080808080C0C0C0C0C0C0C0CC2
:100E90000C0C0C0C0C0C0C0C0C0C0C0C0C0C0C0C92
:100EA0000C0C0C0C0C0C0C0C0C0C0C0C0C0C0C0C82
:100EB0000C0C0C0C0C0C0C0C0C0C0C0C0C0C0C0C72
:100EC00008080808080808080C0C0C0C0C0C0C0C82
:100ED0000C0C0C0C0C0C0C0C0C0C0C0C0C0C0C0C52
:100EE0000C0C0C0C0C0C0C0C0C0C0C0C0C0C0C0C42
:100EF0000C0C0C0C0C0C0C0C0C0C0C0C0C0C0C0C32
:100F000008080808080808080C0C0C0C0C0C0C0C41
:100F10000C0C0C0C0C0C0C0C0C0C0C0C0C0C0C0C11
:100F20000C0C0C0C0C0C0C0C0C0C0C0C0C0C0C0C01
:100F30000C0C0C0C0C0C0C0C0C0C0C0C0C0C0C0CF1
:100F400008080808080808080C0C0C0C0C0C0C0C01
:100F50000C0C0C0C0C0C0C0C0C0C0C0C0C0C0C0CD1
:100F60000C0C0C0C0C0C0C0C0C0C0C0C0C0C0C0CC1
:100F70000C0C0C0C0C0C0C0C0C0C0C0C0C0C0C0CB1
:100F800008080808080808080C0C0C0C0C0C0C0CC1
:100F90000C0C0C0C0C0C0C0C0C0C0C0C0C0C0C0C91
:100FA0000C0C0C0C0C0C0C0C0C0C0C0C0C0C0C0C81
:100FB0000C0C0C0C0C0C0C0C0C0C0C0C0C0C0C0C71
:100FC00008080808080808080C0C0C0C0C0C0C0C81
:100FD0000C0C0C0C0C0C0C0C0C0C0C0C0C0C0C0C51
:100FE0000C0C0C0C0C0C0C0C0C0C0C0C0C0C0C0C41
:100FF0000C0C0C0C0C0C0C0C0C0C0C0C0C0C0C0C31
:1010000008080808080808080C0C0C0C0C0C0C0C40
:101010000C0C0C0C0C0C0C0C0C0C0C0C0C0C0C0C10
:101020000C0C0C0C0C0C0C0C0C0C0C0C0C0C0C0C00
:101030000C0C0C0C0C0C0C0C0C0C0C0C0C0C0C0CF0
:1010400008080808080808080C0C0C0C0C0C0C0C00
:101050000C0C0C0C0C0C0C0C0C0C0C0C0C0C0C0CD0
:101060000C0C0C0C0C0C0C0C0C0C0C0C0C0C0C0CC0
:101070000C0C0C0C0C0C0C0C0C0C0C0C0C0C0C0CB0
:1010800008080808080808080C0C0C0C0C0C0C0CC0
:101090000C0C0C0C0C0C0C0C0C0C0C0C0C0C0C0C90
:1010A0000C0C0C0C0C0C0C0C0C0C0C0C0C0C0C0C80
:1010B0000C0C0C0C0C0C0C0C0C0C0C0C0C0C0C0C70
:1010C00008080808080808080C0C0C0C0C0C0C0C80
:1010D0000C0C0C0C0C0C0C0C0C0C0C0C0C0C0C0C50
:1010E0000C0C0C0C0C0C0C0C0C0C0C0C0C0C0C0C40
:1010F0000C0C0C0C0C0C0C0C0C0C0C0C0C0C0C0C30
:1011000008080808080808080C0C0C0C0C0C0C0C3F
:101110000C0C0C0C0C0C0C0C0C0C0C0C0C0C0C0C0F
:101120000C0C0C0C0C0C0C0C0C0C0C0C0C0C0C0CFF
:101130000C0C0C0C0C0C0C0C0C0C0C0C0C0C0C0CEF
:1011400008080808080808080C0C0C0C0C0C0C0CFF
:101150000C0C0C0C0C0C0C0C0C0C0C0C0C0C0C0CCF
:101160000C0C0C0C0C0C0C0C0C0C0C0C0C0C0C0CBF
:101170000C0C0C0C0C0C0C0C0C0C0C0C0C0C0C0CAF
:1011800008080808080808080C0C0C0C0C0C0C0CBF
:101190000C0C0C0C0C0C0C0C0C0C0C0C0C0C0C0C8F
:1011A0000C0C0C0C0C0C0C0C0C0C0C0C0C0C0C0C7F
:1011B0000C0C0C0C0C0C0C0C0C0C0C0C0C0C0C0C6F
:1011C00008080808080808080C0C0C0C0C0C0C0C7F
:1011D0000C0C0C0C0C0C0C0C0C0C0C0C0C0C0C0C4F
:1011E0000C0C0C0C0C0C0C0C0C0C0C0C0C0C0C0C3F
:1011F0000C0C0C0C0C0C0C0C0C0C0C0C0C0C0C0C2F
:1012000008080808080808080C0C0C0C0C0C0C0C3E
:101210000C0C0C0C0C0C0C0C0C0C0C0C0C0C0C0C0E
:101220000C0C0C0C0C0C0C0C0C0C0C0C0C0C0C0CFE
:101230000C0C0C0C0C0C0C0C0C0C0C0C0C0C0C0CEE
:1012400008080808080808080C0C0C0C0C0C0C0CFE
:101250000C0C0C0C0C0C0C0C0C0C0C0C0C0C0C0CCE
:101260000C0C0C0C0C0C0C0C0C0C0C0C0C0C0C0CBE
:101270000C0C0C0C0C0C0C0C0C0C0C0C0C0C0C0CAE
:1012800008080808080808080C0C0C0C0C0C0C0CBE
:101290000C0C0C0C0C0C0C0C0C0C0C0C0C0C0C0C8E
:1012A0000C0C0C0C0C0C0C0C0C0C0C0C0C0C0C0C7E
:1012B0000C0C0C0C0C0C0C0C0C0C0C0C0C0C0C0C6E
:1012C00008080808080808080C0C0C0C0C0C0C0C7E
:1012D0000C0C0C0C0C0C0C0C0C0C0C0C0C0C0C0C4E
:1012E0000C0C0C0C0C0C0C0C0C0C0C0C0C0C0C0C3E
:1012F0000C0C0C0C0C0C0C0C0C0C0C0C0C0C0C0C2E
:1013000008080808080808080C0C0C0C0C0C0C0C3D
:101310000C0C0C0C0C0C0C0C0C0C0C0C0C0C0C0C0D
:101320000C0C0C0C0C0C0C0C0C0C0C0C0C0C0C0CFD
:101330000C0C0C0C0C0C0C0C0C0C0C0C0C0C0C0CED
:1013400008080808080808080C0C0C0C0C0C0C0CFD
:101350000C0C0C0C0C0C0C0C0C0C0C0C0C0C0C0CCD
:101360000C0C0C0C0C0C0C0C0C0C0C0C0C0C0C0CBD
:101370000C0C0C0C0C0C0C0C0C0C0C0C0C0C0C0CAD
:1013800008080808080808080C0C0C0C0C0C0C0CBD
:101390000C0C0C0C0C0C0C0C0C0C0C0C0C0C0C0C8D
:1013A0000C0C0C0C0C0C0C0C0C0C0C0C0C0C0C0C7D
:1013B0000C0C0C0C0C0C0C0C0C0C0C0C0C0C0C0C6D
:1013C00008080808080808080C0C0C0C0C0C0C0C7D
:1013D0000C0C0C0C0C0C0C0C0C0C0C0C0C0C0C0C4D
:1013E0000C0C0C0C0C0C0C0C0C0C0C0C0C0C0C0C3D
:1013F0000C0C0C0C0C0C0C0C0C0C0C0C0C0C0C0C2D
:1014000008080808080808080C0C0C0C0C0C0C0C3C
:101410000C0C0C0C0C0C0C0C0C0C0C0C0C0C0C0C0C
:101420000C0C0C0C0C0C0C0C0C0C0C0C0C0C0C0CFC
:101430000C0C0C0C0C0C0C0C0C0C0C0C0C0C0C0CEC
:1014400008080808080808080C0C0C0C0C0C0C0CFC
:101450000C0C0C0C0C0C0C0C0C0C0C0C0C0C0C0CCC
:101460000C0C0C0C0C0C0C0C0C0C0C0C0C0C0C0CBC
:101470000C0C0C0C0C0C0C0C0C0C0C0C0C0C0C0CAC
:1014800008080808080808080C0C0C0C0C0C0C0CBC
:101490000C0C0C0C0C0C0C0C0C0C0C0C0C0C0C0C8C
:1014A0000C0C0C0C0C0C0C0C0C0C0C0C0C0C0C0C7C
:1014B0000C0C0C0C0C0C0C0C0C0C0C0C0C0C0C0C6C
:1014C00008080808080808080C0C0C0C0C0C0C0C7C
:1014D0000C0C0C0C0C0C0C0C0C0C0C0C0C0C0C0C4C
:1014E0000C0C0C0C0C0C0C0C0C0C0C0C0C0C0C0C3C
:1014F0000C0C0C0C0C0C0C0C0C0C0C0C0C0C0C0C2C
:1015000008080808080808080C0C0C0C0C0C0C0C3B
:101510000C0C0C0C0C0C0C0C0C0C0C0C0C0C0C0C0B
:101520000C0C0C0C0C0C0C0C0C0C0C0C0C0C0C0CFB
:101530000C0C0C0C0C0C0C0C0C0C0C0C0C0C0C0CEB
:1015400008080808080808080C0C0C0C0C0C0C0CFB
:101550000C0C0C0C0C0C0C0C0C0C0C0C0C0C0C0CCB
:101560000C0C0C0C0C0C0C0C0C0C0C0C0C0C0C0CBB
:101570000C0C0C0C0C0C0C0C0C0C0C0C0C0C0C0CAB
:1015800008080808080808080C0C0C0C0C0C0C0CBB
:101590000C0C0C0C0C0C0C0C0C0C0C0C0C0C0C0C8B
:1015A0000C0C0C0C0C0C0C0C0C0C0C0C0C0C0C0C7B
:1015B0000C0C0C0C0C0C0C0C0C0C0C0C0C0C0C0C6B
:1015C00008080808080808080C0C0C0C0C0C0C0C7B
:1015D0000C0C0C0C0C0C0C0C0C0C0C0C0C0C0C0C4B
:1015E0000C0C0C0C0C0C0C0C0C0C0C0C0C0C0C0C3B
:1015F0000C0C0C0C0C0C0C0C0C0C0C0C0C0C0C0C2B
:1016000008080808080808080C0C0C0C0C0C0C0C3A
:101610000C0C0C0C0C0C0C0C0C0C0C0C0C0C0C0C0A
:101620000C0C0C0C0C0C0C0C0C0C0C0C0C0C0C0CFA
:101630000C0C0C0C0C0C0C0C0C0C0C0C0C0C0C0CEA
:1016400008080808080808080C0C0C0C0C0C0C0CFA
:101650000C0C0C0C0C0C0C0C0C0C0C0C0C0C0C0CCA
:101660000C0C0C0C0C0C0C0C0C0C0C0C0C0C0C0CBA
:101670000C0C0C0C0C0C0C0C0C0C0C0C0C0C0C0CAA
:1016800008080808080808080C0C0C0C0C0C0C0CBA
:101690000C0C0C0C0C0C0C0C0C0C0C0C0C0C0C0C8A
:1016A0000C0C0C0C0C0C0C0C0C0C0C0C0C0C0C0C7A
:1016B0000C0C0C0C0C0C0C0C0C0C0C0C0C0C0C0C6A
:1016C00008080808080808080C0C0C0C0C0C0C0C7A
:1016D0000C0C0C0C0C0C0C0C0C0C0C0C0C0C0C0C4A
:1016E0000C0C0C0C0C0C0C0C0C0C0C0C0C0C0C0C3A
:1016F0000C0C0C0C0C0C0C0C0C0C0C0C0C0C0C0C2A
:1017000008080808080808080C0C0C0C0C0C0C0C39
:101710000C0C0C0C0C0C0C0C0C0C0C0C0C0C0C0C09
:101720000C0C0C0C0C0C0C0C0C0C0C0C0C0C0C0CF9
:101730000C0C0C0C0C0C0C0C0C0C0C0C0C0C0C0CE9
:1017400008080808080808080C0C0C0C0C0C0C0CF9
:101750000C0C0C0C0C0C0C0C0C0C0C0C0C0C0C0CC9
:101760000C0C0C0C0C0C0C0C0C0C0C0C0C0C0C0CB9
:101770000C0C0C0C0C0C0C0C0C0C0C0C0C0C0C0CA9
:1017800008080808080808080C0C0C0C0C0C0C0CB9
:101790000C0C0C0C0C0C0C0C0C0C0C0C0C0C0C0C89
:1017A0000C0C0C0C0C0C0C0C0C0C0C0C0C0C0C0C79
:1017B0000C0C0C0C0C0C0C0C0C0C0C0C0C0C0C0C69
:1017C00008080808080808080C0C0C0C0C0C0C0C79
:1017D0000C0C0C0C0C0C0C0C0C0C0C0C0C0C0C0C49
:1017E0000C0C0C0C0C0C0C0C0C0C0C0C0C0C0C0C39
:1017F0000C0C0C0C0C0C0C0C0C0C0C0C0C0C0C0C29
:1018000008080808080808080C0C0C0C0C0C0C0C38
:101810000C0C0C0C0C0C0C0C0C0C0C0C0C0C0C0C08
:101820000C0C0C0C0C0C0C0C0C0C0C0C0C0C0C0CF8
:101830000C0C0C0C0C0C0C0C0C0C0C0C0C0C0C0CE8
:1018400008080808080808080C0C0C0C0C0C0C0CF8
:101850000C0C0C0C0C0C0C0C0C0C0C0C0C0C0C0CC8
:101860000C0C0C0C0C0C0C0C0C0C0C0C0C0C0C0CB8
:101870000C0C0C0C0C0C0C0C0C0C0C0C0C0C0C0CA8
:1018800008080808080808080C0C0C0C0C0C0C0CB8
:101890000C0C0C0C0C0C0C0C0C0C0C0C0C0C0C0C88
:1018A0000C0C0C0C0C0C0C0C0C0C0C0C0C0C0C0C78
:1018B0000C0C0C0C0C0C0C0C0C0C0C0C0C0C0C0C68
:1018C00008080808080808080C0C0C0C0C0C0C0C78
:1018D0000C0C0C0C0C0C0C0C0C0C0C0C0C0C0C0C48
:1018E0000C0C0C0C0C0C0C0C0C0C0C0C0C0C0C0C38
:1018F0000C0C0C0C0C0C0C0C0C0C0C0C0C0C0C0C28
:1019000008080808080808080C0C0C0C0C0C0C0C37
:101910000C0C0C0C0C0C0C0C0C0C0C0C0C0C0C0C07
:101920000C0C0C0C0C0C0C0C0C0C0C0C0C0C0C0CF7
:101930000C0C0C0C0C0C0C0C0C0C0C0C0C0C0C0CE7
:1019400008080808080808080C0C0C0C0C0C0C0CF7
:101950000C0C0C0C0C0C0C0C0C0C0C0C0C0C0C0CC7
:101960000C0C0C0C0C0C0C0C0C0C0C0C0C0C0C0CB7
:101970000C0C0C0C0C0C0C0C0C0C0C0C0C0C0C0CA7
:1019800008080808080808080C0C0C0C0C0C0C0CB7
:101990000C0C0C0C0C0C0C0C0C0C0C0C0C0C0C0C87
:1019A0000C0C0C0C0C0C0C0C0C0C0C0C0C0C0C0C77
:1019B0000C0C0C0C0C0C0C0C0C0C0C0C0C0C0C0C67
:1019C00008080808080808080C0C0C0C0C0C0C0C77
:1019D0000C0C0C0C0C0C0C0C0C0C0C0C0C0C0C0C47
:1019E0000C0C0C0C0C0C0C0C0C0C0C0C0C0C0C0C37
:1019F0000C0C0C0C0C0C0C0C0C0C0C0C0C0C0C0C27
:101A000008080808080808080C0C0C0C0C0C0C0C36
:101A10000C0C0C0C0C0C0C0C0C0C0C0C0C0C0C0C06
:101A20000C0C0C0C0C0C0C0C0C0C0C0C0C0C0C0CF6
:101A30000C0C0C0C0C0C0C0C0C0C0C0C0C0C0C0CE6
:101A400008080808080808080C0C0C0C0C0C0C0CF6
:101A50000C0C0C0C0C0C0C0C0C0C0C0C0C0C0C0CC6
:101A60000C0C0C0C0C0C0C0C0C0C0C0C0C0C0C0CB6
:101A70000C0C0C0C0C0C0C0C0C0C0C0C0C0C0C0CA6
:101A800008080808080808080C0C0C0C0C0C0C0CB6
:101A90000C0C0C0C0C0C0C0C0C0C0C0C0C0C0C0C86
:101AA0000C0C0C0C0C0C0C0C0C0C0C0C0C0C0C0C76
:101AB0000C0C0C0C0C0C0C0C0C0C0C0C0C0C0C0C66
:101AC00008080808080808080C0C0C0C0C0C0C0C76
:101AD0000C0C0C0C0C0C0C0C0C0C0C0C0C0C0C0C46
:101AE0000C0C0C0C0C0C0C0C0C0C0C0C0C0C0C0C36
:101AF0000C0C0C0C0C0C0C0C0C0C0C0C0C0C0C0C26
:101B000008080808080808080C0C0C0C0C0C0C0C35
:101B10000C0C0C0C0C0C0C0C0C0C0C0C0C0C0C0C05
:101B20000C0C0C0C0C0C0C0C0C0C0C0C0C0C0C0CF5
:101B30000C0C0C0C0C0C0C0C0C0C0C0C0C0C0C0CE5
:101B400008080808080808080C0C0C0C0C0C0C0CF5
:101B50000C0C0C0C0C0C0C0C0C0C0C0C0C0C0C0CC5
:101B60000C0C0C0C0C0C0C0C0C0C0C0C0C0C0C0CB5
:101B70000C0C0C0C0C0C0C0C0C0C0C0C0C0C0C0CA5
:101B800008080808080808080C0C0C0C0C0C0C0CB5
:101B90000C0C0C0C0C0C0C0C0C0C0C0C0C0C0C0C85
:101BA0000C0C0C0C0C0C0C0C0C0C0C0C0C0C0C0C75
:101BB0000C0C0C0C0C0C0C0C0C0C0C0C0C0C0C0C65
:101BC00008080808080808080C0C0C0C0C0C0C0C75
:101BD0000C0C0C0C0C0C0C0C0C0C0C0C0C0C0C0C45
:101BE0000C0C0C0C0C0C0C0C0C0C0C0C0C0C0C0C35
:101BF0000C0C0C0C0C0C0C0C0C0C0C0C0C0C0C0C25
:101C000008080808080808080C0C0C0C0C0C0C0C34
:101C10000C0C0C0C0C0C0C0C0C0C0C0C0C0C0C0C04
:101C20000C0C0C0C0C0C0C0C0C0C0C0C0C0C0C0CF4
:101C30000C0C0C0C0C0C0C0C0C0C0C0C0C0C0C0CE4
:101C400008080808080808080C0C0C0C0C0C0C0CF4
:101C50000C0C0C0C0C0C0C0C0C0C0C0C0C0C0C0CC4
:101C60000C0C0C0C0C0C0C0C0C0C0C0C0C0C0C0CB4
:101C70000C0C0C0C0C0C0C0C0C0C0C0C0C0C0C0CA4
:101C800008080808080808080C0C0C0C0C0C0C0CB4
:101C90000C0C0C0C0C0C0C0C0C0C0C0C0C0C0C0C84
:101CA0000C0C0C0C0C0C0C0C0C0C0C0C0C0C0C0C74
:101CB0000C0C0C0C0C0C0C0C0C0C0C0C0C0C0C0C64
:101CC00008080808080808080C0C0C0C0C0C0C0C74
:101CD0000C0C0C0C0C0C0C0C0C0C0C0C0C0C0C0C44
:101CE0000C0C0C0C0C0C0C0C0C0C0C0C0C0C0C0C34
:101CF0000C0C0C0C0C0C0C0C0C0C0C0C0C0C0C0C24
:101D000008080808080808080C0C0C0C0C0C0C0C33
:101D10000C0C0C0C0C0C0C0C0C0C0C0C0C0C0C0C03
:101D20000C0C0C0C0C0C0C0C0C0C0C0C0C0C0C0CF3
:101D30000C0C0C0C0C0C0C0C0C0C0C0C0C0C0C0CE3
:101D400008080808080808080C0C0C0C0C0C0C0CF3
:101D50000C0C0C0C0C0C0C0C0C0C0C0C0C0C0C0CC3
:101D60000C0C0C0C0C0C0C0C0C0C0C0C0C0C0C0CB3
:101D70000C0C0C0C0C0C0C0C0C0C0C0C0C0C0C0CA3
:101D800008080808080808080C0C0C0C0C0C0C0CB3
:101D90000C0C0C0C0C0C0C0C0C0C0C0C0C0C0C0C83
:101DA0000C0C0C0C0C0C0C0C0C0C0C0C0C0C0C0C73
:101DB0000C0C0C0C0C0C0C0C0C0C0C0C0C0C0C0C63
:101DC00008080808080808080C0C0C0C0C0C0C0C73
:101DD0000C0C0C0C0C0C0C0C0C0C0C0C0C0C0C0C43
:101DE0000C0C0C0C0C0C0C0C0C0C0C0C0C0C0C0C33
:101DF0000C0C0C0C0C0C0C0C0C0C0C0C0C0C0C0C23
:101E000008080808080808080C0C0C0C0C0C0C0C32
:101E10000C0C0C0C0C0C0C0C0C0C0C0C0C0C0C0C02
:101E20000C0C0C0C0C0C0C0C0C0C0C0C0C0C0C0CF2
:101E30000C0C0C0C0C0C0C0C0C0C0C0C0C0C0C0CE2
:101E400008080808080808080C0C0C0C0C0C0C0CF2
:101E50000C0C0C0C0C0C0C0C0C0C0C0C0C0C0C0CC2
:101E60000C0C0C0C0C0C0C0C0C0C0C0C0C0C0C0CB2
:101E70000C0C0C0C0C0C0C0C0C0C0C0C0C0C0C0CA2
:101E800008080808080808080C0C0C0C0C0C0C0CB2
:101E90000C0C0C0C0C0C0C0C0C0C0C0C0C0C0C0C82
:101EA0000C0C0C0C0C0C0C0C0C0C0C0C0C0C0C0C72
:101EB0000C0C0C0C0C0C0C0C0C0C0C0C0C0C0C0C62
:101EC00008080808080808080C0C0C0C0C0C0C0C72
:101ED0000C0C0C0C0C0C0C0C0C0C0C0C0C0C0C0C42
:101EE0000C0C0C0C0C0C0C0C0C0C0C0C0C0C0C0C32
:101EF0000C0C0C0C0C0C0C0C0C0C0C0C0C0C0C0C22
:101F000008080808080808080C0C0C0C0C0C0C0C31
:101F10000C0C0C0C0C0C0C0C0C0C0C0C0C0C0C0C01
:101F20000C0C0C0C0C0C0C0C0C0C0C0C0C0C0C0CF1
:101F30000C0C0C0C0C0C0C0C0C0C0C0C0C0C0C0CE1
:101F400008080808080808080C0C0C0C0C0C0C0CF1
:101F50000C0C0C0C0C0C0C0C0C0C0C0C0C0C0C0CC1
:101F60000C0C0C0C0C0C0C0C0C0C0C0C0C0C0C0CB1
:101F70000C0C0C0C0C0C0C0C0C0C0C0C0C0C0C0CA1
:101F800008080808080808080C0C0C0C0C0C0C0CB1
:101F90000C0C0C0C0C0C0C0C0C0C0C0C0C0C0C0C81
:101FA0000C0C0C0C0C0C0C0C0C0C0C0C0C0C0C0C71
:101FB0000C0C0C0C0C0C0C0C0C0C0C0C0C0C0C0C61
:101FC00008080808080808080C0C0C0C0C0C0C0C71
:101FD0000C0C0C0C0C0C0C0C0C0C0C0C0C0C0C0C41
:101FE0000C0C0C0C0C0C0C0C0C0C0C0C0C0C0C0C31
:101FF0000C0C0C0C0C0C0C0C0C0C0C0C0C0C0C0C21
:1020000008080808080808080C0C0C0C0C0C0C0C30
:102010000C0C0C0C0C0C0C0C0C0C0C0C0C0C0C0C00
:102020000C0C0C0C0C0C0C0C0C0C0C0C0C0C0C0CF0
:102030000C0C0C0C0C0C0C0C0C0C0C0C0C0C0C0CE0
:1020400008080808080808080C0C0C0C0C0C0C0CF0
:102050000C0C0C0C0C0C0C0C0C0C0C0C0C0C0C0CC0
:102060000C0C0C0C0C0C0C0C0C0C0C0C0C0C0C0CB0
:102070000C0C0C0C0C0C0C0C0C0C0C0C0C0C0C0CA0
:1020800008080808080808080C0C0C0C0C0C0C0CB0
:102090000C0C0C0C0C0C0C0C0C0C0C0C0C0C0C0C80
:1020A0000C0C0C0C0C0C0C0C0C0C0C0C0C0C0C0C70
:1020B0000C0C0C0C0C0C0C0C0C0C0C0C0C0C0C0C60
:1020C00008080808080808080C0C0C0C0C0C0C0C70
:1020D0000C0C0C0C0C0C0C0C0C0C0C0C0C0C0C0C40
:1020E0000C0C0C0C0C0C0C0C0C0C0C0C0C0C0C0C30
:1020F0000C0C0C0C0C0C0C0C0C0C0C0C0C0C0C0C20
:1021000008080808080808080C0C0C0C0C0C0C0C2F
:102110000C0C0C0C0C0C0C0C0C0C0C0C0C0C0C0CFF
:102120000C0C0C0C0C0C0C0C0C0C0C0C0C0C0C0CEF
:102130000C0C0C0C0C0C0C0C0C0C0C0C0C0C0C0CDF
:1021400008080808080808080C0C0C0C0C0C0C0CEF
:102150000C0C0C0C0C0C0C0C0C0C0C0C0C0C0C0CBF
:102160000C0C0C0C0C0C0C0C0C0C0C0C0C0C0C0CAF
:102170000C0C0C0C0C0C0C0C0C0C0C0C0C0C0C0C9F
:1021800008080808080808080C0C0C0C0C0C0C0CAF
:102190000C0C0C0C0C0C0C0C0C0C0C0C0C0C0C0C7F
:1021A0000C0C0C0C0C0C0C0C0C0C0C0C0C0C0C0C6F
:1021B0000C0C0C0C0C0C0C0C0C0C0C0C0C0C0C0C5F
:1021C00008080808080808080C0C0C0C0C0C0C0C6F
:1021D0000C0C0C0C0C0C0C0C0C0C0C0C0C0C0C0C3F
:1021E0000C0C0C0C0C0C0C0C0C0C0C0C0C0C0C0C2F
:1021F0000C0C0C0C0C0C0C0C0C0C0C0C0C0C0C0C1F
:1022000008080808080808080C0C0C0C0C0C0C0C2E
:102210000C0C0C0C0C0C0C0C0C0C0C0C0C0C0C0CFE
:102220000C0C0C0C0C0C0C0C0C0C0C0C0C0C0C0CEE
:102230000C0C0C0C0C0C0C0C0C0C0C0C0C0C0C0CDE
:1022400008080808080808080C0C0C0C0C0C0C0CEE
:102250000C0C0C0C0C0C0C0C0C0C0C0C0C0C0C0CBE
:102260000C0C0C0C0C0C0C0C0C0C0C0C0C0C0C0CAE
:102270000C0C0C0C0C0C0C0C0C0C0C0C0C0C0C0C9E
:1022800008080808080808080C0C0C0C0C0C0C0CAE
:102290000C0C0C0C0C0C0C0C0C0C0C0C0C0C0C0C7E
:1022A0000C0C0C0C0C0C0C0C0C0C0C0C0C0C0C0C6E
:1022B0000C0C0C0C0C0C0C0C0C0C0C0C0C0C0C0C5E
:1022C00008080808080808080C0C0C0C0C0C0C0C6E
:1022D0000C0C0C0C0C0C0C0C0C0C0C0C0C0C0C0C3E
:1022E0000C0C0C0C0C0C0C0C0C0C0C0C0C0C0C0C2E
:1022F0000C0C0C0C0C0C0C0C0C0C0C0C0C0C0C0C1E
:1023000008080808080808080C0C0C0C0C0C0C0C2D
:102310000C0C0C0C0C0C0C0C0C0C0C0C0C0C0C0CFD
:102320000C0C0C0C0C0C0C0C0C0C0C0C0C0C0C0CED
:102330000C0C0C0C0C0C0C0C0C0C0C0C0C0C0C0CDD
:1023400008080808080808080C0C0C0C0C0C0C0CED
:102350000C0C0C0C0C0C0C0C0C0C0C0C0C0C0C0CBD
:102360000C0C0C0C0C0C0C0C0C0C0C0C0C0C0C0CAD
:102370000C0C0C0C0C0C0C0C0C0C0C0C0C0C0C0C9D
:1023800008080808080808080C0C0C0C0C0C0C0CAD
:102390000C0C0C0C0C0C0C0C0C0C0C0C0C0C0C0C7D
:1023A0000C0C0C0C0C0C0C0C0C0C0C0C0C0C0C0C6D
:1023B0000C0C0C0C0C0C0C0C0C0C0C0C0C0C0C0C5D
:1023C00008080808080808080C0C0C0C0C0C0C0C6D
:1023D0000C0C0C0C0C0C0C0C0C0C0C0C0C0C0C0C3D
:1023E0000C0C0C0C0C0C0C0C0C0C0C0C0C0C0C0C2D
:1023F0000C0C0C0C0C0C0C0C0C0C0C0C0C0C0C0C1D
:1024000008080808080808080C0C0C0C0C0C0C0C2C
:102410000C0C0C0C0C0C0C0C0C0C0C0C0C0C0C0CFC
:102420000C0C0C0C0C0C0C0C0C0C0C0C0C0C0C0CEC
:102430000C0C0C0C0C0C0C0C0C0C0C0C0C0C0C0CDC
:1024400008080808080808080C0C0C0C0C0C0C0CEC
:102450000C0C0C0C0C0C0C0C0C0C0C0C0C0C0C0CBC
:102460000C0C0C0C0C0C0C0C0C0C0C0C0C0C0C0CAC
:102470000C0C0C0C0C0C0C0C0C0C0C0C0C0C0C0C9C
:1024800008080808080808080C0C0C0C0C0C0C0CAC
:102490000C0C0C0C0C0C0C0C0C0C0C0C0C0C0C0C7C
:1024A0000C0C0C0C0C0C0C0C0C0C0C0C0C0C0C0C6C
:1024B0000C0C0C0C0C0C0C0C0C0C0C0C0C0C0C0C5C
:1024C00008080808080808080C0C0C0C0C0C0C0C6C
:1024D0000C0C0C0C0C0C0C0C0C0C0C0C0C0C0C0C3C
:1024E0000C0C0C0C0C0C0C0C0C0C0C0C0C0C0C0C2C
:1024F0000C0C0C0C0C0C0C0C0C0C0C0C0C0C0C0C1C
:1025000008080808080808080C0C0C0C0C0C0C0C2B
:102510000C0C0C0C0C0C0C0C0C0C0C0C0C0C0C0CFB
:102520000C0C0C0C0C0C0C0C0C0C0C0C0C0C0C0CEB
:102530000C0C0C0C0C0C0C0C0C0C0C0C0C0C0C0CDB
:1025400008080808080808080C0C0C0C0C0C0C0CEB
:102550000C0C0C0C0C0C0C0C0C0C0C0C0C0C0C0CBB
:102560000C0C0C0C0C0C0C0C0C0C0C0C0C0C0C0CAB
:102570000C0C0C0C0C0C0C0C0C0C0C0C0C0C0C0C9B
:1025800008080808080808080C0C0C0C0C0C0C0CAB
:102590000C0C0C0C0C0C0C0C0C0C0C0C0C0C0C0C7B
:1025A0000C0C0C0C0C0C0C0C0C0C0C0C0C0C0C0C6B
:1025B0000C0C0C0C0C0C0C0C0C0C0C0C0C0C0C0C5B
:1025C00008080808080808080C0C0C0C0C0C0C0C6B
:1025D0000C0C0C0C0C0C0C0C0C0C0C0C0C0C0C0C3B
:1025E0000C0C0C0C0C0C0C0C0C0C0C0C0C0C0C0C2B
:1025F0000C0C0C0C0C0C0C0C0C0C0C0C0C0C0C0C1B
:1026000008080808080808080C0C0C0C0C0C0C0C2A
:102610000C0C0C0C0C0C0C0C0C0C0C0C0C0C0C0CFA
:102620000C0C0C0C0C0C0C0C0C0C0C0C0C0C0C0CEA
:102630000C0C0C0C0C0C0C0C0C0C0C0C0C0C0C0CDA
:1026400008080808080808080C0C0C0C0C0C0C0CEA
:102650000C0C0C0C0C0C0C0C0C0C0C0C0C0C0C0CBA
:102660000C0C0C0C0C0C0C0C0C0C0C0C0C0C0C0CAA
:102670000C0C0C0C0C0C0C0C0C0C0C0C0C0C0C0C9A
:1026800008080808080808080C0C0C0C0C0C0C0CAA
:102690000C0C0C0C0C0C0C0C0C0C0C0C0C0C0C0C7A
:1026A0000C0C0C0C0C0C0C0C0C0C0C0C0C0C0C0C6A
:1026B0000C0C0C0C0C0C0C0C0C0C0C0C0C0C0C0C5A
:1026C00008080808080808080C0C0C0C0C0C0C0C6A
:1026D0000C0C0C0C0C0C0C0C0C0C0C0C0C0C0C0C3A
:1026E0000C0C0C0C0C0C0C0C0C0C0C0C0C0C0C0C2A
:1026F0000C0C0C0C0C0C0C0C0C0C0C0C0C0C0C0C1A
:1027000008080808080808080C0C0C0C0C0C0C0C29
:102710000C0C0C0C0C0C0C0C0C0C0C0C0C0C0C0CF9
:102720000C0C0C0C0C0C0C0C0C0C0C0C0C0C0C0CE9
:102730000C0C0C0C0C0C0C0C0C0C0C0C0C0C0C0CD9
:1027400008080808080808080C0C0C0C0C0C0C0CE9
:102750000C0C0C0C0C0C0C0C0C0C0C0C0C0C0C0CB9
:102760000C0C0C0C0C0C0C0C0C0C0C0C0C0C0C0CA9
:102770000C0C0C0C0C0C0C0C0C0C0C0C0C0C0C0C99
:1027800008080808080808080C0C0C0C0C0C0C0CA9
:102790000C0C0C0C0C0C0C0C0C0C0C0C0C0C0C0C79
:1027A0000C0C0C0C0C0C0C0C0C0C0C0C0C0C0C0C69
:1027B0000C0C0C0C0C0C0C0C0C0C0C0C0C0C0C0C59
:1027C00008080808080808080C0C0C0C0C0C0C0C69
:1027D0000C0C0C0C0C0C0C0C0C0C0C0C0C0C0C0C39
:1027E0000C0C0C0C0C0C0C0C0C0C0C0C0C0C0C0C29
:1027F0000C0C0C0C0C0C0C0C0C0C0C0C0C0C0C0C19
:1028000008080808080808080C0C0C0C0C0C0C0C28
:102810000C0C0C0C0C0C0C0C0C0C0C0C0C0C0C0CF8
:102820000C0C0C0C0C0C0C0C0C0C0C0C0C0C0C0CE8
:102830000C0C0C0C0C0C0C0C0C0C0C0C0C0C0C0CD8
:1028400008080808080808080C0C0C0C0C0C0C0CE8
:102850000C0C0C0C0C0C0C0C0C0C0C0C0C0C0C0CB8
:102860000C0C0C0C0C0C0C0C0C0C0C0C0C0C0C0CA8
:102870000C0C0C0C0C0C0C0C0C0C0C0C0C0C0C0C98
:1028800008080808080808080C0C0C0C0C0C0C0CA8
:102890000C0C0C0C0C0C0C0C0C0C0C0C0C0C0C0C78
:1028A0000C0C0C0C0C0C0C0C0C0C0C0C0C0C0C0C68
:1028B0000C0C0C0C0C0C0C0C0C0C0C0C0C0C0C0C58
:1028C00008080808080808080C0C0C0C0C0C0C0C68
:1028D0000C0C0C0C0C0C0C0C0C0C0C0C0C0C0C0C38
:1028E0000C0C0C0C0C0C0C0C0C0C0C0C0C0C0C0C28
:1028F0000C0C0C0C0C0C0C0C0C0C0C0C0C0C0C0C18
:1029000008080808080808080C0C0C0C0C0C0C0C27
:102910000C0C0C0C0C0C0C0C0C0C0C0C0C0C0C0CF7
:102920000C0C0C0C0C0C0C0C0C0C0C0C0C0C0C0CE7
:102930000C0C0C0C0C0C0C0C0C0C0C0C0C0C0C0CD7
:1029400008080808080808080C0C0C0C0C0C0C0CE7
:102950000C0C0C0C0C0C0C0C0C0C0C0C0C0C0C0CB7
:102960000C0C0C0C0C0C0C0C0C0C0C0C0C0C0C0CA7
:102970000C0C0C0C0C0C0C0C0C0C0C0C0C0C0C0C97
:1029800008080808080808080C0C0C0C0C0C0C0CA7
:102990000C0C0C0C0C0C0C0C0C0C0C0C0C0C0C0C77
:1029A0000C0C0C0C0C0C0C0C0C0C0C0C0C0C0C0C67
:1029B0000C0C0C0C0C0C0C0C0C0C0C0C0C0C0C0C57
:1029C00008080808080808080C0C0C0C0C0C0C0C67
:1029D0000C0C0C0C0C0C0C0C0C0C0C0C0C0C0C0C37
:1029E0000C0C0C0C0C0C0C0C0C0C0C0C0C0C0C0C27
:1029F0000C0C0C0C0C0C0C0C0C0C0C0C0C0C0C0C17
:102A000008080808080808080C0C0C0C0C0C0C0C26
:102A10000C0C0C0C0C0C0C0C0C0C0C0C0C0C0C0CF6
:102A20000C0C0C0C0C0C0C0C0C0C0C0C0C0C0C0CE6
:102A30000C0C0C0C0C0C0C0C0C0C0C0C0C0C0C0CD6
:102A400008080808080808080C0C0C0C0C0C0C0CE6
:102A50000C0C0C0C0C0C0C0C0C0C0C0C0C0C0C0CB6
:102A60000C0C0C0C0C0C0C0C0C0C0C0C0C0C0C0CA6
:102A70000C0C0C0C0C0C0C0C0C0C0C0C0C0C0C0C96
:102A800008080808080808080C0C0C0C0C0C0C0CA6
:102A90000C0C0C0C0C0C0C0C0C0C0C0C0C0C0C0C76
:102AA0000C0C0C0C0C0C0C0C0C0C0C0C0C0C0C0C66
:102AB0000C0C0C0C0C0C0C0C0C0C0C0C0C0C0C0C56
:102AC00008080808080808080C0C0C0C0C0C0C0C66
:102AD0000C0C0C0C0C0C0C0C0C0C0C0C0C0C0C0C36
:102AE0000C0C0C0C0C0C0C0C0C0C0C0C0C0C0C0C26
:102AF0000C0C0C0C0C0C0C0C0C0C0C0C0C0C0C0C16
:102B000008080808080808080C0C0C0C0C0C0C0C25
:102B10000C0C0C0C0C0C0C0C0C0C0C0C0C0C0C0CF5
:102B20000C0C0C0C0C0C0C0C0C0C0C0C0C0C0C0CE5
:102B30000C0C0C0C0C0C0C0C0C0C0C0C0C0C0C0CD5
:102B400008080808080808080C0C0C0C0C0C0C0CE5
:102B50000C0C0C0C0C0C0C0C0C0C0C0C0C0C0C0CB5
:102B60000C0C0C0C0C0C0C0C0C0C0C0C0C0C0C0CA5
:102B70000C0C0C0C0C0C0C0C0C0C0C0C0C0C0C0C95
:102B800008080808080808080C0C0C0C0C0C0C0CA5
:102B90000C0C0C0C0C0C0C0C0C0C0C0C0C0C0C0C75
:102BA0000C0C0C0C0C0C0C0C0C0C0C0C0C0C0C0C65
:102BB0000C0C0C0C0C0C0C0C0C0C0C0C0C0C0C0C55
:102BC00008080808080808080C0C0C0C0C0C0C0C65
:102BD0000C0C0C0C0C0C0C0C0C0C0C0C0C0C0C0C35
:102BE0000C0C0C0C0C0C0C0C0C0C0C0C0C0C0C0C25
:102BF0000C0C0C0C0C0C0C0C0C0C0C0C0C0C0C0C15
:102C000008080808080808080C0C0C0C0C0C0C0C24
:102C10000C0C0C0C0C0C0C0C0C0C0C0C0C0C0C0CF4
:102C20000C0C0C0C0C0C0C0C0C0C0C0C0C0C0C0CE4
:102C30000C0C0C0C0C0C0C0C0C0C0C0C0C0C0C0CD4
:102C400008080808080808080C0C0C0C0C0C0C0CE4
:102C50000C0C0C0C0C0C0C0C0C0C0C0C0C0C0C0CB4
:102C60000C0C0C0C0C0C0C0C0C0C0C0C0C0C0C0CA4
:102C70000C0C0C0C0C0C0C0C0C0C0C0C0C0C0C0C94
:102C800008080808080808080C0C0C0C0C0C0C0CA4
:102C90000C0C0C0C0C0C0C0C0C0C0C0C0C0C0C0C74
:102CA0000C0C0C0C0C0C0C0C0C0C0C0C0C0C0C0C64
:102CB0000C0C0C0C0C0C0C0C0C0C0C0C0C0C0C0C54
:102CC00008080808080808080C0C0C0C0C0C0C0C64
:102CD0000C0C0C0C0C0C0C0C0C0C0C0C0C0C0C0C34
:102CE0000C0C0C0C0C0C0C0C0C0C0C0C0C0C0C0C24
:102CF0000C0C0C0C0C0C0C0C0C0C0C0C0C0C0C0C14
:102D000008080808080808080C0C0C0C0C0C0C0C23
:102D10000C0C0C0C0C0C0C0C0C0C0C0C0C0C0C0CF3
:102D20000C0C0C0C0C0C0C0C0C0C0C0C0C0C0C0CE3
:102D30000C0C0C0C0C0C0C0C0C0C0C0C0C0C0C0CD3
:102D400008080808080808080C0C0C0C0C0C0C0CE3
:102D50000C0C0C0C0C0C0C0C0C0C0C0C0C0C0C0CB3
:102D60000C0C0C0C0C0C0C0C0C0C0C0C0C0C0C0CA3
:102D70000C0C0C0C0C0C0C0C0C0C0C0C0C0C0C0C93
:102D800008080808080808080C0C0C0C0C0C0C0CA3
:102D90000C0C0C0C0C0C0C0C0C0C0C0C0C0C0C0C73
:102DA0000C0C0C0C0C0C0C0C0C0C0C0C0C0C0C0C63
:102DB0000C0C0C0C0C0C0C0C0C0C0C0C0C0C0C0C53
:102DC00008080808080808080C0C0C0C0C0C0C0C63
:102DD0000C0C0C0C0C0C0C0C0C0C0C0C0C0C0C0C33
:102DE0000C0C0C0C0C0C0C0C0C0C0C0C0C0C0C0C23
:102DF0000C0C0C0C0C0C0C0C0C0C0C0C0C0C0C0C13
:102E000008080808080808080C0C0C0C0C0C0C0C22
:102E10000C0C0C0C0C0C0C0C0C0C0C0C0C0C0C0CF2
:102E20000C0C0C0C0C0C0C0C0C0C0C0C0C0C0C0CE2
:102E30000C0C0C0C0C0C0C0C0C0C0C0C0C0C0C0CD2
:102E400008080808080808080C0C0C0C0C0C0C0CE2
:102E50000C0C0C0C0C0C0C0C0C0C0C0C0C0C0C0CB2
:102E60000C0C0C0C0C0C0C0C0C0C0C0C0C0C0C0CA2
:102E70000C0C0C0C0C0C0C0C0C0C0C0C0C0C0C0C92
:102E800008080808080808080C0C0C0C0C0C0C0CA2
:102E90000C0C0C0C0C0C0C0C0C0C0C0C0C0C0C0C72
:102EA0000C0C0C0C0C0C0C0C0C0C0C0C0C0C0C0C62
:102EB0000C0C0C0C0C0C0C0C0C0C0C0C0C0C0C0C52
:102EC00008080808080808080C0C0C0C0C0C0C0C62
:102ED0000C0C0C0C0C0C0C0C0C0C0C0C0C0C0C0C32
:102EE0000C0C0C0C0C0C0C0C0C0C0C0C0C0C0C0C22
:102EF0000C0C0C0C0C0C0C0C0C0C0C0C0C0C0C0C12
:102F000008080808080808080C0C0C0C0C0C0C0C21
:102F10000C0C0C0C0C0C0C0C0C0C0C0C0C0C0C0CF1
:102F20000C0C0C0C0C0C0C0C0C0C0C0C0C0C0C0CE1
:102F30000C0C0C0C0C0C0C0C0C0C0C0C0C0C0C0CD1
:102F400008080808080808080C0C0C0C0C0C0C0CE1
:102F50000C0C0C0C0C0C0C0C0C0C0C0C0C0C0C0CB1
:102F60000C0C0C0C0C0C0C0C0C0C0C0C0C0C0C0CA1
:102F70000C0C0C0C0C0C0C0C0C0C0C0C0C0C0C0C91
:102F800008080808080808080C0C0C0C0C0C0C0CA1
:102F90000C0C0C0C0C0C0C0C0C0C0C0C0C0C0C0C71
:102FA0000C0C0C0C0C0C0C0C0C0C0C0C0C0C0C0C61
:102FB0000C0C0C0C0C0C0C0C0C0C0C0C0C0C0C0C51
:102FC00008080808080808080C0C0C0C0C0C0C0C61
:102FD0000C0C0C0C0C0C0C0C0C0C0C0C0C0C0C0C31
:102FE0000C0C0C0C0C0C0C0C0C0C0C0C0C0C0C0C21
:102FF0000C0C0C0C0C0C0C0C0C0C0C0C0C0C0C0C11
:1030000008080808080808080C0C0C0C0C0C0C0C20
:103010000C0C0C0C0C0C0C0C0C0C0C0C0C0C0C0CF0
:103020000C0C0C0C0C0C0C0C0C0C0C0C0C0C0C0CE0
:103030000C0C0C0C0C0C0C0C0C0C0C0C0C0C0C0CD0
:1030400008080808080808080C0C0C0C0C0C0C0CE0
:103050000C0C0C0C0C0C0C0C0C0C0C0C0C0C0C0CB0
:103060000C0C0C0C0C0C0C0C0C0C0C0C0C0C0C0CA0
:103070000C0C0C0C0C0C0C0C0C0C0C0C0C0C0C0C90
:1030800008080808080808080C0C0C0C0C0C0C0CA0
:103090000C0C0C0C0C0C0C0C0C0C0C0C0C0C0C0C70
:1030A0000C0C0C0C0C0C0C0C0C0C0C0C0C0C0C0C60
:1030B0000C0C0C0C0C0C0C0C0C0C0C0C0C0C0C0C50
:1030C00008080808080808080C0C0C0C0C0C0C0C60
:1030D0000C0C0C0C0C0C0C0C0C0C0C0C0C0C0C0C30
:1030E0000C0C0C0C0C0C0C0C0C0C0C0C0C0C0C0C20
:1030F0000C0C0C0C0C0C0C0C0C0C0C0C0C0C0C0C10
:1031000008080808080808080C0C0C0C0C0C0C0C1F
:103110000C0C0C0C0C0C0C0C0C0C0C0C0C0C0C0CEF
:103120000C0C0C0C0C0C0C0C0C0C0C0C0C0C0C0CDF
:103130000C0C0C0C0C0C0C0C0C0C0C0C0C0C0C0CCF
:1031400008080808080808080C0C0C0C0C0C0C0CDF
:103150000C0C0C0C0C0C0C0C0C0C0C0C0C0C0C0CAF
:103160000C0C0C0C0C0C0C0C0C0C0C0C0C0C0C0C9F
:103170000C0C0C0C0C0C0C0C0C0C0C0C0C0C0C0C8F
:1031800008080808080808080C0C0C0C0C0C0C0C9F
:103190000C0C0C0C0C0C0C0C0C0C0C0C0C0C0C0C6F
:1031A0000C0C0C0C0C0C0C0C0C0C0C0C0C0C0C0C5F
:1031B0000C0C0C0C0C0C0C0C0C0C0C0C0C0C0C0C4F
:1031C00008080808080808080C0C0C0C0C0C0C0C5F
:1031D0000C0C0C0C0C0C0C0C0C0C0C0C0C0C0C0C2F
:1031E0000C0C0C0C0C0C0C0C0C0C0C0C0C0C0C0C1F
:1031F0000C0C0C0C0C0C0C0C0C0C0C0C0C0C0C0C0F
:1032000008080808080808080C0C0C0C0C0C0C0C1E
:103210000C0C0C0C0C0C0C0C0C0C0C0C0C0C0C0CEE
:103220000C0C0C0C0C0C0C0C0C0C0C0C0C0C0C0CDE
:103230000C0C0C0C0C0C0C0C0C0C0C0C0C0C0C0CCE
:1032400008080808080808080C0C0C0C0C0C0C0CDE
:103250000C0C0C0C0C0C0C0C0C0C0C0C0C0C0C0CAE
:103260000C0C0C0C0C0C0C0C0C0C0C0C0C0C0C0C9E
:103270000C0C0C0C0C0C0C0C0C0C0C0C0C0C0C0C8E
:1032800008080808080808080C0C0C0C0C0C0C0C9E
:103290000C0C0C0C0C0C0C0C0C0C0C0C0C0C0C0C6E
:1032A0000C0C0C0C0C0C0C0C0C0C0C0C0C0C0C0C5E
:1032B0000C0C0C0C0C0C0C0C0C0C0C0C0C0C0C0C4E
:1032C00008080808080808080C0C0C0C0C0C0C0C5E
:1032D0000C0C0C0C0C0C0C0C0C0C0C0C0C0C0C0C2E
:1032E0000C0C0C0C0C0C0C0C0C0C0C0C0C0C0C0C1E
:1032F0000C0C0C0C0C0C0C0C0C0C0C0C0C0C0C0C0E
:1033000008080808080808080C0C0C0C0C0C0C0C1D
:103310000C0C0C0C0C0C0C0C0C0C0C0C0C0C0C0CED
:103320000C0C0C0C0C0C0C0C0C0C0C0C0C0C0C0CDD
:103330000C0C0C0C0C0C0C0C0C0C0C0C0C0C0C0CCD
:1033400008080808080808080C0C0C0C0C0C0C0CDD
:103350000C0C0C0C0C0C0C0C0C0C0C0C0C0C0C0CAD
:103360000C0C0C0C0C0C0C0C0C0C0C0C0C0C0C0C9D
:103370000C0C0C0C0C0C0C0C0C0C0C0C0C0C0C0C8D
:1033800008080808080808080C0C0C0C0C0C0C0C9D
:103390000C0C0C0C0C0C0C0C0C0C0C0C0C0C0C0C6D
:1033A0000C0C0C0C0C0C0C0C0C0C0C0C0C0C0C0C5D
:1033B0000C0C0C0C0C0C0C0C0C0C0C0C0C0C0C0C4D
:1033C00008080808080808080C0C0C0C0C0C0C0C5D
:1033D0000C0C0C0C0C0C0C0C0C0C0C0C0C0C0C0C2D
:1033E0000C0C0C0C0C0C0C0C0C0C0C0C0C0C0C0C1D
:1033F0000C0C0C0C0C0C0C0C0C0C0C0C0C0C0C0C0D
:1034000008080808080808080C0C0C0C0C0C0C0C1C
:103410000C0C0C0C0C0C0C0C0C0C0C0C0C0C0C0CEC
:103420000C0C0C0C0C0C0C0C0C0C0C0C0C0C0C0CDC
:103430000C0C0C0C0C0C0C0C0C0C0C0C0C0C0C0CCC
:1034400008080808080808080C0C0C0C0C0C0C0CDC
:103450000C0C0C0C0C0C0C0C0C0C0C0C0C0C0C0CAC
:103460000C0C0C0C0C0C0C0C0C0C0C0C0C0C0C0C9C
:103470000C0C0C0C0C0C0C0C0C0C0C0C0C0C0C0C8C
:1034800008080808080808080C0C0C0C0C0C0C0C9C
:103490000C0C0C0C0C0C0C0C0C0C0C0C0C0C0C0C6C
:1034A0000C0C0C0C0C0C0C0C0C0C0C0C0C0C0C0C5C
:1034B0000C0C0C0C0C0C0C0C0C0C0C0C0C0C0C0C4C
:1034C00008080808080808080C0C0C0C0C0C0C0C5C
:1034D0000C0C0C0C0C0C0C0C0C0C0C0C0C0C0C0C2C
:1034E0000C0C0C0C0C0C0C0C0C0C0C0C0C0C0C0C1C
:1034F0000C0C0C0C0C0C0C0C0C0C0C0C0C0C0C0C0C
:1035000008080808080808080C0C0C0C0C0C0C0C1B
:103510000C0C0C0C0C0C0C0C0C0C0C0C0C0C0C0CEB
:103520000C0C0C0C0C0C0C0C0C0C0C0C0C0C0C0CDB
:103530000C0C0C0C0C0C0C0C0C0C0C0C0C0C0C0CCB
:1035400008080808080808080C0C0C0C0C0C0C0CDB
:103550000C0C0C0C0C0C0C0C0C0C0C0C0C0C0C0CAB
:103560000C0C0C0C0C0C0C0C0C0C0C0C0C0C0C0C9B
:103570000C0C0C0C0C0C0C0C0C0C0C0C0C0C0C0C8B
:1035800008080808080808080C0C0C0C0C0C0C0C9B
:103590000C0C0C0C0C0C0C0C0C0C0C0C0C0C0C0C6B
:1035A0000C0C0C0C0C0C0C0C0C0C0C0C0C0C0C0C5B
:1035B0000C0C0C0C0C0C0C0C0C0C0C0C0C0C0C0C4B
:1035C00008080808080808080C0C0C0C0C0C0C0C5B
:1035D0000C0C0C0C0C0C0C0C0C0C0C0C0C0C0C0C2B
:1035E0000C0C0C0C0C0C0C0C0C0C0C0C0C0C0C0C1B
:1035F0000C0C0C0C0C0C0C0C0C0C0C0C0C0C0C0C0B
:1036000008080808080808080C0C0C0C0C0C0C0C1A
:103610000C0C0C0C0C0C0C0C0C0C0C0C0C0C0C0CEA
:103620000C0C0C0C0C0C0C0C0C0C0C0C0C0C0C0CDA
:103630000C0C0C0C0C0C0C0C0C0C0C0C0C0C0C0CCA
:1036400008080808080808080C0C0C0C0C0C0C0CDA
:103650000C0C0C0C0C0C0C0C0C0C0C0C0C0C0C0CAA
:103660000C0C0C0C0C0C0C0C0C0C0C0C0C0C0C0C9A
:103670000C0C0C0C0C0C0C0C0C0C0C0C0C0C0C0C8A
:1036800008080808080808080C0C0C0C0C0C0C0C9A
:103690000C0C0C0C0C0C0C0C0C0C0C0C0C0C0C0C6A
:1036A0000C0C0C0C0C0C0C0C0C0C0C0C0C0C0C0C5A
:1036B0000C0C0C0C0C0C0C0C0C0C0C0C0C0C0C0C4A
:1036C00008080808080808080C0C0C0C0C0C0C0C5A
:1036D0000C0C0C0C0C0C0C0C0C0C0C0C0C0C0C0C2A
:1036E0000C0C0C0C0C0C0C0C0C0C0C0C0C0C0C0C1A
:1036F0000C0C0C0C0C0C0C0C0C0C0C0C0C0C0C0C0A
:1037000008080808080808080C0C0C0C0C0C0C0C19
:103710000C0C0C0C0C0C0C0C0C0C0C0C0C0C0C0CE9
:103720000C0C0C0C0C0C0C0C0C0C0C0C0C0C0C0CD9
:103730000C0C0C0C0C0C0C0C0C0C0C0C0C0C0C0CC9
:1037400008080808080808080C0C0C0C0C0C0C0CD9
:103750000C0C0C0C0C0C0C0C0C0C0C0C0C0C0C0CA9
:103760000C0C0C0C0C0C0C0C0C0C0C0C0C0C0C0C99
:103770000C0C0C0C0C0C0C0C0C0C0C0C0C0C0C0C89
:1037800008080808080808080C0C0C0C0C0C0C0C99
:103790000C0C0C0C0C0C0C0C0C0C0C0C0C0C0C0C69
:1037A0000C0C0C0C0C0C0C0C0C0C0C0C0C0C0C0C59
:1037B0000C0C0C0C0C0C0C0C0C0C0C0C0C0C0C0C49
:1037C00008080808080808080C0C0C0C0C0C0C0C59
:1037D0000C0C0C0C0C0C0C0C0C0C0C0C0C0C0C0C29
:1037E0000C0C0C0C0C0C0C0C0C0C0C0C0C0C0C0C19
:1037F0000C0C0C0C0C0C0C0C0C0C0C0C0C0C0C0C09
:1038000008080808080808080C0C0C0C0C0C0C0C18
:103810000C0C0C0C0C0C0C0C0C0C0C0C0C0C0C0CE8
:103820000C0C0C0C0C0C0C0C0C0C0C0C0C0C0C0CD8
:103830000C0C0C0C0C0C0C0C0C0C0C0C0C0C0C0CC8
:1038400008080808080808080C0C0C0C0C0C0C0CD8
:103850000C0C0C0C0C0C0C0C0C0C0C0C0C0C0C0CA8
:103860000C0C0C0C0C0C0C0C0C0C0C0C0C0C0C0C98
:103870000C0C0C0C0C0C0C0C0C0C0C0C0C0C0C0C88
:1038800008080808080808080C0C0C0C0C0C0C0C98
:103890000C0C0C0C0C0C0C0C0C0C0C0C0C0C0C0C68
:1038A0000C0C0C0C0C0C0C0C0C0C0C0C0C0C0C0C58
:1038B0000C0C0C0C0C0C0C0C0C0C0C0C0C0C0C0C48
:1038C00008080808080808080C0C0C0C0C0C0C0C58
:1038D0000C0C0C0C0C0C0C0C0C0C0C0C0C0C0C0C28
:1038E0000C0C0C0C0C0C0C0C0C0C0C0C0C0C0C0C18
:1038F0000C0C0C0C0C0C0C0C0C0C0C0C0C0C0C0C08
:1039000008080808080808080C0C0C0C0C0C0C0C17
:103910000C0C0C0C0C0C0C0C0C0C0C0C0C0C0C0CE7
:103920000C0C0C0C0C0C0C0C0C0C0C0C0C0C0C0CD7
:103930000C0C0C0C0C0C0C0C0C0C0C0C0C0C0C0CC7
:1039400008080808080808080C0C0C0C0C0C0C0CD7
:103950000C0C0C0C0C0C0C0C0C0C0C0C0C0C0C0CA7
:103960000C0C0C0C0C0C0C0C0C0C0C0C0C0C0C0C97
:103970000C0C0C0C0C0C0C0C0C0C0C0C0C0C0C0C87
:1039800008080808080808080C0C0C0C0C0C0C0C97
:103990000C0C0C0C0C0C0C0C0C0C0C0C0C0C0C0C67
:1039A0000C0C0C0C0C0C0C0C0C0C0C0C0C0C0C0C57
:1039B0000C0C0C0C0C0C0C0C0C0C0C0C0C0C0C0C47
:1039C00008080808080808080C0C0C0C0C0C0C0C57
:1039D0000C0C0C0C0C0C0C0C0C0C0C0C0C0C0C0C27
:1039E0000C0C0C0C0C0C0C0C0C0C0C0C0C0C0C0C17
:1039F0000C0C0C0C0C0C0C0C0C0C0C0C0C0C0C0C07
:103A000008080808080808080C0C0C0C0C0C0C0C16
:103A10000C0C0C0C0C0C0C0C0C0C0C0C0C0C0C0CE6
:103A20000C0C0C0C0C0C0C0C0C0C0C0C0C0C0C0CD6
:103A30000C0C0C0C0C0C0C0C0C0C0C0C0C0C0C0CC6
:103A400008080808080808080C0C0C0C0C0C0C0CD6
:103A50000C0C0C0C0C0C0C0C0C0C0C0C0C0C0C0CA6
:103A60000C0C0C0C0C0C0C0C0C0C0C0C0C0C0C0C96
:103A70000C0C0C0C0C0C0C0C0C0C0C0C0C0C0C0C86
:103A800008080808080808080C0C0C0C0C0C0C0C96
:103A90000C0C0C0C0C0C0C0C0C0C0C0C0C0C0C0C66
:103AA0000C0C0C0C0C0C0C0C0C0C0C0C0C0C0C0C56
:103AB0000C0C0C0C0C0C0C0C0C0C0C0C0C0C0C0C46
:103AC00008080808080808080C0C0C0C0C0C0C0C56
:103AD0000C0C0C0C0C0C0C0C0C0C0C0C0C0C0C0C26
:103AE0000C0C0C0C0C0C0C0C0C0C0C0C0C0C0C0C16
:103AF0000C0C0C0C0C0C0C0C0C0C0C0C0C0C0C0C06
:103B000008080808080808080C0C0C0C0C0C0C0C15
:103B10000C0C0C0C0C0C0C0C0C0C0C0C0C0C0C0CE5
:103B20000C0C0C0C0C0C0C0C0C0C0C0C0C0C0C0CD5
:103B30000C0C0C0C0C0C0C0C0C0C0C0C0C0C0C0CC5
:103B400008080808080808080C0C0C0C0C0C0C0CD5
:103B50000C0C0C0C0C0C0C0C0C0C0C0C0C0C0C0CA5
:103B60000C0C0C0C0C0C0C0C0C0C0C0C0C0C0C0C95
:103B70000C0C0C0C0C0C0C0C0C0C0C0C0C0C0C0C85
:103B800008080808080808080C0C0C0C0C0C0C0C95
:103B90000C0C0C0C0C0C0C0C0C0C0C0C0C0C0C0C65
:103BA0000C0C0C0C0C0C0C0C0C0C0C0C0C0C0C0C55
:103BB0000C0C0C0C0C0C0C0C0C0C0C0C0C0C0C0C45
:103BC00008080808080808080C0C0C0C0C0C0C0C55
:103BD0000C0C0C0C0C0C0C0C0C0C0C0C0C0C0C0C25
:103BE0000C0C0C0C0C0C0C0C0C0C0C0C0C0C0C0C15
:103BF0000C0C0C0C0C0C0C0C0C0C0C0C0C0C0C0C05
:103C000008080808080808080C0C0C0C0C0C0C0C14
:103C10000C0C0C0C0C0C0C0C0C0C0C0C0C0C0C0CE4
:103C20000C0C0C0C0C0C0C0C0C0C0C0C0C0C0C0CD4
:103C30000C0C0C0C0C0C0C0C0C0C0C0C0C0C0C0CC4
:103C400008080808080808080C0C0C0C0C0C0C0CD4
:103C50000C0C0C0C0C0C0C0C0C0C0C0C0C0C0C0CA4
:103C60000C0C0C0C0C0C0C0C0C0C0C0C0C0C0C0C94
:103C70000C0C0C0C0C0C0C0C0C0C0C0C0C0C0C0C84
:103C800008080808080808080C0C0C0C0C0C0C0C94
:103C90000C0C0C0C0C0C0C0C0C0C0C0C0C0C0C0C64
:103CA0000C0C0C0C0C0C0C0C0C0C0C0C0C0C0C0C54
:103CB0000C0C0C0C0C0C0C0C0C0C0C0C0C0C0C0C44
:103CC00008080808080808080C0C0C0C0C0C0C0C54
:103CD0000C0C0C0C0C0C0C0C0C0C0C0C0C0C0C0C24
:103CE0000C0C0C0C0C0C0C0C0C0C0C0C0C0C0C0C14
:103CF0000C0C0C0C0C0C0C0C0C0C0C0C0C0C0C0C04
:103D000008080808080808080C0C0C0C0C0C0C0C13
:103D10000C0C0C0C0C0C0C0C0C0C0C0C0C0C0C0CE3
:103D20000C0C0C0C0C0C0C0C0C0C0C0C0C0C0C0CD3
:103D30000C0C0C0C0C0C0C0C0C0C0C0C0C0C0C0CC3
:103D400008080808080808080C0C0C0C0C0C0C0CD3
:103D50000C0C0C0C0C0C0C0C0C0C0C0C0C0C0C0CA3
:103D60000C0C0C0C0C0C0C0C0C0C0C0C0C0C0C0C93
:103D70000C0C0C0C0C0C0C0C0C0C0C0C0C0C0C0C83
:103D800008080808080808080C0C0C0C0C0C0C0C93
:103D90000C0C0C0C0C0C0C0C0C0C0C0C0C0C0C0C63
:103DA0000C0C0C0C0C0C0C0C0C0C0C0C0C0C0C0C53
:103DB0000C0C0C0C0C0C0C0C0C0C0C0C0C0C0C0C43
:103DC00008080808080808080C0C0C0C0C0C0C0C53
:103DD0000C0C0C0C0C0C0C0C0C0C0C0C0C0C0C0C23
:103DE0000C0C0C0C0C0C0C0C0C0C0C0C0C0C0C0C13
:103DF0000C0C0C0C0C0C0C0C0C0C0C0C0C0C0C0C03
:103E000008080808080808080C0C0C0C0C0C0C0C12
:103E10000C0C0C0C0C0C0C0C0C0C0C0C0C0C0C0CE2
:103E20000C0C0C0C0C0C0C0C0C0C0C0C0C0C0C0CD2
:103E30000C0C0C0C0C0C0C0C0C0C0C0C0C0C0C0CC2
:103E400008080808080808080C0C0C0C0C0C0C0CD2
:103E50000C0C0C0C0C0C0C0C0C0C0C0C0C0C0C0CA2
:103E60000C0C0C0C0C0C0C0C0C0C0C0C0C0C0C0C92
:103E70000C0C0C0C0C0C0C0C0C0C0C0C0C0C0C0C82
:103E800008080808080808080C0C0C0C0C0C0C0C92
:103E90000C0C0C0C0C0C0C0C0C0C0C0C0C0C0C0C62
:103EA0000C0C0C0C0C0C0C0C0C0C0C0C0C0C0C0C52
:103EB0000C0C0C0C0C0C0C0C0C0C0C0C0C0C0C0C42
:103EC00008080808080808080C0C0C0C0C0C0C0C52
:103ED0000C0C0C0C0C0C0C0C0C0C0C0C0C0C0C0C22
:103EE0000C0C0C0C0C0C0C0C0C0C0C0C0C0C0C0C12
:103EF0000C0C0C0C0C0C0C0C0C0C0C0C0C0C0C0C02
:103F000008080808080808080C0C0C0C0C0C0C0C11
:103F10000C0C0C0C0C0C0C0C0C0C0C0C0C0C0C0CE1
:103F20000C0C0C0C0C0C0C0C0C0C0C0C0C0C0C0CD1
:103F30000C0C0C0C0C0C0C0C0C0C0C0C0C0C0C0CC1
:103F400008080808080808080C0C0C0C0C0C0C0CD1
:103F50000C0C0C0C0C0C0C0C0C0C0C0C0C0C0C0CA1
:103F60000C0C0C0C0C0C0C0C0C0C0C0C0C0C0C0C91
:103F70000C0C0C0C0C0C0C0C0C0C0C0C0C0C0C0C81
:103F800008080808080808080C0C0C0C0C0C0C0C91
:103F90000C0C0C0C0C0C0C0C0C0C0C0C0C0C0C0C61
:103FA0000C0C0C0C0C0C0C0C0C0C0C0C0C0C0C0C51
:103FB0000C0C0C0C0C0C0C0C0C0C0C0C0C0C0C0C41
:103FC00008080808080808080C0C0C0C0C0C0C0C51
:103FD0000C0C0C0C0C0C0C0C0C0C0C0C0C0C0C0C21
:103FE0000C0C0C0C0C0C0C0C0C0C0C0C0C0C0C0C11
:103FF0000C0C0C0C0C0C0C0C0C0C0C0C0C0C0C0C01
:1040000008080808080808080C0C0C0C0C0C0C0C10
:104010000C0C0C0C0C0C0C0C0C0C0C0C0C0C0C0CE0
:104020000C0C0C0C0C0C0C0C0C0C0C0C0C0C0C0CD0
:104030000C0C0C0C0C0C0C0C0C0C0C0C0C0C0C0CC0
:1040400008080808080808080C0C0C0C0C0C0C0CD0
:104050000C0C0C0C0C0C0C0C0C0C0C0C0C0C0C0CA0
:104060000C0C0C0C0C0C0C0C0C0C0C0C0C0C0C0C90
:104070000C0C0C0C0C0C0C0C0C0C0C0C0C0C0C0C80
:1040800008080808080808080C0C0C0C0C0C0C0C90
:104090000C0C0C0C0C0C0C0C0C0C0C0C0C0C0C0C60
:1040A0000C0C0C0C0C0C0C0C0C0C0C0C0C0C0C0C50
:1040B0000C0C0C0C0C0C0C0C0C0C0C0C0C0C0C0C40
:1040C00008080808080808080C0C0C0C0C0C0C0C50
:1040D0000C0C0C0C0C0C0C0C0C0C0C0C0C0C0C0C20
:1040E0000C0C0C0C0C0C0C0C0C0C0C0C0C0C0C0C10
:1040F0000C0C0C0C0C0C0C0C0C0C0C0C0C0C0C0C00
:1041000008080808080808080C0C0C0C0C0C0C0C0F
:104110000C0C0C0C0C0C0C0C0C0C0C0C0C0C0C0CDF
:104120000C0C0C0C0C0C0C0C0C0C0C0C0C0C0C0CCF
:104130000C0C0C0C0C0C0C0C0C0C0C0C0C0C0C0CBF
:1041400008080808080808080C0C0C0C0C0C0C0CCF
:104150000C0C0C0C0C0C0C0C0C0C0C0C0C0C0C0C9F
:104160000C0C0C0C0C0C0C0C0C0C0C0C0C0C0C0C8F
:104170000C0C0C0C0C0C0C0C0C0C0C0C0C0C0C0C7F
:1041800008080808080808080C0C0C0C0C0C0C0C8F
:104190000C0C0C0C0C0C0C0C0C0C0C0C0C0C0C0C5F
:1041A0000C0C0C0C0C0C0C0C0C0C0C0C0C0C0C0C4F
:1041B0000C0C0C0C0C0C0C0C0C0C0C0C0C0C0C0C3F
:1041C00008080808080808080C0C0C0C0C0C0C0C4F
:1041D0000C0C0C0C0C0C0C0C0C0C0C0C0C0C0C0C1F
:1041E0000C0C0C0C0C0C0C0C0C0C0C0C0C0C0C0C0F
:1041F0000C0C0C0C0C0C0C0C0C0C0C0C0C0C0C0CFF
:1042000008080808080808080C0C0C0C0C0C0C0C0E
:104210000C0C0C0C0C0C0C0C0C0C0C0C0C0C0C0CDE
:104220000C0C0C0C0C0C0C0C0C0C0C0C0C0C0C0CCE
:104230000C0C0C0C0C0C0C0C0C0C0C0C0C0C0C0CBE
:1042400008080808080808080C0C0C0C0C0C0C0CCE
:104250000C0C0C0C0C0C0C0C0C0C0C0C0C0C0C0C9E
:104260000C0C0C0C0C0C0C0C0C0C0C0C0C0C0C0C8E
:104270000C0C0C0C0C0C0C0C0C0C0C0C0C0C0C0C7E
:1042800008080808080808080C0C0C0C0C0C0C0C8E
:104290000C0C0C0C0C0C0C0C0C0C0C0C0C0C0C0C5E
:1042A0000C0C0C0C0C0C0C0C0C0C0C0C0C0C0C0C4E
:1042B0000C0C0C0C0C0C0C0C0C0C0C0C0C0C0C0C3E
:1042C00008080808080808080C0C0C0C0C0C0C0C4E
:1042D0000C0C0C0C0C0C0C0C0C0C0C0C0C0C0C0C1E
:1042E0000C0C0C0C0C0C0C0C0C0C0C0C0C0C0C0C0E
:1042F0000C0C0C0C0C0C0C0C0C0C0C0C0C0C0C0CFE
:1043000008080808080808080C0C0C0C0C0C0C0C0D
:104310000C0C0C0C0C0C0C0C0C0C0C0C0C0C0C0CDD
:104320000C0C0C0C0C0C0C0C0C0C0C0C0C0C0C0CCD
:104330000C0C0C0C0C0C0C0C0C0C0C0C0C0C0C0CBD
:1043400008080808080808080C0C0C0C0C0C0C0CCD
:104350000C0C0C0C0C0C0C0C0C0C0C0C0C0C0C0C9D
:104360000C0C0C0C0C0C0C0C0C0C0C0C0C0C0C0C8D
:104370000C0C0C0C0C0C0C0C0C0C0C0C0C0C0C0C7D
:1043800008080808080808080C0C0C0C0C0C0C0C8D
:104390000C0C0C0C0C0C0C0C0C0C0C0C0C0C0C0C5D
:1043A0000C0C0C0C0C0C0C0C0C0C0C0C0C0C0C0C4D
:1043B0000C0C0C0C0C0C0C0C0C0C0C0C0C0C0C0C3D
:1043C00008080808080808080C0C0C0C0C0C0C0C4D
:1043D0000C0C0C0C0C0C0C0C0C0C0C0C0C0C0C0C1D
:1043E0000C0C0C0C0C0C0C0C0C0C0C0C0C0C0C0C0D
:1043F0000C0C0C0C0C0C0C0C0C0C0C0C0C0C0C0CFD
:1044000008080808080808080C0C0C0C0C0C0C0C0C
:104410000C0C0C0C0C0C0C0C0C0C0C0C0C0C0C0CDC
:104420000C0C0C0C0C0C0C0C0C0C0C0C0C0C0C0CCC
:104430000C0C0C0C0C0C0C0C0C0C0C0C0C0C0C0CBC
:1044400008080808080808080C0C0C0C0C0C0C0CCC
:104450000C0C0C0C0C0C0C0C0C0C0C0C0C0C0C0C9C
:104460000C0C0C0C0C0C0C0C0C0C0C0C0C0C0C0C8C
:104470000C0C0C0C0C0C0C0C0C0C0C0C0C0C0C0C7C
:1044800008080808080808080C0C0C0C0C0C0C0C8C
:104490000C0C0C0C0C0C0C0C0C0C0C0C0C0C0C0C5C
:1044A0000C0C0C0C0C0C0C0C0C0C0C0C0C0C0C0C4C
:1044B0000C0C0C0C0C0C0C0C0C0C0C0C0C0C0C0C3C
:1044C00008080808080808080C0C0C0C0C0C0C0C4C
:1044D0000C0C0C0C0C0C0C0C0C0C0C0C0C0C0C0C1C
:1044E0000C0C0C0C0C0C0C0C0C0C0C0C0C0C0C0C0C
:1044F0000C0C0C0C0C0C0C0C0C0C0C0C0C0C0C0CFC
:1045000008080808080808080C0C0C0C0C0C0C0C0B
:104510000C0C0C0C0C0C0C0C0C0C0C0C0C0C0C0CDB
:104520000C0C0C0C0C0C0C0C0C0C0C0C0C0C0C0CCB
:104530000C0C0C0C0C0C0C0C0C0C0C0C0C0C0C0CBB
:1045400008080808080808080C0C0C0C0C0C0C0CCB
:104550000C0C0C0C0C0C0C0C0C0C0C0C0C0C0C0C9B
:104560000C0C0C0C0C0C0C0C0C0C0C0C0C0C0C0C8B
:104570000C0C0C0C0C0C0C0C0C0C0C0C0C0C0C0C7B
:1045800008080808080808080C0C0C0C0C0C0C0C8B
:104590000C0C0C0C0C0C0C0C0C0C0C0C0C0C0C0C5B
:1045A0000C0C0C0C0C0C0C0C0C0C0C0C0C0C0C0C4B
:1045B0000C0C0C0C0C0C0C0C0C0C0C0C0C0C0C0C3B
:1045C00008080808080808080C0C0C0C0C0C0C0C4B
:1045D0000C0C0C0C0C0C0C0C0C0C0C0C0C0C0C0C1B
:1045E0000C0C0C0C0C0C0C0C0C0C0C0C0C0C0C0C0B
:1045F0000C0C0C0C0C0C0C0C0C0C0C0C0C0C0C0CFB
:1046000008080808080808080C0C0C0C0C0C0C0C0A
:104610000C0C0C0C0C0C0C0C0C0C0C0C0C0C0C0CDA
:104620000C0C0C0C0C0C0C0C0C0C0C0C0C0C0C0CCA
:104630000C0C0C0C0C0C0C0C0C0C0C0C0C0C0C0CBA
:1046400008080808080808080C0C0C0C0C0C0C0CCA
:104650000C0C0C0C0C0C0C0C0C0C0C0C0C0C0C0C9A
:104660000C0C0C0C0C0C0C0C0C0C0C0C0C0C0C0C8A
:104670000C0C0C0C0C0C0C0C0C0C0C0C0C0C0C0C7A
:1046800008080808080808080C0C0C0C0C0C0C0C8A
:104690000C0C0C0C0C0C0C0C0C0C0C0C0C0C0C0C5A
:1046A0000C0C0C0C0C0C0C0C0C0C0C0C0C0C0C0C4A
:1046B0000C0C0C0C0C0C0C0C0C0C0C0C0C0C0C0C3A
:1046C00008080808080808080C0C0C0C0C0C0C0C4A
:1046D0000C0C0C0C0C0C0C0C0C0C0C0C0C0C0C0C1A
:1046E0000C0C0C0C0C0C0C0C0C0C0C0C0C0C0C0C0A
:1046F0000C0C0C0C0C0C0C0C0C0C0C0C0C0C0C0CFA
:1047000008080808080808080C0C0C0C0C0C0C0C09
:104710000C0C0C0C0C0C0C0C0C0C0C0C0C0C0C0CD9
:104720000C0C0C0C0C0C0C0C0C0C0C0C0C0C0C0CC9
:104730000C0C0C0C0C0C0C0C0C0C0C0C0C0C0C0CB9
:1047400008080808080808080C0C0C0C0C0C0C0CC9
:104750000C0C0C0C0C0C0C0C0C0C0C0C0C0C0C0C99
:104760000C0C0C0C0C0C0C0C0C0C0C0C0C0C0C0C89
:104770000C0C0C0C0C0C0C0C0C0C0C0C0C0C0C0C79
:1047800008080808080808080C0C0C0C0C0C0C0C89
:104790000C0C0C0C0C0C0C0C0C0C0C0C0C0C0C0C59
:1047A0000C0C0C0C0C0C0C0C0C0C0C0C0C0C0C0C49
:1047B0000C0C0C0C0C0C0C0C0C0C0C0C0C0C0C0C39
:1047C00008080808080808080C0C0C0C0C0C0C0C49
:1047D0000C0C0C0C0C0C0C0C0C0C0C0C0C0C0C0C19
:1047E0000C0C0C0C0C0C0C0C0C0C0C0C0C0C0C0C09
:1047F0000C0C0C0C0C0C0C0C0C0C0C0C0C0C0C0CF9
:1048000008080808080808080C0C0C0C0C0C0C0C08
:104810000C0C0C0C0C0C0C0C0C0C0C0C0C0C0C0CD8
:104820000C0C0C0C0C0C0C0C0C0C0C0C0C0C0C0CC8
:104830000C0C0C0C0C0C0C0C0C0C0C0C0C0C0C0CB8
:1048400008080808080808080C0C0C0C0C0C0C0CC8
:104850000C0C0C0C0C0C0C0C0C0C0C0C0C0C0C0C98
:104860000C0C0C0C0C0C0C0C0C0C0C0C0C0C0C0C88
:104870000C0C0C0C0C0C0C0C0C0C0C0C0C0C0C0C78
:1048800008080808080808080C0C0C0C0C0C0C0C88
:104890000C0C0C0C0C0C0C0C0C0C0C0C0C0C0C0C58
:1048A0000C0C0C0C0C0C0C0C0C0C0C0C0C0C0C0C48
:1048B0000C0C0C0C0C0C0C0C0C0C0C0C0C0C0C0C38
:1048C00008080808080808080C0C0C0C0C0C0C0C48
:1048D0000C0C0C0C0C0C0C0C0C0C0C0C0C0C0C0C18
:1048E0000C0C0C0C0C0C0C0C0C0C0C0C0C0C0C0C08
:1048F0000C0C0C0C0C0C0C0C0C0C0C0C0C0C0C0CF8
:1049000008080808080808080C0C0C0C0C0C0C0C07
:104910000C0C0C0C0C0C0C0C0C0C0C0C0C0C0C0CD7
:104920000C0C0C0C0C0C0C0C0C0C0C0C0C0C0C0CC7
:104930000C0C0C0C0C0C0C0C0C0C0C0C0C0C0C0CB7
:1049400008080808080808080C0C0C0C0C0C0C0CC7
:104950000C0C0C0C0C0C0C0C0C0C0C0C0C0C0C0C97
:104960000C0C0C0C0C0C0C0C0C0C0C0C0C0C0C0C87
:104970000C0C0C0C0C0C0C0C0C0C0C0C0C0C0C0C77
:1049800008080808080808080C0C0C0C0C0C0C0C87
:104990000C0C0C0C0C0C0C0C0C0C0C0C0C0C0C0C57
:1049A0000C0C0C0C0C0C0C0C0C0C0C0C0C0C0C0C47
:1049B0000C0C0C0C0C0C0C0C0C0C0C0C0C0C0C0C37
:1049C00008080808080808080C0C0C0C0C0C0C0C47
:1049D0000C0C0C0C0C0C0C0C0C0C0C0C0C0C0C0C17
:1049E0000C0C0C0C0C0C0C0C0C0C0C0C0C0C0C0C07
:1049F0000C0C0C0C0C0C0C0C0C0C0C0C0C0C0C0CF7
:104A000008080808080808080C0C0C0C0C0C0C0C06
:104A10000C0C0C0C0C0C0C0C0C0C0C0C0C0C0C0CD6
:104A20000C0C0C0C0C0C0C0C0C0C0C0C0C0C0C0CC6
:104A30000C0C0C0C0C0C0C0C0C0C0C0C0C0C0C0CB6
:104A400008080808080808080C0C0C0C0C0C0C0CC6
:104A50000C0C0C0C0C0C0C0C0C0C0C0C0C0C0C0C96
:104A60000C0C0C0C0C0C0C0C0C0C0C0C0C0C0C0C86
:104A70000C0C0C0C0C0C0C0C0C0C0C0C0C0C0C0C76
:104A800008080808080808080C0C0C0C0C0C0C0C86
:104A90000C0C0C0C0C0C0C0C0C0C0C0C0C0C0C0C56
:104AA0000C0C0C0C0C0C0C0C0C0C0C0C0C0C0C0C46
:104AB0000C0C0C0C0C0C0C0C0C0C0C0C0C0C0C0C36
:104AC00008080808080808080C0C0C0C0C0C0C0C46
:104AD0000C0C0C0C0C0C0C0C0C0C0C0C0C0C0C0C16
:104AE0000C0C0C0C0C0C0C0C0C0C0C0C0C0C0C0C06
:104AF0000C0C0C0C0C0C0C0C0C0C0C0C0C0C0C0CF6
:104B000008080808080808080C0C0C0C0C0C0C0C05
:104B10000C0C0C0C0C0C0C0C0C0C0C0C0C0C0C0CD5
:104B20000C0C0C0C0C0C0C0C0C0C0C0C0C0C0C0CC5
:104B30000C0C0C0C0C0C0C0C0C0C0C0C0C0C0C0CB5
:104B400008080808080808080C0C0C0C0C0C0C0CC5
:104B50000C0C0C0C0C0C0C0C0C0C0C0C0C0C0C0C95
:104B60000C0C0C0C0C0C0C0C0C0C0C0C0C0C0C0C85
:104B70000C0C0C0C0C0C0C0C0C0C0C0C0C0C0C0C75
:104B800008080808080808080C0C0C0C0C0C0C0C85
:104B90000C0C0C0C0C0C0C0C0C0C0C0C0C0C0C0C55
:104BA0000C0C0C0C0C0C0C0C0C0C0C0C0C0C0C0C45
:104BB0000C0C0C0C0C0C0C0C0C0C0C0C0C0C0C0C35
:104BC00008080808080808080C0C0C0C0C0C0C0C45
:104BD0000C0C0C0C0C0C0C0C0C0C0C0C0C0C0C0C15
:104BE0000C0C0C0C0C0C0C0C0C0C0C0C0C0C0C0C05
:104BF0000C0C0C0C0C0C0C0C0C0C0C0C0C0C0C0CF5
:104C000008080808080808080C0C0C0C0C0C0C0C04
:104C10000C0C0C0C0C0C0C0C0C0C0C0C0C0C0C0CD4
:104C20000C0C0C0C0C0C0C0C0C0C0C0C0C0C0C0CC4
:104C30000C0C0C0C0C0C0C0C0C0C0C0C0C0C0C0CB4
:104C400008080808080808080C0C0C0C0C0C0C0CC4
:104C50000C0C0C0C0C0C0C0C0C0C0C0C0C0C0C0C94
:104C60000C0C0C0C0C0C0C0C0C0C0C0C0C0C0C0C84
:104C70000C0C0C0C0C0C0C0C0C0C0C0C0C0C0C0C74
:104C800008080808080808080C0C0C0C0C0C0C0C84
:104C90000C0C0C0C0C0C0C0C0C0C0C0C0C0C0C0C54
:104CA0000C0C0C0C0C0C0C0C0C0C0C0C0C0C0C0C44
:104CB0000C0C0C0C0C0C0C0C0C0C0C0C0C0C0C0C34
:104CC00008080808080808080C0C0C0C0C0C0C0C44
:104CD0000C0C0C0C0C0C0C0C0C0C0C0C0C0C0C0C14
:104CE0000C0C0C0C0C0C0C0C0C0C0C0C0C0C0C0C04
:104CF0000C0C0C0C0C0C0C0C0C0C0C0C0C0C0C0CF4
:104D000008080808080808080C0C0C0C0C0C0C0C03
:104D10000C0C0C0C0C0C0C0C0C0C0C0C0C0C0C0CD3
:104D20000C0C0C0C0C0C0C0C0C0C0C0C0C0C0C0CC3
:104D30000C0C0C0C0C0C0C0C0C0C0C0C0C0C0C0CB3
:104D400008080808080808080C0C0C0C0C0C0C0CC3
:104D50000C0C0C0C0C0C0C0C0C0C0C0C0C0C0C0C93
:104D60000C0C0C0C0C0C0C0C0C0C0C0C0C0C0C0C83
:104D70000C0C0C0C0C0C0C0C0C0C0C0C0C0C0C0C73
:104D800008080808080808080C0C0C0C0C0C0C0C83
:104D90000C0C0C0C0C0C0C0C0C0C0C0C0C0C0C0C53
:104DA0000C0C0C0C0C0C0C0C0C0C0C0C0C0C0C0C43
:104DB0000C0C0C0C0C0C0C0C0C0C0C0C0C0C0C0C33
:104DC00008080808080808080C0C0C0C0C0C0C0C43
:104DD0000C0C0C0C0C0C0C0C0C0C0C0C0C0C0C0C13
:104DE0000C0C0C0C0C0C0C0C0C0C0C0C0C0C0C0C03
:104DF0000C0C0C0C0C0C0C0C0C0C0C0C0C0C0C0CF3
:104E000008080808080808080C0C0C0C0C0C0C0C02
:104E10000C0C0C0C0C0C0C0C0C0C0C0C0C0C0C0CD2
:104E20000C0C0C0C0C0C0C0C0C0C0C0C0C0C0C0CC2
:104E30000C0C0C0C0C0C0C0C0C0C0C0C0C0C0C0CB2
:104E400008080808080808080C0C0C0C0C0C0C0CC2
:104E50000C0C0C0C0C0C0C0C0C0C0C0C0C0C0C0C92
:104E60000C0C0C0C0C0C0C0C0C0C0C0C0C0C0C0C82
:104E70000C0C0C0C0C0C0C0C0C0C0C0C0C0C0C0C72
:104E800008080808080808080C0C0C0C0C0C0C0C82
:104E90000C0C0C0C0C0C0C0C0C0C0C0C0C0C0C0C52
:104EA0000C0C0C0C0C0C0C0C0C0C0C0C0C0C0C0C42
:104EB0000C0C0C0C0C0C0C0C0C0C0C0C0C0C0C0C32
:104EC00008080808080808080C0C0C0C0C0C0C0C42
:104ED0000C0C0C0C0C0C0C0C0C0C0C0C0C0C0C0C12
:104EE0000C0C0C0C0C0C0C0C0C0C0C0C0C0C0C0C02
:104EF0000C0C0C0C0C0C0C0C0C0C0C0C0C0C0C0CF2
:104F000008080808080808080C0C0C0C0C0C0C0C01
:104F10000C0C0C0C0C0C0C0C0C0C0C0C0C0C0C0CD1
:104F20000C0C0C0C0C0C0C0C0C0C0C0C0C0C0C0CC1
:104F30000C0C0C0C0C0C0C0C0C0C0C0C0C0C0C0CB1
:104F400008080808080808080C0C0C0C0C0C0C0CC1
:104F50000C0C0C0C0C0C0C0C0C0C0C0C0C0C0C0C91
:104F60000C0C0C0C0C0C0C0C0C0C0C0C0C0C0C0C81
:104F70000C0C0C0C0C0C0C0C0C0C0C0C0C0C0C0C71
:104F800008080808080808080C0C0C0C0C0C0C0C81
:104F90000C0C0C0C0C0C0C0C0C0C0C0C0C0C0C0C51
:104FA0000C0C0C0C0C0C0C0C0C0C0C0C0C0C0C0C41
:104FB0000C0C0C0C0C0C0C0C0C0C0C0C0C0C0C0C31
:104FC00008080808080808080C0C0C0C0C0C0C0C41
:104FD0000C0C0C0C0C0C0C0C0C0C0C0C0C0C0C0C11
:104FE0000C0C0C0C0C0C0C0C0C0C0C0C0C0C0C0C01
:104FF0000C0C0C0C0C0C0C0C0C0C0C0C0C0C0C0CF1
:1050000008080808080808080C0C0C0C0C0C0C0C00
:105010000C0C0C0C0C0C0C0C0C0C0C0C0C0C0C0CD0
:105020000C0C0C0C0C0C0C0C0C0C0C0C0C0C0C0CC0
:105030000C0C0C0C0C0C0C0C0C0C0C0C0C0C0C0CB0
:1050400008080808080808080C0C0C0C0C0C0C0CC0
:105050000C0C0C0C0C0C0C0C0C0C0C0C0C0C0C0C90
:105060000C0C0C0C0C0C0C0C0C0C0C0C0C0C0C0C80
:105070000C0C0C0C0C0C0C0C0C0C0C0C0C0C0C0C70
:1050800008080808080808080C0C0C0C0C0C0C0C80
:105090000C0C0C0C0C0C0C0C0C0C0C0C0C0C0C0C50
:1050A0000C0C0C0C0C0C0C0C0C0C0C0C0C0C0C0C40
:1050B0000C0C0C0C0C0C0C0C0C0C0C0C0C0C0C0C30
:1050C00008080808080808080C0C0C0C0C0C0C0C40
:1050D0000C0C0C0C0C0C0C0C0C0C0C0C0C0C0C0C10
:1050E0000C0C0C0C0C0C0C0C0C0C0C0C0C0C0C0C00
:1050F0000C0C0C0C0C0C0C0C0C0C0C0C0C0C0C0CF0
:1051000008080808080808080C0C0C0C0C0C0C0CFF
:105110000C0C0C0C0C0C0C0C0C0C0C0C0C0C0C0CCF
:105120000C0C0C0C0C0C0C0C0C0C0C0C0C0C0C0CBF
:105130000C0C0C0C0C0C0C0C0C0C0C0C0C0C0C0CAF
:1051400008080808080808080C0C0C0C0C0C0C0CBF
:105150000C0C0C0C0C0C0C0C0C0C0C0C0C0C0C0C8F
:105160000C0C0C0C0C0C0C0C0C0C0C0C0C0C0C0C7F
:105170000C0C0C0C0C0C0C0C0C0C0C0C0C0C0C0C6F
:1051800008080808080808080C0C0C0C0C0C0C0C7F
:105190000C0C0C0C0C0C0C0C0C0C0C0C0C0C0C0C4F
:1051A0000C0C0C0C0C0C0C0C0C0C0C0C0C0C0C0C3F
:1051B0000C0C0C0C0C0C0C0C0C0C0C0C0C0C0C0C2F
:1051C00008080808080808080C0C0C0C0C0C0C0C3F
:1051D0000C0C0C0C0C0C0C0C0C0C0C0C0C0C0C0C0F
:1051E0000C0C0C0C0C0C0C0C0C0C0C0C0C0C0C0CFF
:1051F0000C0C0C0C0C0C0C0C0C0C0C0C0C0C0C0CEF
:1052000008080808080808080C0C0C0C0C0C0C0CFE
:105210000C0C0C0C0C0C0C0C0C0C0C0C0C0C0C0CCE
:105220000C0C0C0C0C0C0C0C0C0C0C0C0C0C0C0CBE
:105230000C0C0C0C0C0C0C0C0C0C0C0C0C0C0C0CAE
:1052400008080808080808080C0C0C0C0C0C0C0CBE
:105250000C0C0C0C0C0C0C0C0C0C0C0C0C0C0C0C8E
:105260000C0C0C0C0C0C0C0C0C0C0C0C0C0C0C0C7E
:105270000C0C0C0C0C0C0C0C0C0C0C0C0C0C0C0C6E
:1052800008080808080808080C0C0C0C0C0C0C0C7E
:105290000C0C0C0C0C0C0C0C0C0C0C0C0C0C0C0C4E
:1052A0000C0C0C0C0C0C0C0C0C0C0C0C0C0C0C0C3E
:1052B0000C0C0C0C0C0C0C0C0C0C0C0C0C0C0C0C2E
:1052C00008080808080808080C0C0C0C0C0C0C0C3E
:1052D0000C0C0C0C0C0C0C0C0C0C0C0C0C0C0C0C0E
:1052E0000C0C0C0C0C0C0C0C0C0C0C0C0C0C0C0CFE
:1052F0000C0C0C0C0C0C0C0C0C0C0C0C0C0C0C0CEE
:1053000008080808080808080C0C0C0C0C0C0C0CFD
:105310000C0C0C0C0C0C0C0C0C0C0C0C0C0C0C0CCD
:105320000C0C0C0C0C0C0C0C0C0C0C0C0C0C0C0CBD
:105330000C0C0C0C0C0C0C0C0C0C0C0C0C0C0C0CAD
:1053400008080808080808080C0C0C0C0C0C0C0CBD
:105350000C0C0C0C0C0C0C0C0C0C0C0C0C0C0C0C8D
:105360000C0C0C0C0C0C0C0C0C0C0C0C0C0C0C0C7D
:105370000C0C0C0C0C0C0C0C0C0C0C0C0C0C0C0C6D
:1053800008080808080808080C0C0C0C0C0C0C0C7D
:105390000C0C0C0C0C0C0C0C0C0C0C0C0C0C0C0C4D
:1053A0000C0C0C0C0C0C0C0C0C0C0C0C0C0C0C0C3D
:1053B0000C0C0C0C0C0C0C0C0C0C0C0C0C0C0C0C2D
:1053C00008080808080808080C0C0C0C0C0C0C0C3D
:1053D0000C0C0C0C0C0C0C0C0C0C0C0C0C0C0C0C0D
:1053E0000C0C0C0C0C0C0C0C0C0C0C0C0C0C0C0CFD
:1053F0000C0C0C0C0C0C0C0C0C0C0C0C0C0C0C0CED
:1054000008080808080808080C0C0C0C0C0C0C0CFC
:105410000C0C0C0C0C0C0C0C0C0C0C0C0C0C0C0CCC
:105420000C0C0C0C0C0C0C0C0C0C0C0C0C0C0C0CBC
:105430000C0C0C0C0C0C0C0C0C0C0C0C0C0C0C0CAC
:1054400008080808080808080C0C0C0C0C0C0C0CBC
:105450000C0C0C0C0C0C0C0C0C0C0C0C0C0C0C0C8C
:105460000C0C0C0C0C0C0C0C0C0C0C0C0C0C0C0C7C
:105470000C0C0C0C0C0C0C0C0C0C0C0C0C0C0C0C6C
:1054800008080808080808080C0C0C0C0C0C0C0C7C
:105490000C0C0C0C0C0C0C0C0C0C0C0C0C0C0C0C4C
:1054A0000C0C0C0C0C0C0C0C0C0C0C0C0C0C0C0C3C
:1054B0000C0C0C0C0C0C0C0C0C0C0C0C0C0C0C0C2C
:1054C00008080808080808080C0C0C0C0C0C0C0C3C
:1054D0000C0C0C0C0C0C0C0C0C0C0C0C0C0C0C0C0C
:1054E0000C0C0C0C0C0C0C0C0C0C0C0C0C0C0C0CFC
:1054F0000C0C0C0C0C0C0C0C0C0C0C0C0C0C0C0CEC
:1055000008080808080808080C0C0C0C0C0C0C0CFB
:105510000C0C0C0C0C0C0C0C0C0C0C0C0C0C0C0CCB
:105520000C0C0C0C0C0C0C0C0C0C0C0C0C0C0C0CBB
:105530000C0C0C0C0C0C0C0C0C0C0C0C0C0C0C0CAB
:1055400008080808080808080C0C0C0C0C0C0C0CBB
:105550000C0C0C0C0C0C0C0C0C0C0C0C0C0C0C0C8B
:105560000C0C0C0C0C0C0C0C0C0C0C0C0C0C0C0C7B
:105570000C0C0C0C0C0C0C0C0C0C0C0C0C0C0C0C6B
:1055800008080808080808080C0C0C0C0C0C0C0C7B
:105590000C0C0C0C0C0C0C0C0C0C0C0C0C0C0C0C4B
:1055A0000C0C0C0C0C0C0C0C0C0C0C0C0C0C0C0C3B
:1055B0000C0C0C0C0C0C0C0C0C0C0C0C0C0C0C0C2B
:1055C00008080808080808080C0C0C0C0C0C0C0C3B
:1055D0000C0C0C0C0C0C0C0C0C0C0C0C0C0C0C0C0B
:1055E0000C0C0C0C0C0C0C0C0C0C0C0C0C0C0C0CFB
:1055F0000C0C0C0C0C0C0C0C0C0C0C0C0C0C0C0CEB
:1056000008080808080808080C0C0C0C0C0C0C0CFA
:105610000C0C0C0C0C0C0C0C0C0C0C0C0C0C0C0CCA
:105620000C0C0C0C0C0C0C0C0C0C0C0C0C0C0C0CBA
:105630000C0C0C0C0C0C0C0C0C0C0C0C0C0C0C0CAA
:1056400008080808080808080C0C0C0C0C0C0C0CBA
:105650000C0C0C0C0C0C0C0C0C0C0C0C0C0C0C0C8A
:105660000C0C0C0C0C0C0C0C0C0C0C0C0C0C0C0C7A
:105670000C0C0C0C0C0C0C0C0C0C0C0C0C0C0C0C6A
:1056800008080808080808080C0C0C0C0C0C0C0C7A
:105690000C0C0C0C0C0C0C0C0C0C0C0C0C0C0C0C4A
:1056A0000C0C0C0C0C0C0C0C0C0C0C0C0C0C0C0C3A
:1056B0000C0C0C0C0C0C0C0C0C0C0C0C0C0C0C0C2A
:1056C00008080808080808080C0C0C0C0C0C0C0C3A
:1056D0000C0C0C0C0C0C0C0C0C0C0C0C0C0C0C0C0A
:1056E0000C0C0C0C0C0C0C0C0C0C0C0C0C0C0C0CFA
:1056F0000C0C0C0C0C0C0C0C0C0C0C0C0C0C0C0CEA
:1057000008080808080808080C0C0C0C0C0C0C0CF9
:105710000C0C0C0C0C0C0C0C0C0C0C0C0C0C0C0CC9
:105720000C0C0C0C0C0C0C0C0C0C0C0C0C0C0C0CB9
:105730000C0C0C0C0C0C0C0C0C0C0C0C0C0C0C0CA9
:1057400008080808080808080C0C0C0C0C0C0C0CB9
:105750000C0C0C0C0C0C0C0C0C0C0C0C0C0C0C0C89
:105760000C0C0C0C0C0C0C0C0C0C0C0C0C0C0C0C79
:105770000C0C0C0C0C0C0C0C0C0C0C0C0C0C0C0C69
:1057800008080808080808080C0C0C0C0C0C0C0C79
:105790000C0C0C0C0C0C0C0C0C0C0C0C0C0C0C0C49
:1057A0000C0C0C0C0C0C0C0C0C0C0C0C0C0C0C0C39
:1057B0000C0C0C0C0C0C0C0C0C0C0C0C0C0C0C0C29
:1057C00008080808080808080C0C0C0C0C0C0C0C39
:1057D0000C0C0C0C0C0C0C0C0C0C0C0C0C0C0C0C09
:1057E0000C0C0C0C0C0C0C0C0C0C0C0C0C0C0C0CF9
:1057F0000C0C0C0C0C0C0C0C0C0C0C0C0C0C0C0CE9
:1058000008080808080808080C0C0C0C0C0C0C0CF8
:105810000C0C0C0C0C0C0C0C0C0C0C0C0C0C0C0CC8
:105820000C0C0C0C0C0C0C0C0C0C0C0C0C0C0C0CB8
:105830000C0C0C0C0C0C0C0C0C0C0C0C0C0C0C0CA8
:1058400008080808080808080C0C0C0C0C0C0C0CB8
:105850000C0C0C0C0C0C0C0C0C0C0C0C0C0C0C0C88
:105860000C0C0C0C0C0C0C0C0C0C0C0C0C0C0C0C78
:105870000C0C0C0C0C0C0C0C0C0C0C0C0C0C0C0C68
:1058800008080808080808080C0C0C0C0C0C0C0C78
:105890000C0C0C0C0C0C0C0C0C0C0C0C0C0C0C0C48
:1058A0000C0C0C0C0C0C0C0C0C0C0C0C0C0C0C0C38
:1058B0000C0C0C0C0C0C0C0C0C0C0C0C0C0C0C0C28
:1058C00008080808080808080C0C0C0C0C0C0C0C38
:1058D0000C0C0C0C0C0C0C0C0C0C0C0C0C0C0C0C08
:1058E0000C0C0C0C0C0C0C0C0C0C0C0C0C0C0C0CF8
:1058F0000C0C0C0C0C0C0C0C0C0C0C0C0C0C0C0CE8
:1059000008080808080808080C0C0C0C0C0C0C0CF7
:105910000C0C0C0C0C0C0C0C0C0C0C0C0C0C0C0CC7
:105920000C0C0C0C0C0C0C0C0C0C0C0C0C0C0C0CB7
:105930000C0C0C0C0C0C0C0C0C0C0C0C0C0C0C0CA7
:1059400008080808080808080C0C0C0C0C0C0C0CB7
:105950000C0C0C0C0C0C0C0C0C0C0C0C0C0C0C0C87
:105960000C0C0C0C0C0C0C0C0C0C0C0C0C0C0C0C77
:105970000C0C0C0C0C0C0C0C0C0C0C0C0C0C0C0C67
:1059800008080808080808080C0C0C0C0C0C0C0C77
:105990000C0C0C0C0C0C0C0C0C0C0C0C0C0C0C0C47
:1059A0000C0C0C0C0C0C0C0C0C0C0C0C0C0C0C0C37
:1059B0000C0C0C0C0C0C0C0C0C0C0C0C0C0C0C0C27
:1059C00008080808080808080C0C0C0C0C0C0C0C37
:1059D0000C0C0C0C0C0C0C0C0C0C0C0C0C0C0C0C07
:1059E0000C0C0C0C0C0C0C0C0C0C0C0C0C0C0C0CF7
:1059F0000C0C0C0C0C0C0C0C0C0C0C0C0C0C0C0CE7
:105A000008080808080808080C0C0C0C0C0C0C0CF6
:105A10000C0C0C0C0C0C0C0C0C0C0C0C0C0C0C0CC6
:105A20000C0C0C0C0C0C0C0C0C0C0C0C0C0C0C0CB6
:105A30000C0C0C0C0C0C0C0C0C0C0C0C0C0C0C0CA6
:105A400008080808080808080C0C0C0C0C0C0C0CB6
:105A50000C0C0C0C0C0C0C0C0C0C0C0C0C0C0C0C86
:105A60000C0C0C0C0C0C0C0C0C0C0C0C0C0C0C0C76
:105A70000C0C0C0C0C0C0C0C0C0C0C0C0C0C0C0C66
:105A800008080808080808080C0C0C0C0C0C0C0C76
:105A90000C0C0C0C0C0C0C0C0C0C0C0C0C0C0C0C46
:105AA0000C0C0C0C0C0C0C0C0C0C0C0C0C0C0C0C36
:105AB0000C0C0C0C0C0C0C0C0C0C0C0C0C0C0C0C26
:105AC00008080808080808080C0C0C0C0C0C0C0C36
:105AD0000C0C0C0C0C0C0C0C0C0C0C0C0C0C0C0C06
:105AE0000C0C0C0C0C0C0C0C0C0C0C0C0C0C0C0CF6
:105AF0000C0C0C0C0C0C0C0C0C0C0C0C0C0C0C0CE6
:105B000008080808080808080C0C0C0C0C0C0C0CF5
:105B10000C0C0C0C0C0C0C0C0C0C0C0C0C0C0C0CC5
:105B20000C0C0C0C0C0C0C0C0C0C0C0C0C0C0C0CB5
:105B30000C0C0C0C0C0C0C0C0C0C0C0C0C0C0C0CA5
:105B400008080808080808080C0C0C0C0C0C0C0CB5
:105B50000C0C0C0C0C0C0C0C0C0C0C0C0C0C0C0C85
:105B60000C0C0C0C0C0C0C0C0C0C0C0C0C0C0C0C75
:105B70000C0C0C0C0C0C0C0C0C0C0C0C0C0C0C0C65
:105B800008080808080808080C0C0C0C0C0C0C0C75
:105B90000C0C0C0C0C0C0C0C0C0C0C0C0C0C0C0C45
:105BA0000C0C0C0C0C0C0C0C0C0C0C0C0C0C0C0C35
:105BB0000C0C0C0C0C0C0C0C0C0C0C0C0C0C0C0C25
:105BC00008080808080808080C0C0C0C0C0C0C0C35
:105BD0000C0C0C0C0C0C0C0C0C0C0C0C0C0C0C0C05
:105BE0000C0C0C0C0C0C0C0C0C0C0C0C0C0C0C0CF5
:105BF0000C0C0C0C0C0C0C0C0C0C0C0C0C0C0C0CE5
:105C000008080808080808080C0C0C0C0C0C0C0CF4
:105C10000C0C0C0C0C0C0C0C0C0C0C0C0C0C0C0CC4
:105C20000C0C0C0C0C0C0C0C0C0C0C0C0C0C0C0CB4
:105C30000C0C0C0C0C0C0C0C0C0C0C0C0C0C0C0CA4
:105C400008080808080808080C0C0C0C0C0C0C0CB4
:105C50000C0C0C0C0C0C0C0C0C0C0C0C0C0C0C0C84
:105C60000C0C0C0C0C0C0C0C0C0C0C0C0C0C0C0C74
:105C70000C0C0C0C0C0C0C0C0C0C0C0C0C0C0C0C64
:105C800008080808080808080C0C0C0C0C0C0C0C74
:105C90000C0C0C0C0C0C0C0C0C0C0C0C0C0C0C0C44
:105CA0000C0C0C0C0C0C0C0C0C0C0C0C0C0C0C0C34
:105CB0000C0C0C0C0C0C0C0C0C0C0C0C0C0C0C0C24
:105CC00008080808080808080C0C0C0C0C0C0C0C34
:105CD0000C0C0C0C0C0C0C0C0C0C0C0C0C0C0C0C04
:105CE0000C0C0C0C0C0C0C0C0C0C0C0C0C0C0C0CF4
:105CF0000C0C0C0C0C0C0C0C0C0C0C0C0C0C0C0CE4
:105D000008080808080808080C0C0C0C0C0C0C0CF3
:105D10000C0C0C0C0C0C0C0C0C0C0C0C0C0C0C0CC3
:105D20000C0C0C0C0C0C0C0C0C0C0C0C0C0C0C0CB3
:105D30000C0C0C0C0C0C0C0C0C0C0C0C0C0C0C0CA3
:105D400008080808080808080C0C0C0C0C0C0C0CB3
:105D50000C0C0C0C0C0C0C0C0C0C0C0C0C0C0C0C83
:105D60000C0C0C0C0C0C0C0C0C0C0C0C0C0C0C0C73
:105D70000C0C0C0C0C0C0C0C0C0C0C0C0C0C0C0C63
:105D800008080808080808080C0C0C0C0C0C0C0C73
:105D90000C0C0C0C0C0C0C0C0C0C0C0C0C0C0C0C43
:105DA0000C0C0C0C0C0C0C0C0C0C0C0C0C0C0C0C33
:105DB0000C0C0C0C0C0C0C0C0C0C0C0C0C0C0C0C23
:105DC00008080808080808080C0C0C0C0C0C0C0C33
:105DD0000C0C0C0C0C0C0C0C0C0C0C0C0C0C0C0C03
:105DE0000C0C0C0C0C0C0C0C0C0C0C0C0C0C0C0CF3
:105DF0000C0C0C0C0C0C0C0C0C0C0C0C0C0C0C0CE3
:105E000008080808080808080C0C0C0C0C0C0C0CF2
:105E10000C0C0C0C0C0C0C0C0C0C0C0C0C0C0C0CC2
:105E20000C0C0C0C0C0C0C0C0C0C0C0C0C0C0C0CB2
:105E30000C0C0C0C0C0C0C0C0C0C0C0C0C0C0C0CA2
:105E400008080808080808080C0C0C0C0C0C0C0CB2
:105E50000C0C0C0C0C0C0C0C0C0C0C0C0C0C0C0C82
:105E60000C0C0C0C0C0C0C0C0C0C0C0C0C0C0C0C72
:105E70000C0C0C0C0C0C0C0C0C0C0C0C0C0C0C0C62
:105E800008080808080808080C0C0C0C0C0C0C0C72
:105E90000C0C0C0C0C0C0C0C0C0C0C0C0C0C0C0C42
:105EA0000C0C0C0C0C0C0C0C0C0C0C0C0C0C0C0C32
:105EB0000C0C0C0C0C0C0C0C0C0C0C0C0C0C0C0C22
:105EC00008080808080808080C0C0C0C0C0C0C0C32
:105ED0000C0C0C0C0C0C0C0C0C0C0C0C0C0C0C0C02
:105EE0000C0C0C0C0C0C0C0C0C0C0C0C0C0C0C0CF2
:105EF0000C0C0C0C0C0C0C0C0C0C0C0C0C0C0C0CE2
:105F000008080808080808080C0C0C0C0C0C0C0CF1
:105F10000C0C0C0C0C0C0C0C0C0C0C0C0C0C0C0CC1
:105F20000C0C0C0C0C0C0C0C0C0C0C0C0C0C0C0CB1
:105F30000C0C0C0C0C0C0C0C0C0C0C0C0C0C0C0CA1
:105F400008080808080808080C0C0C0C0C0C0C0CB1
:105F50000C0C0C0C0C0C0C0C0C0C0C0C0C0C0C0C81
:105F60000C0C0C0C0C0C0C0C0C0C0C0C0C0C0C0C71
:105F70000C0C0C0C0C0C0C0C0C0C0C0C0C0C0C0C61
:105F800008080808080808080C0C0C0C0C0C0C0C71
:105F90000C0C0C0C0C0C0C0C0C0C0C0C0C0C0C0C41
:105FA0000C0C0C0C0C0C0C0C0C0C0C0C0C0C0C0C31
:105FB0000C0C0C0C0C0C0C0C0C0C0C0C0C0C0C0C21
:105FC00008080808080808080C0C0C0C0C0C0C0C31
:105FD0000C0C0C0C0C0C0C0C0C0C0C0C0C0C0C0C01
:105FE0000C0C0C0C0C0C0C0C0C0C0C0C0C0C0C0CF1
:105FF0000C0C0C0C0C0C0C0C0C0C0C0C0C0C0C0CE1
:1060000008080808080808080C0C0C0C0C0C0C0CF0
:106010000C0C0C0C0C0C0C0C0C0C0C0C0C0C0C0CC0
:106020000C0C0C0C0C0C0C0C0C0C0C0C0C0C0C0CB0
:106030000C0C0C0C0C0C0C0C0C0C0C0C0C0C0C0CA0
:1060400008080808080808080C0C0C0C0C0C0C0CB0
:106050000C0C0C0C0C0C0C0C0C0C0C0C0C0C0C0C80
:106060000C0C0C0C0C0C0C0C0C0C0C0C0C0C0C0C70
:106070000C0C0C0C0C0C0C0C0C0C0C0C0C0C0C0C60
:1060800008080808080808080C0C0C0C0C0C0C0C70
:106090000C0C0C0C0C0C0C0C0C0C0C0C0C0C0C0C40
:1060A0000C0C0C0C0C0C0C0C0C0C0C0C0C0C0C0C30
:1060B0000C0C0C0C0C0C0C0C0C0C0C0C0C0C0C0C20
:1060C00008080808080808080C0C0C0C0C0C0C0C30
:1060D0000C0C0C0C0C0C0C0C0C0C0C0C0C0C0C0C00
:1060E0000C0C0C0C0C0C0C0C0C0C0C0C0C0C0C0CF0
:1060F0000C0C0C0C0C0C0C0C0C0C0C0C0C0C0C0CE0
:1061000008080808080808080C0C0C0C0C0C0C0CEF
:106110000C0C0C0C0C0C0C0C0C0C0C0C0C0C0C0CBF
:106120000C0C0C0C0C0C0C0C0C0C0C0C0C0C0C0CAF
:106130000C0C0C0C0C0C0C0C0C0C0C0C0C0C0C0C9F
:1061400008080808080808080C0C0C0C0C0C0C0CAF
:106150000C0C0C0C0C0C0C0C0C0C0C0C0C0C0C0C7F
:106160000C0C0C0C0C0C0C0C0C0C0C0C0C0C0C0C6F
:106170000C0C0C0C0C0C0C0C0C0C0C0C0C0C0C0C5F
:1061800008080808080808080C0C0C0C0C0C0C0C6F
:106190000C0C0C0C0C0C0C0C0C0C0C0C0C0C0C0C3F
:1061A0000C0C0C0C0C0C0C0C0C0C0C0C0C0C0C0C2F
:1061B0000C0C0C0C0C0C0C0C0C0C0C0C0C0C0C0C1F
:1061C00008080808080808080C0C0C0C0C0C0C0C2F
:1061D0000C0C0C0C0C0C0C0C0C0C0C0C0C0C0C0CFF
:1061E0000C0C0C0C0C0C0C0C0C0C0C0C0C0C0C0CEF
:1061F0000C0C0C0C0C0C0C0C0C0C0C0C0C0C0C0CDF
:1062000008080808080808080C0C0C0C0C0C0C0CEE
:106210000C0C0C0C0C0C0C0C0C0C0C0C0C0C0C0CBE
:106220000C0C0C0C0C0C0C0C0C0C0C0C0C0C0C0CAE
:106230000C0C0C0C0C0C0C0C0C0C0C0C0C0C0C0C9E
:1062400008080808080808080C0C0C0C0C0C0C0CAE
:106250000C0C0C0C0C0C0C0C0C0C0C0C0C0C0C0C7E
:106260000C0C0C0C0C0C0C0C0C0C0C0C0C0C0C0C6E
:106270000C0C0C0C0C0C0C0C0C0C0C0C0C0C0C0C5E
:1062800008080808080808080C0C0C0C0C0C0C0C6E
:106290000C0C0C0C0C0C0C0C0C0C0C0C0C0C0C0C3E
:1062A0000C0C0C0C0C0C0C0C0C0C0C0C0C0C0C0C2E
:1062B0000C0C0C0C0C0C0C0C0C0C0C0C0C0C0C0C1E
:1062C00008080808080808080C0C0C0C0C0C0C0C2E
:1062D0000C0C0C0C0C0C0C0C0C0C0C0C0C0C0C0CFE
:1062E0000C0C0C0C0C0C0C0C0C0C0C0C0C0C0C0CEE
:1062F0000C0C0C0C0C0C0C0C0C0C0C0C0C0C0C0CDE
:1063000008080808080808080C0C0C0C0C0C0C0CED
:106310000C0C0C0C0C0C0C0C0C0C0C0C0C0C0C0CBD
:106320000C0C0C0C0C0C0C0C0C0C0C0C0C0C0C0CAD
:106330000C0C0C0C0C0C0C0C0C0C0C0C0C0C0C0C9D
:1063400008080808080808080C0C0C0C0C0C0C0CAD
:106350000C0C0C0C0C0C0C0C0C0C0C0C0C0C0C0C7D
:106360000C0C0C0C0C0C0C0C0C0C0C0C0C0C0C0C6D
:106370000C0C0C0C0C0C0C0C0C0C0C0C0C0C0C0C5D
:1063800008080808080808080C0C0C0C0C0C0C0C6D
:106390000C0C0C0C0C0C0C0C0C0C0C0C0C0C0C0C3D
:1063A0000C0C0C0C0C0C0C0C0C0C0C0C0C0C0C0C2D
:1063B0000C0C0C0C0C0C0C0C0C0C0C0C0C0C0C0C1D
:1063C00008080808080808080C0C0C0C0C0C0C0C2D
:1063D0000C0C0C0C0C0C0C0C0C0C0C0C0C0C0C0CFD
:1063E0000C0C0C0C0C0C0C0C0C0C0C0C0C0C0C0CED
:1063F0000C0C0C0C0C0C0C0C0C0C0C0C0C0C0C0CDD
:1064000008080808080808080C0C0C0C0C0C0C0CEC
:106410000C0C0C0C0C0C0C0C0C0C0C0C0C0C0C0CBC
:106420000C0C0C0C0C0C0C0C0C0C0C0C0C0C0C0CAC
:106430000C0C0C0C0C0C0C0C0C0C0C0C0C0C0C0C9C
:1064400008080808080808080C0C0C0C0C0C0C0CAC
:106450000C0C0C0C0C0C0C0C0C0C0C0C0C0C0C0C7C
:106460000C0C0C0C0C0C0C0C0C0C0C0C0C0C0C0C6C
:106470000C0C0C0C0C0C0C0C0C0C0C0C0C0C0C0C5C
:1064800008080808080808080C0C0C0C0C0C0C0C6C
:106490000C0C0C0C0C0C0C0C0C0C0C0C0C0C0C0C3C
:1064A0000C0C0C0C0C0C0C0C0C0C0C0C0C0C0C0C2C
:1064B0000C0C0C0C0C0C0C0C0C0C0C0C0C0C0C0C1C
:1064C00008080808080808080C0C0C0C0C0C0C0C2C
:1064D0000C0C0C0C0C0C0C0C0C0C0C0C0C0C0C0CFC
:1064E0000C0C0C0C0C0C0C0C0C0C0C0C0C0C0C0CEC
:1064F0000C0C0C0C0C0C0C0C0C0C0C0C0C0C0C0CDC
:1065000008080808080808080C0C0C0C0C0C0C0CEB
:106510000C0C0C0C0C0C0C0C0C0C0C0C0C0C0C0CBB
:106520000C0C0C0C0C0C0C0C0C0C0C0C0C0C0C0CAB
:106530000C0C0C0C0C0C0C0C0C0C0C0C0C0C0C0C9B
:1065400008080808080808080C0C0C0C0C0C0C0CAB
:106550000C0C0C0C0C0C0C0C0C0C0C0C0C0C0C0C7B
:106560000C0C0C0C0C0C0C0C0C0C0C0C0C0C0C0C6B
:106570000C0C0C0C0C0C0C0C0C0C0C0C0C0C0C0C5B
:1065800008080808080808080C0C0C0C0C0C0C0C6B
:106590000C0C0C0C0C0C0C0C0C0C0C0C0C0C0C0C3B
:1065A0000C0C0C0C0C0C0C0C0C0C0C0C0C0C0C0C2B
:1065B0000C0C0C0C0C0C0C0C0C0C0C0C0C0C0C0C1B
:1065C00008080808080808080C0C0C0C0C0C0C0C2B
:1065D0000C0C0C0C0C0C0C0C0C0C0C0C0C0C0C0CFB
:1065E0000C0C0C0C0C0C0C0C0C0C0C0C0C0C0C0CEB
:1065F0000C0C0C0C0C0C0C0C0C0C0C0C0C0C0C0CDB
:1066000008080808080808080C0C0C0C0C0C0C0CEA
:106610000C0C0C0C0C0C0C0C0C0C0C0C0C0C0C0CBA
:106620000C0C0C0C0C0C0C0C0C0C0C0C0C0C0C0CAA
:106630000C0C0C0C0C0C0C0C0C0C0C0C0C0C0C0C9A
:1066400008080808080808080C0C0C0C0C0C0C0CAA
:106650000C0C0C0C0C0C0C0C0C0C0C0C0C0C0C0C7A
:106660000C0C0C0C0C0C0C0C0C0C0C0C0C0C0C0C6A
:106670000C0C0C0C0C0C0C0C0C0C0C0C0C0C0C0C5A
:1066800008080808080808080C0C0C0C0C0C0C0C6A
:106690000C0C0C0C0C0C0C0C0C0C0C0C0C0C0C0C3A
:1066A0000C0C0C0C0C0C0C0C0C0C0C0C0C0C0C0C2A
:1066B0000C0C0C0C0C0C0C0C0C0C0C0C0C0C0C0C1A
:1066C00008080808080808080C0C0C0C0C0C0C0C2A
:1066D0000C0C0C0C0C0C0C0C0C0C0C0C0C0C0C0CFA
:1066E0000C0C0C0C0C0C0C0C0C0C0C0C0C0C0C0CEA
:1066F0000C0C0C0C0C0C0C0C0C0C0C0C0C0C0C0CDA
:1067000008080808080808080C0C0C0C0C0C0C0CE9
:106710000C0C0C0C0C0C0C0C0C0C0C0C0C0C0C0CB9
:106720000C0C0C0C0C0C0C0C0C0C0C0C0C0C0C0CA9
:106730000C0C0C0C0C0C0C0C0C0C0C0C0C0C0C0C99
:1067400008080808080808080C0C0C0C0C0C0C0CA9
:106750000C0C0C0C0C0C0C0C0C0C0C0C0C0C0C0C79
:106760000C0C0C0C0C0C0C0C0C0C0C0C0C0C0C0C69
:106770000C0C0C0C0C0C0C0C0C0C0C0C0C0C0C0C59
:1067800008080808080808080C0C0C0C0C0C0C0C69
:106790000C0C0C0C0C0C0C0C0C0C0C0C0C0C0C0C39
:1067A0000C0C0C0C0C0C0C0C0C0C0C0C0C0C0C0C29
:1067B0000C0C0C0C0C0C0C0C0C0C0C0C0C0C0C0C19
:1067C00008080808080808080C0C0C0C0C0C0C0C29
:1067D0000C0C0C0C0C0C0C0C0C0C0C0C0C0C0C0CF9
:1067E0000C0C0C0C0C0C0C0C0C0C0C0C0C0C0C0CE9
:1067F0000C0C0C0C0C0C0C0C0C0C0C0C0C0C0C0CD9
:1068000008080808080808080C0C0C0C0C0C0C0CE8
:106810000C0C0C0C0C0C0C0C0C0C0C0C0C0C0C0CB8
:106820000C0C0C0C0C0C0C0C0C0C0C0C0C0C0C0CA8
:106830000C0C0C0C0C0C0C0C0C0C0C0C0C0C0C0C98
:1068400008080808080808080C0C0C0C0C0C0C0CA8
:106850000C0C0C0C0C0C0C0C0C0C0C0C0C0C0C0C78
:106860000C0C0C0C0C0C0C0C0C0C0C0C0C0C0C0C68
:106870000C0C0C0C0C0C0C0C0C0C0C0C0C0C0C0C58
:1068800008080808080808080C0C0C0C0C0C0C0C68
:106890000C0C0C0C0C0C0C0C0C0C0C0C0C0C0C0C38
:1068A0000C0C0C0C0C0C0C0C0C0C0C0C0C0C0C0C28
:1068B0000C0C0C0C0C0C0C0C0C0C0C0C0C0C0C0C18
:1068C00008080808080808080C0C0C0C0C0C0C0C28
:1068D0000C0C0C0C0C0C0C0C0C0C0C0C0C0C0C0CF8
:1068E0000C0C0C0C0C0C0C0C0C0C0C0C0C0C0C0CE8
:1068F0000C0C0C0C0C0C0C0C0C0C0C0C0C0C0C0CD8
:1069000008080808080808080C0C0C0C0C0C0C0CE7
:106910000C0C0C0C0C0C0C0C0C0C0C0C0C0C0C0CB7
:106920000C0C0C0C0C0C0C0C0C0C0C0C0C0C0C0CA7
:106930000C0C0C0C0C0C0C0C0C0C0C0C0C0C0C0C97
:1069400008080808080808080C0C0C0C0C0C0C0CA7
:106950000C0C0C0C0C0C0C0C0C0C0C0C0C0C0C0C77
:106960000C0C0C0C0C0C0C0C0C0C0C0C0C0C0C0C67
:106970000C0C0C0C0C0C0C0C0C0C0C0C0C0C0C0C57
:1069800008080808080808080C0C0C0C0C0C0C0C67
:106990000C0C0C0C0C0C0C0C0C0C0C0C0C0C0C0C37
:1069A0000C0C0C0C0C0C0C0C0C0C0C0C0C0C0C0C27
:1069B0000C0C0C0C0C0C0C0C0C0C0C0C0C0C0C0C17
:1069C00008080808080808080C0C0C0C0C0C0C0C27
:1069D0000C0C0C0C0C0C0C0C0C0C0C0C0C0C0C0CF7
:1069E0000C0C0C0C0C0C0C0C0C0C0C0C0C0C0C0CE7
:1069F0000C0C0C0C0C0C0C0C0C0C0C0C0C0C0C0CD7
:106A000008080808080808080C0C0C0C0C0C0C0CE6
:106A10000C0C0C0C0C0C0C0C0C0C0C0C0C0C0C0CB6
:106A20000C0C0C0C0C0C0C0C0C0C0C0C0C0C0C0CA6
:106A30000C0C0C0C0C0C0C0C0C0C0C0C0C0C0C0C96
:106A400008080808080808080C0C0C0C0C0C0C0CA6
:106A50000C0C0C0C0C0C0C0C0C0C0C0C0C0C0C0C76
:106A60000C0C0C0C0C0C0C0C0C0C0C0C0C0C0C0C66
:106A70000C0C0C0C0C0C0C0C0C0C0C0C0C0C0C0C56
:106A800008080808080808080C0C0C0C0C0C0C0C66
:106A90000C0C0C0C0C0C0C0C0C0C0C0C0C0C0C0C36
:106AA0000C0C0C0C0C0C0C0C0C0C0C0C0C0C0C0C26
:106AB0000C0C0C0C0C0C0C0C0C0C0C0C0C0C0C0C16
:106AC00008080808080808080C0C0C0C0C0C0C0C26
:106AD0000C0C0C0C0C0C0C0C0C0C0C0C0C0C0C0CF6
:106AE0000C0C0C0C0C0C0C0C0C0C0C0C0C0C0C0CE6
:106AF0000C0C0C0C0C0C0C0C0C0C0C0C0C0C0C0CD6
:106B000008080808080808080C0C0C0C0C0C0C0CE5
:106B10000C0C0C0C0C0C0C0C0C0C0C0C0C0C0C0CB5
:106B20000C0C0C0C0C0C0C0C0C0C0C0C0C0C0C0CA5
:106B30000C0C0C0C0C0C0C0C0C0C0C0C0C0C0C0C95
:106B400008080808080808080C0C0C0C0C0C0C0CA5
:106B50000C0C0C0C0C0C0C0C0C0C0C0C0C0C0C0C75
:106B60000C0C0C0C0C0C0C0C0C0C0C0C0C0C0C0C65
:106B70000C0C0C0C0C0C0C0C0C0C0C0C0C0C0C0C55
:106B800008080808080808080C0C0C0C0C0C0C0C65
:106B90000C0C0C0C0C0C0C0C0C0C0C0C0C0C0C0C35
:106BA0000C0C0C0C0C0C0C0C0C0C0C0C0C0C0C0C25
:106BB0000C0C0C0C0C0C0C0C0C0C0C0C0C0C0C0C15
:106BC00008080808080808080C0C0C0C0C0C0C0C25
:106BD0000C0C0C0C0C0C0C0C0C0C0C0C0C0C0C0CF5
:106BE0000C0C0C0C0C0C0C0C0C0C0C0C0C0C0C0CE5
:106BF0000C0C0C0C0C0C0C0C0C0C0C0C0C0C0C0CD5
:106C000008080808080808080C0C0C0C0C0C0C0CE4
:106C10000C0C0C0C0C0C0C0C0C0C0C0C0C0C0C0CB4
:106C20000C0C0C0C0C0C0C0C0C0C0C0C0C0C0C0CA4
:106C30000C0C0C0C0C0C0C0C0C0C0C0C0C0C0C0C94
:106C400008080808080808080C0C0C0C0C0C0C0CA4
:106C50000C0C0C0C0C0C0C0C0C0C0C0C0C0C0C0C74
:106C60000C0C0C0C0C0C0C0C0C0C0C0C0C0C0C0C64
:106C70000C0C0C0C0C0C0C0C0C0C0C0C0C0C0C0C54
:106C800008080808080808080C0C0C0C0C0C0C0C64
:106C90000C0C0C0C0C0C0C0C0C0C0C0C0C0C0C0C34
:106CA0000C0C0C0C0C0C0C0C0C0C0C0C0C0C0C0C24
:106CB0000C0C0C0C0C0C0C0C0C0C0C0C0C0C0C0C14
:106CC00008080808080808080C0C0C0C0C0C0C0C24
:106CD0000C0C0C0C0C0C0C0C0C0C0C0C0C0C0C0CF4
:106CE0000C0C0C0C0C0C0C0C0C0C0C0C0C0C0C0CE4
:106CF0000C0C0C0C0C0C0C0C0C0C0C0C0C0C0C0CD4
:106D000008080808080808080C0C0C0C0C0C0C0CE3
:106D10000C0C0C0C0C0C0C0C0C0C0C0C0C0C0C0CB3
:106D20000C0C0C0C0C0C0C0C0C0C0C0C0C0C0C0CA3
:106D30000C0C0C0C0C0C0C0C0C0C0C0C0C0C0C0C93
:106D400008080808080808080C0C0C0C0C0C0C0CA3
:106D50000C0C0C0C0C0C0C0C0C0C0C0C0C0C0C0C73
:106D60000C0C0C0C0C0C0C0C0C0C0C0C0C0C0C0C63
:106D70000C0C0C0C0C0C0C0C0C0C0C0C0C0C0C0C53
:106D800008080808080808080C0C0C0C0C0C0C0C63
:106D90000C0C0C0C0C0C0C0C0C0C0C0C0C0C0C0C33
:106DA0000C0C0C0C0C0C0C0C0C0C0C0C0C0C0C0C23
:106DB0000C0C0C0C0C0C0C0C0C0C0C0C0C0C0C0C13
:106DC00008080808080808080C0C0C0C0C0C0C0C23
:106DD0000C0C0C0C0C0C0C0C0C0C0C0C0C0C0C0CF3
:106DE0000C0C0C0C0C0C0C0C0C0C0C0C0C0C0C0CE3
:106DF0000C0C0C0C0C0C0C0C0C0C0C0C0C0C0C0CD3
:106E000008080808080808080C0C0C0C0C0C0C0CE2
:106E10000C0C0C0C0C0C0C0C0C0C0C0C0C0C0C0CB2
:106E20000C0C0C0C0C0C0C0C0C0C0C0C0C0C0C0CA2
:106E30000C0C0C0C0C0C0C0C0C0C0C0C0C0C0C0C92
:106E400008080808080808080C0C0C0C0C0C0C0CA2
:106E50000C0C0C0C0C0C0C0C0C0C0C0C0C0C0C0C72
:106E60000C0C0C0C0C0C0C0C0C0C0C0C0C0C0C0C62
:106E70000C0C0C0C0C0C0C0C0C0C0C0C0C0C0C0C52
:106E800008080808080808080C0C0C0C0C0C0C0C62
:106E90000C0C0C0C0C0C0C0C0C0C0C0C0C0C0C0C32
:106EA0000C0C0C0C0C0C0C0C0C0C0C0C0C0C0C0C22
:106EB0000C0C0C0C0C0C0C0C0C0C0C0C0C0C0C0C12
:106EC00008080808080808080C0C0C0C0C0C0C0C22
:106ED0000C0C0C0C0C0C0C0C0C0C0C0C0C0C0C0CF2
:106EE0000C0C0C0C0C0C0C0C0C0C0C0C0C0C0C0CE2
:106EF0000C0C0C0C0C0C0C0C0C0C0C0C0C0C0C0CD2
:106F000008080808080808080C0C0C0C0C0C0C0CE1
:106F10000C0C0C0C0C0C0C0C0C0C0C0C0C0C0C0CB1
:106F20000C0C0C0C0C0C0C0C0C0C0C0C0C0C0C0CA1
:106F30000C0C0C0C0C0C0C0C0C0C0C0C0C0C0C0C91
:106F400008080808080808080C0C0C0C0C0C0C0CA1
:106F50000C0C0C0C0C0C0C0C0C0C0C0C0C0C0C0C71
:106F60000C0C0C0C0C0C0C0C0C0C0C0C0C0C0C0C61
:106F70000C0C0C0C0C0C0C0C0C0C0C0C0C0C0C0C51
:106F800008080808080808080C0C0C0C0C0C0C0C61
:106F90000C0C0C0C0C0C0C0C0C0C0C0C0C0C0C0C31
:106FA0000C0C0C0C0C0C0C0C0C0C0C0C0C0C0C0C21
:106FB0000C0C0C0C0C0C0C0C0C0C0C0C0C0C0C0C11
:106FC00008080808080808080C0C0C0C0C0C0C0C21
:106FD0000C0C0C0C0C0C0C0C0C0C0C0C0C0C0C0CF1
:106FE0000C0C0C0C0C0C0C0C0C0C0C0C0C0C0C0CE1
:106FF0000C0C0C0C0C0C0C0C0C0C0C0C0C0C0C0CD1
:1070000008080808080808080C0C0C0C0C0C0C0CE0
:107010000C0C0C0C0C0C0C0C0C0C0C0C0C0C0C0CB0
:107020000C0C0C0C0C0C0C0C0C0C0C0C0C0C0C0CA0
:107030000C0C0C0C0C0C0C0C0C0C0C0C0C0C0C0C90
:1070400008080808080808080C0C0C0C0C0C0C0CA0
:107050000C0C0C0C0C0C0C0C0C0C0C0C0C0C0C0C70
:107060000C0C0C0C0C0C0C0C0C0C0C0C0C0C0C0C60
:107070000C0C0C0C0C0C0C0C0C0C0C0C0C0C0C0C50
:1070800008080808080808080C0C0C0C0C0C0C0C60
:107090000C0C0C0C0C0C0C0C0C0C0C0C0C0C0C0C30
:1070A0000C0C0C0C0C0C0C0C0C0C0C0C0C0C0C0C20
:1070B0000C0C0C0C0C0C0C0C0C0C0C0C0C0C0C0C10
:1070C00008080808080808080C0C0C0C0C0C0C0C20
:1070D0000C0C0C0C0C0C0C0C0C0C0C0C0C0C0C0CF0
:1070E0000C0C0C0C0C0C0C0C0C0C0C0C0C0C0C0CE0
:1070F0000C0C0C0C0C0C0C0C0C0C0C0C0C0C0C0CD0
:1071000008080808080808080C0C0C0C0C0C0C0CDF
:107110000C0C0C0C0C0C0C0C0C0C0C0C0C0C0C0CAF
:107120000C0C0C0C0C0C0C0C0C0C0C0C0C0C0C0C9F
:107130000C0C0C0C0C0C0C0C0C0C0C0C0C0C0C0C8F
:1071400008080808080808080C0C0C0C0C0C0C0C9F
:107150000C0C0C0C0C0C0C0C0C0C0C0C0C0C0C0C6F
:107160000C0C0C0C0C0C0C0C0C0C0C0C0C0C0C0C5F
:107170000C0C0C0C0C0C0C0C0C0C0C0C0C0C0C0C4F
:1071800008080808080808080C0C0C0C0C0C0C0C5F
:107190000C0C0C0C0C0C0C0C0C0C0C0C0C0C0C0C2F
:1071A0000C0C0C0C0C0C0C0C0C0C0C0C0C0C0C0C1F
:1071B0000C0C0C0C0C0C0C0C0C0C0C0C0C0C0C0C0F
:1071C00008080808080808080C0C0C0C0C0C0C0C1F
:1071D0000C0C0C0C0C0C0C0C0C0C0C0C0C0C0C0CEF
:1071E0000C0C0C0C0C0C0C0C0C0C0C0C0C0C0C0CDF
:1071F0000C0C0C0C0C0C0C0C0C0C0C0C0C0C0C0CCF
:1072000008080808080808080C0C0C0C0C0C0C0CDE
:107210000C0C0C0C0C0C0C0C0C0C0C0C0C0C0C0CAE
:107220000C0C0C0C0C0C0C0C0C0C0C0C0C0C0C0C9E
:107230000C0C0C0C0C0C0C0C0C0C0C0C0C0C0C0C8E
:1072400008080808080808080C0C0C0C0C0C0C0C9E
:107250000C0C0C0C0C0C0C0C0C0C0C0C0C0C0C0C6E
:107260000C0C0C0C0C0C0C0C0C0C0C0C0C0C0C0C5E
:107270000C0C0C0C0C0C0C0C0C0C0C0C0C0C0C0C4E
:1072800008080808080808080C0C0C0C0C0C0C0C5E
:107290000C0C0C0C0C0C0C0C0C0C0C0C0C0C0C0C2E
:1072A0000C0C0C0C0C0C0C0C0C0C0C0C0C0C0C0C1E
:1072B0000C0C0C0C0C0C0C0C0C0C0C0C0C0C0C0C0E
:1072C00008080808080808080C0C0C0C0C0C0C0C1E
:1072D0000C0C0C0C0C0C0C0C0C0C0C0C0C0C0C0CEE
:1072E0000C0C0C0C0C0C0C0C0C0C0C0C0C0C0C0CDE
:1072F0000C0C0C0C0C0C0C0C0C0C0C0C0C0C0C0CCE
:1073000008080808080808080C0C0C0C0C0C0C0CDD
:107310000C0C0C0C0C0C0C0C0C0C0C0C0C0C0C0CAD
:107320000C0C0C0C0C0C0C0C0C0C0C0C0C0C0C0C9D
:107330000C0C0C0C0C0C0C0C0C0C0C0C0C0C0C0C8D
:1073400008080808080808080C0C0C0C0C0C0C0C9D
:107350000C0C0C0C0C0C0C0C0C0C0C0C0C0C0C0C6D
:107360000C0C0C0C0C0C0C0C0C0C0C0C0C0C0C0C5D
:107370000C0C0C0C0C0C0C0C0C0C0C0C0C0C0C0C4D
:1073800008080808080808080C0C0C0C0C0C0C0C5D
:107390000C0C0C0C0C0C0C0C0C0C0C0C0C0C0C0C2D
:1073A0000C0C0C0C0C0C0C0C0C0C0C0C0C0C0C0C1D
:1073B0000C0C0C0C0C0C0C0C0C0C0C0C0C0C0C0C0D
:1073C00008080808080808080C0C0C0C0C0C0C0C1D
:1073D0000C0C0C0C0C0C0C0C0C0C0C0C0C0C0C0CED
:1073E0000C0C0C0C0C0C0C0C0C0C0C0C0C0C0C0CDD
:1073F0000C0C0C0C0C0C0C0C0C0C0C0C0C0C0C0CCD
:1074000008080808080808080C0C0C0C0C0C0C0CDC
:107410000C0C0C0C0C0C0C0C0C0C0C0C0C0C0C0CAC
:107420000C0C0C0C0C0C0C0C0C0C0C0C0C0C0C0C9C
:107430000C0C0C0C0C0C0C0C0C0C0C0C0C0C0C0C8C
:1074400008080808080808080C0C0C0C0C0C0C0C9C
:107450000C0C0C0C0C0C0C0C0C0C0C0C0C0C0C0C6C
:107460000C0C0C0C0C0C0C0C0C0C0C0C0C0C0C0C5C
:107470000C0C0C0C0C0C0C0C0C0C0C0C0C0C0C0C4C
:1074800008080808080808080C0C0C0C0C0C0C0C5C
:107490000C0C0C0C0C0C0C0C0C0C0C0C0C0C0C0C2C
:1074A0000C0C0C0C0C0C0C0C0C0C0C0C0C0C0C0C1C
:1074B0000C0C0C0C0C0C0C0C0C0C0C0C0C0C0C0C0C
:1074C00008080808080808080C0C0C0C0C0C0C0C1C
:1074D0000C0C0C0C0C0C0C0C0C0C0C0C0C0C0C0CEC
:1074E0000C0C0C0C0C0C0C0C0C0C0C0C0C0C0C0CDC
:1074F0000C0C0C0C0C0C0C0C0C0C0C0C0C0C0C0CCC
:1075000008080808080808080C0C0C0C0C0C0C0CDB
:107510000C0C0C0C0C0C0C0C0C0C0C0C0C0C0C0CAB
:107520000C0C0C0C0C0C0C0C0C0C0C0C0C0C0C0C9B
:107530000C0C0C0C0C0C0C0C0C0C0C0C0C0C0C0C8B
:1075400008080808080808080C0C0C0C0C0C0C0C9B
:107550000C0C0C0C0C0C0C0C0C0C0C0C0C0C0C0C6B
:107560000C0C0C0C0C0C0C0C0C0C0C0C0C0C0C0C5B
:107570000C0C0C0C0C0C0C0C0C0C0C0C0C0C0C0C4B
:1075800008080808080808080C0C0C0C0C0C0C0C5B
:107590000C0C0C0C0C0C0C0C0C0C0C0C0C0C0C0C2B
:1075A0000C0C0C0C0C0C0C0C0C0C0C0C0C0C0C0C1B
:1075B0000C0C0C0C0C0C0C0C0C0C0C0C0C0C0C0C0B
:1075C00008080808080808080C0C0C0C0C0C0C0C1B
:1075D0000C0C0C0C0C0C0C0C0C0C0C0C0C0C0C0CEB
:1075E0000C0C0C0C0C0C0C0C0C0C0C0C0C0C0C0CDB
:1075F0000C0C0C0C0C0C0C0C0C0C0C0C0C0C0C0CCB
:1076000008080808080808080C0C0C0C0C0C0C0CDA
:107610000C0C0C0C0C0C0C0C0C0C0C0C0C0C0C0CAA
:107620000C0C0C0C0C0C0C0C0C0C0C0C0C0C0C0C9A
:107630000C0C0C0C0C0C0C0C0C0C0C0C0C0C0C0C8A
:1076400008080808080808080C0C0C0C0C0C0C0C9A
:107650000C0C0C0C0C0C0C0C0C0C0C0C0C0C0C0C6A
:107660000C0C0C0C0C0C0C0C0C0C0C0C0C0C0C0C5A
:107670000C0C0C0C0C0C0C0C0C0C0C0C0C0C0C0C4A
:1076800008080808080808080C0C0C0C0C0C0C0C5A
:107690000C0C0C0C0C0C0C0C0C0C0C0C0C0C0C0C2A
:1076A0000C0C0C0C0C0C0C0C0C0C0C0C0C0C0C0C1A
:1076B0000C0C0C0C0C0C0C0C0C0C0C0C0C0C0C0C0A
:1076C00008080808080808080C0C0C0C0C0C0C0C1A
:1076D0000C0C0C0C0C0C0C0C0C0C0C0C0C0C0C0CEA
:1076E0000C0C0C0C0C0C0C0C0C0C0C0C0C0C0C0CDA
:1076F0000C0C0C0C0C0C0C0C0C0C0C0C0C0C0C0CCA
:1077000008080808080808080C0C0C0C0C0C0C0CD9
:107710000C0C0C0C0C0C0C0C0C0C0C0C0C0C0C0CA9
:107720000C0C0C0C0C0C0C0C0C0C0C0C0C0C0C0C99
:107730000C0C0C0C0C0C0C0C0C0C0C0C0C0C0C0C89
:1077400008080808080808080C0C0C0C0C0C0C0C99
:107750000C0C0C0C0C0C0C0C0C0C0C0C0C0C0C0C69
:107760000C0C0C0C0C0C0C0C0C0C0C0C0C0C0C0C59
:107770000C0C0C0C0C0C0C0C0C0C0C0C0C0C0C0C49
:1077800008080808080808080C0C0C0C0C0C0C0C59
:107790000C0C0C0C0C0C0C0C0C0C0C0C0C0C0C0C29
:1077A0000C0C0C0C0C0C0C0C0C0C0C0C0C0C0C0C19
:1077B0000C0C0C0C0C0C0C0C0C0C0C0C0C0C0C0C09
:1077C00008080808080808080C0C0C0C0C0C0C0C19
:1077D0000C0C0C0C0C0C0C0C0C0C0C0C0C0C0C0CE9
:1077E0000C0C0C0C0C0C0C0C0C0C0C0C0C0C0C0CD9
:1077F0000C0C0C0C0C0C0C0C0C0C0C0C0C0C0C0CC9
:1078000008080808080808080C0C0C0C0C0C0C0CD8
:107810000C0C0C0C0C0C0C0C0C0C0C0C0C0C0C0CA8
:107820000C0C0C0C0C0C0C0C0C0C0C0C0C0C0C0C98
:107830000C0C0C0C0C0C0C0C0C0C0C0C0C0C0C0C88
:1078400008080808080808080C0C0C0C0C0C0C0C98
:107850000C0C0C0C0C0C0C0C0C0C0C0C0C0C0C0C68
:107860000C0C0C0C0C0C0C0C0C0C0C0C0C0C0C0C58
:107870000C0C0C0C0C0C0C0C0C0C0C0C0C0C0C0C48
:1078800008080808080808080C0C0C0C0C0C0C0C58
:107890000C0C0C0C0C0C0C0C0C0C0C0C0C0C0C0C28
:1078A0000C0C0C0C0C0C0C0C0C0C0C0C0C0C0C0C18
:1078B0000C0C0C0C0C0C0C0C0C0C0C0C0C0C0C0C08
:1078C00008080808080808080C0C0C0C0C0C0C0C18
:1078D0000C0C0C0C0C0C0C0C0C0C0C0C0C0C0C0CE8
:1078E0000C0C0C0C0C0C0C0C0C0C0C0C0C0C0C0CD8
:1078F0000C0C0C0C0C0C0C0C0C0C0C0C0C0C0C0CC8
:1079000008080808080808080C0C0C0C0C0C0C0CD7
:107910000C0C0C0C0C0C0C0C0C0C0C0C0C0C0C0CA7
:107920000C0C0C0C0C0C0C0C0C0C0C0C0C0C0C0C97
:107930000C0C0C0C0C0C0C0C0C0C0C0C0C0C0C0C87
:1079400008080808080808080C0C0C0C0C0C0C0C97
:107950000C0C0C0C0C0C0C0C0C0C0C0C0C0C0C0C67
:107960000C0C0C0C0C0C0C0C0C0C0C0C0C0C0C0C57
:107970000C0C0C0C0C0C0C0C0C0C0C0C0C0C0C0C47
:1079800008080808080808080C0C0C0C0C0C0C0C57
:107990000C0C0C0C0C0C0C0C0C0C0C0C0C0C0C0C27
:1079A0000C0C0C0C0C0C0C0C0C0C0C0C0C0C0C0C17
:1079B0000C0C0C0C0C0C0C0C0C0C0C0C0C0C0C0C07
:1079C00008080808080808080C0C0C0C0C0C0C0C17
:1079D0000C0C0C0C0C0C0C0C0C0C0C0C0C0C0C0CE7
:1079E0000C0C0C0C0C0C0C0C0C0C0C0C0C0C0C0CD7
:1079F0000C0C0C0C0C0C0C0C0C0C0C0C0C0C0C0CC7
:107A000008080808080808080C0C0C0C0C0C0C0CD6
:107A10000C0C0C0C0C0C0C0C0C0C0C0C0C0C0C0CA6
:107A20000C0C0C0C0C0C0C0C0C0C0C0C0C0C0C0C96
:107A30000C0C0C0C0C0C0C0C0C0C0C0C0C0C0C0C86
:107A400008080808080808080C0C0C0C0C0C0C0C96
:107A50000C0C0C0C0C0C0C0C0C0C0C0C0C0C0C0C66
:107A60000C0C0C0C0C0C0C0C0C0C0C0C0C0C0C0C56
:107A70000C0C0C0C0C0C0C0C0C0C0C0C0C0C0C0C46
:107A800008080808080808080C0C0C0C0C0C0C0C56
:107A90000C0C0C0C0C0C0C0C0C0C0C0C0C0C0C0C26
:107AA0000C0C0C0C0C0C0C0C0C0C0C0C0C0C0C0C16
:107AB0000C0C0C0C0C0C0C0C0C0C0C0C0C0C0C0C06
:107AC00008080808080808080C0C0C0C0C0C0C0C16
:107AD0000C0C0C0C0C0C0C0C0C0C0C0C0C0C0C0CE6
:107AE0000C0C0C0C0C0C0C0C0C0C0C0C0C0C0C0CD6
:107AF0000C0C0C0C0C0C0C0C0C0C0C0C0C0C0C0CC6
:107B000008080808080808080C0C0C0C0C0C0C0CD5
:107B10000C0C0C0C0C0C0C0C0C0C0C0C0C0C0C0CA5
:107B20000C0C0C0C0C0C0C0C0C0C0C0C0C0C0C0C95
:107B30000C0C0C0C0C0C0C0C0C0C0C0C0C0C0C0C85
:107B400008080808080808080C0C0C0C0C0C0C0C95
:107B50000C0C0C0C0C0C0C0C0C0C0C0C0C0C0C0C65
:107B60000C0C0C0C0C0C0C0C0C0C0C0C0C0C0C0C55
:107B70000C0C0C0C0C0C0C0C0C0C0C0C0C0C0C0C45
:107B800008080808080808080C0C0C0C0C0C0C0C55
:107B90000C0C0C0C0C0C0C0C0C0C0C0C0C0C0C0C25
:107BA0000C0C0C0C0C0C0C0C0C0C0C0C0C0C0C0C15
:107BB0000C0C0C0C0C0C0C0C0C0C0C0C0C0C0C0C05
:107BC00008080808080808080C0C0C0C0C0C0C0C15
:107BD0000C0C0C0C0C0C0C0C0C0C0C0C0C0C0C0CE5
:107BE0000C0C0C0C0C0C0C0C0C0C0C0C0C0C0C0CD5
:107BF0000C0C0C0C0C0C0C0C0C0C0C0C0C0C0C0CC5
:107C000008080808080808080C0C0C0C0C0C0C0CD4
:107C10000C0C0C0C0C0C0C0C0C0C0C0C0C0C0C0CA4
:107C20000C0C0C0C0C0C0C0C0C0C0C0C0C0C0C0C94
:107C30000C0C0C0C0C0C0C0C0C0C0C0C0C0C0C0C84
:107C400008080808080808080C0C0C0C0C0C0C0C94
:107C50000C0C0C0C0C0C0C0C0C0C0C0C0C0C0C0C64
:107C60000C0C0C0C0C0C0C0C0C0C0C0C0C0C0C0C54
:107C70000C0C0C0C0C0C0C0C0C0C0C0C0C0C0C0C44
:107C800008080808080808080C0C0C0C0C0C0C0C54
:107C90000C0C0C0C0C0C0C0C0C0C0C0C0C0C0C0C24
:107CA0000C0C0C0C0C0C0C0C0C0C0C0C0C0C0C0C14
:107CB0000C0C0C0C0C0C0C0C0C0C0C0C0C0C0C0C04
:107CC00008080808080808080C0C0C0C0C0C0C0C14
:107CD0000C0C0C0C0C0C0C0C0C0C0C0C0C0C0C0CE4
:107CE0000C0C0C0C0C0C0C0C0C0C0C0C0C0C0C0CD4
:107CF0000C0C0C0C0C0C0C0C0C0C0C0C0C0C0C0CC4
:107D000008080808080808080C0C0C0C0C0C0C0CD3
:107D10000C0C0C0C0C0C0C0C0C0C0C0C0C0C0C0CA3
:107D20000C0C0C0C0C0C0C0C0C0C0C0C0C0C0C0C93
:107D30000C0C0C0C0C0C0C0C0C0C0C0C0C0C0C0C83
:107D400008080808080808080C0C0C0C0C0C0C0C93
:107D50000C0C0C0C0C0C0C0C0C0C0C0C0C0C0C0C63
:107D60000C0C0C0C0C0C0C0C0C0C0C0C0C0C0C0C53
:107D70000C0C0C0C0C0C0C0C0C0C0C0C0C0C0C0C43
:107D800008080808080808080C0C0C0C0C0C0C0C53
:107D90000C0C0C0C0C0C0C0C0C0C0C0C0C0C0C0C23
:107DA0000C0C0C0C0C0C0C0C0C0C0C0C0C0C0C0C13
:107DB0000C0C0C0C0C0C0C0C0C0C0C0C0C0C0C0C03
:107DC00008080808080808080C0C0C0C0C0C0C0C13
:107DD0000C0C0C0C0C0C0C0C0C0C0C0C0C0C0C0CE3
:107DE0000C0C0C0C0C0C0C0C0C0C0C0C0C0C0C0CD3
:107DF0000C0C0C0C0C0C0C0C0C0C0C0C0C0C0C0CC3
:107E000008080808080808080C0C0C0C0C0C0C0CD2
:107E10000C0C0C0C0C0C0C0C0C0C0C0C0C0C0C0CA2
:107E20000C0C0C0C0C0C0C0C0C0C0C0C0C0C0C0C92
:107E30000C0C0C0C0C0C0C0C0C0C0C0C0C0C0C0C82
:107E400008080808080808080C0C0C0C0C0C0C0C92
:107E50000C0C0C0C0C0C0C0C0C0C0C0C0C0C0C0C62
:107E60000C0C0C0C0C0C0C0C0C0C0C0C0C0C0C0C52
:107E70000C0C0C0C0C0C0C0C0C0C0C0C0C0C0C0C42
:107E800008080808080808080C0C0C0C0C0C0C0C52
:107E90000C0C0C0C0C0C0C0C0C0C0C0C0C0C0C0C22
:107EA0000C0C0C0C0C0C0C0C0C0C0C0C0C0C0C0C12
:107EB0000C0C0C0C0C0C0C0C0C0C0C0C0C0C0C0C02
:107EC00008080808080808080C0C0C0C0C0C0C0C12
:107ED0000C0C0C0C0C0C0C0C0C0C0C0C0C0C0C0CE2
:107EE0000C0C0C0C0C0C0C0C0C0C0C0C0C0C0C0CD2
:107EF0000C0C0C0C0C0C0C0C0C0C0C0C0C0C0C0CC2
:107F000008080808080808080C0C0C0C0C0C0C0CD1
:107F10000C0C0C0C0C0C0C0C0C0C0C0C0C0C0C0CA1
:107F20000C0C0C0C0C0C0C0C0C0C0C0C0C0C0C0C91
:107F30000C0C0C0C0C0C0C0C0C0C0C0C0C0C0C0C81
:107F400008080808080808080C0C0C0C0C0C0C0C91
:107F50000C0C0C0C0C0C0C0C0C0C0C0C0C0C0C0C61
:107F60000C0C0C0C0C0C0C0C0C0C0C0C0C0C0C0C51
:107F70000C0C0C0C0C0C0C0C0C0C0C0C0C0C0C0C41
:107F800008080808080808080C0C0C0C0C0C0C0C51
:107F90000C0C0C0C0C0C0C0C0C0C0C0C0C0C0C0C21
:107FA0000C0C0C0C0C0C0C0C0C0C0C0C0C0C0C0C11
:107FB0000C0C0C0C0C0C0C0C0C0C0C0C0C0C0C0C01
:107FC00008080808080808080C0C0C0C0C0C0C0C11
:107FD0000C0C0C0C0C0C0C0C0C0C0C0C0C0C0C0CE1
:107FE0000C0C0C0C0C0C0C0C0C0C0C0C0C0C0C0CD1
:107FF0000C0C0C0C0C0C0C0C0C0C0C0C0C0C0C0CC1
:1080000008080808080808080C0C0C0C0C0C0C0CD0
:108010000C0C0C0C0C0C0C0C0C0C0C0C0C0C0C0CA0
:108020000C0C0C0C0C0C0C0C0C0C0C0C0C0C0C0C90
:108030000C0C0C0C0C0C0C0C0C0C0C0C0C0C0C0C80
:1080400008080808080808080C0C0C0C0C0C0C0C90
:108050000C0C0C0C0C0C0C0C0C0C0C0C0C0C0C0C60
:108060000C0C0C0C0C0C0C0C0C0C0C0C0C0C0C0C50
:108070000C0C0C0C0C0C0C0C0C0C0C0C0C0C0C0C40
:1080800008080808080808080C0C0C0C0C0C0C0C50
:108090000C0C0C0C0C0C0C0C0C0C0C0C0C0C0C0C20
:1080A0000C0C0C0C0C0C0C0C0C0C0C0C0C0C0C0C10
:1080B0000C0C0C0C0C0C0C0C0C0C0C0C0C0C0C0C00
:1080C00008080808080808080C0C0C0C0C0C0C0C10
:1080D0000C0C0C0C0C0C0C0C0C0C0C0C0C0C0C0CE0
:1080E0000C0C0C0C0C0C0C0C0C0C0C0C0C0C0C0CD0
:1080F0000C0C0C0C0C0C0C0C0C0C0C0C0C0C0C0CC0
:1081000008080808080808080C0C0C0C0C0C0C0CCF
:108110000C0C0C0C0C0C0C0C0C0C0C0C0C0C0C0C9F
:108120000C0C0C0C0C0C0C0C0C0C0C0C0C0C0C0C8F
:108130000C0C0C0C0C0C0C0C0C0C0C0C0C0C0C0C7F
:1081400008080808080808080C0C0C0C0C0C0C0C8F
:108150000C0C0C0C0C0C0C0C0C0C0C0C0C0C0C0C5F
:108160000C0C0C0C0C0C0C0C0C0C0C0C0C0C0C0C4F
:108170000C0C0C0C0C0C0C0C0C0C0C0C0C0C0C0C3F
:1081800008080808080808080C0C0C0C0C0C0C0C4F
:108190000C0C0C0C0C0C0C0C0C0C0C0C0C0C0C0C1F
:1081A0000C0C0C0C0C0C0C0C0C0C0C0C0C0C0C0C0F
:1081B0000C0C0C0C0C0C0C0C0C0C0C0C0C0C0C0CFF
:1081C00008080808080808080C0C0C0C0C0C0C0C0F
:1081D0000C0C0C0C0C0C0C0C0C0C0C0C0C0C0C0CDF
:1081E0000C0C0C0C0C0C0C0C0C0C0C0C0C0C0C0CCF
:1081F0000C0C0C0C0C0C0C0C0C0C0C0C0C0C0C0CBF
:1082000008080808080808080C0C0C0C0C0C0C0CCE
:108210000C0C0C0C0C0C0C0C0C0C0C0C0C0C0C0C9E
:108220000C0C0C0C0C0C0C0C0C0C0C0C0C0C0C0C8E
:108230000C0C0C0C0C0C0C0C0C0C0C0C0C0C0C0C7E
:1082400008080808080808080C0C0C0C0C0C0C0C8E
:108250000C0C0C0C0C0C0C0C0C0C0C0C0C0C0C0C5E
:108260000C0C0C0C0C0C0C0C0C0C0C0C0C0C0C0C4E
:108270000C0C0C0C0C0C0C0C0C0C0C0C0C0C0C0C3E
:1082800008080808080808080C0C0C0C0C0C0C0C4E
:108290000C0C0C0C0C0C0C0C0C0C0C0C0C0C0C0C1E
:1082A0000C0C0C0C0C0C0C0C0C0C0C0C0C0C0C0C0E
:1082B0000C0C0C0C0C0C0C0C0C0C0C0C0C0C0C0CFE
:1082C00008080808080808080C0C0C0C0C0C0C0C0E
:1082D0000C0C0C0C0C0C0C0C0C0C0C0C0C0C0C0CDE
:1082E0000C0C0C0C0C0C0C0C0C0C0C0C0C0C0C0CCE
:1082F0000C0C0C0C0C0C0C0C0C0C0C0C0C0C0C0CBE
:1083000008080808080808080C0C0C0C0C0C0C0CCD
:108310000C0C0C0C0C0C0C0C0C0C0C0C0C0C0C0C9D
:108320000C0C0C0C0C0C0C0C0C0C0C0C0C0C0C0C8D
:108330000C0C0C0C0C0C0C0C0C0C0C0C0C0C0C0C7D
:1083400008080808080808080C0C0C0C0C0C0C0C8D
:108350000C0C0C0C0C0C0C0C0C0C0C0C0C0C0C0C5D
:108360000C0C0C0C0C0C0C0C0C0C0C0C0C0C0C0C4D
:108370000C0C0C0C0C0C0C0C0C0C0C0C0C0C0C0C3D
:1083800008080808080808080C0C0C0C0C0C0C0C4D
:108390000C0C0C0C0C0C0C0C0C0C0C0C0C0C0C0C1D
:1083A0000C0C0C0C0C0C0C0C0C0C0C0C0C0C0C0C0D
:1083B0000C0C0C0C0C0C0C0C0C0C0C0C0C0C0C0CFD
:1083C00008080808080808080C0C0C0C0C0C0C0C0D
:1083D0000C0C0C0C0C0C0C0C0C0C0C0C0C0C0C0CDD
:1083E0000C0C0C0C0C0C0C0C0C0C0C0C0C0C0C0CCD
:1083F0000C0C0C0C0C0C0C0C0C0C0C0C0C0C0C0CBD
:1084000008080808080808080C0C0C0C0C0C0C0CCC
:108410000C0C0C0C0C0C0C0C0C0C0C0C0C0C0C0C9C
:108420000C0C0C0C0C0C0C0C0C0C0C0C0C0C0C0C8C
:108430000C0C0C0C0C0C0C0C0C0C0C0C0C0C0C0C7C
:1084400008080808080808080C0C0C0C0C0C0C0C8C
:108450000C0C0C0C0C0C0C0C0C0C0C0C0C0C0C0C5C
:108460000C0C0C0C0C0C0C0C0C0C0C0C0C0C0C0C4C
:108470000C0C0C0C0C0C0C0C0C0C0C0C0C0C0C0C3C
:1084800008080808080808080C0C0C0C0C0C0C0C4C
:108490000C0C0C0C0C0C0C0C0C0C0C0C0C0C0C0C1C
:1084A0000C0C0C0C0C0C0C0C0C0C0C0C0C0C0C0C0C
:1084B0000C0C0C0C0C0C0C0C0C0C0C0C0C0C0C0CFC
:1084C00008080808080808080C0C0C0C0C0C0C0C0C
:1084D0000C0C0C0C0C0C0C0C0C0C0C0C0C0C0C0CDC
:1084E0000C0C0C0C0C0C0C0C0C0C0C0C0C0C0C0CCC
:1084F0000C0C0C0C0C0C0C0C0C0C0C0C0C0C0C0CBC
:1085000008080808080808080C0C0C0C0C0C0C0CCB
:108510000C0C0C0C0C0C0C0C0C0C0C0C0C0C0C0C9B
:108520000C0C0C0C0C0C0C0C0C0C0C0C0C0C0C0C8B
:108530000C0C0C0C0C0C0C0C0C0C0C0C0C0C0C0C7B
:1085400008080808080808080C0C0C0C0C0C0C0C8B
:108550000C0C0C0C0C0C0C0C0C0C0C0C0C0C0C0C5B
:108560000C0C0C0C0C0C0C0C0C0C0C0C0C0C0C0C4B
:108570000C0C0C0C0C0C0C0C0C0C0C0C0C0C0C0C3B
:1085800008080808080808080C0C0C0C0C0C0C0C4B
:108590000C0C0C0C0C0C0C0C0C0C0C0C0C0C0C0C1B
:1085A0000C0C0C0C0C0C0C0C0C0C0C0C0C0C0C0C0B
:1085B0000C0C0C0C0C0C0C0C0C0C0C0C0C0C0C0CFB
:1085C00008080808080808080C0C0C0C0C0C0C0C0B
:1085D0000C0C0C0C0C0C0C0C0C0C0C0C0C0C0C0CDB
:1085E0000C0C0C0C0C0C0C0C0C0C0C0C0C0C0C0CCB
:1085F0000C0C0C0C0C0C0C0C0C0C0C0C0C0C0C0CBB
:1086000008080808080808080C0C0C0C0C0C0C0CCA
:108610000C0C0C0C0C0C0C0C0C0C0C0C0C0C0C0C9A
:108620000C0C0C0C0C0C0C0C0C0C0C0C0C0C0C0C8A
:108630000C0C0C0C0C0C0C0C0C0C0C0C0C0C0C0C7A
:1086400008080808080808080C0C0C0C0C0C0C0C8A
:108650000C0C0C0C0C0C0C0C0C0C0C0C0C0C0C0C5A
:108660000C0C0C0C0C0C0C0C0C0C0C0C0C0C0C0C4A
:108670000C0C0C0C0C0C0C0C0C0C0C0C0C0C0C0C3A
:1086800008080808080808080C0C0C0C0C0C0C0C4A
:108690000C0C0C0C0C0C0C0C0C0C0C0C0C0C0C0C1A
:1086A0000C0C0C0C0C0C0C0C0C0C0C0C0C0C0C0C0A
:1086B0000C0C0C0C0C0C0C0C0C0C0C0C0C0C0C0CFA
:1086C00008080808080808080C0C0C0C0C0C0C0C0A
:1086D0000C0C0C0C0C0C0C0C0C0C0C0C0C0C0C0CDA
:1086E0000C0C0C0C0C0C0C0C0C0C0C0C0C0C0C0CCA
:1086F0000C0C0C0C0C0C0C0C0C0C0C0C0C0C0C0CBA
:1087000008080808080808080C0C0C0C0C0C0C0CC9
:108710000C0C0C0C0C0C0C0C0C0C0C0C0C0C0C0C99
:108720000C0C0C0C0C0C0C0C0C0C0C0C0C0C0C0C89
:108730000C0C0C0C0C0C0C0C0C0C0C0C0C0C0C0C79
:1087400008080808080808080C0C0C0C0C0C0C0C89
:108750000C0C0C0C0C0C0C0C0C0C0C0C0C0C0C0C59
:108760000C0C0C0C0C0C0C0C0C0C0C0C0C0C0C0C49
:108770000C0C0C0C0C0C0C0C0C0C0C0C0C0C0C0C39
:1087800008080808080808080C0C0C0C0C0C0C0C49
:108790000C0C0C0C0C0C0C0C0C0C0C0C0C0C0C0C19
:1087A0000C0C0C0C0C0C0C0C0C0C0C0C0C0C0C0C09
:1087B0000C0C0C0C0C0C0C0C0C0C0C0C0C0C0C0CF9
:1087C00008080808080808080C0C0C0C0C0C0C0C09
:1087D0000C0C0C0C0C0C0C0C0C0C0C0C0C0C0C0CD9
:1087E0000C0C0C0C0C0C0C0C0C0C0C0C0C0C0C0CC9
:1087F0000C0C0C0C0C0C0C0C0C0C0C0C0C0C0C0CB9
:1088000008080808080808080C0C0C0C0C0C0C0CC8
:108810000C0C0C0C0C0C0C0C0C0C0C0C0C0C0C0C98
:108820000C0C0C0C0C0C0C0C0C0C0C0C0C0C0C0C88
:108830000C0C0C0C0C0C0C0C0C0C0C0C0C0C0C0C78
:1088400008080808080808080C0C0C0C0C0C0C0C88
:108850000C0C0C0C0C0C0C0C0C0C0C0C0C0C0C0C58
:108860000C0C0C0C0C0C0C0C0C0C0C0C0C0C0C0C48
:108870000C0C0C0C0C0C0C0C0C0C0C0C0C0C0C0C38
:1088800008080808080808080C0C0C0C0C0C0C0C48
:108890000C0C0C0C0C0C0C0C0C0C0C0C0C0C0C0C18
:1088A0000C0C0C0C0C0C0C0C0C0C0C0C0C0C0C0C08
:1088B0000C0C0C0C0C0C0C0C0C0C0C0C0C0C0C0CF8
:1088C00008080808080808080C0C0C0C0C0C0C0C08
:1088D0000C0C0C0C0C0C0C0C0C0C0C0C0C0C0C0CD8
:1088E0000C0C0C0C0C0C0C0C0C0C0C0C0C0C0C0CC8
:1088F0000C0C0C0C0C0C0C0C0C0C0C0C0C0C0C0CB8
:1089000008080808080808080C0C0C0C0C0C0C0CC7
:108910000C0C0C0C0C0C0C0C0C0C0C0C0C0C0C0C97
:108920000C0C0C0C0C0C0C0C0C0C0C0C0C0C0C0C87
:108930000C0C0C0C0C0C0C0C0C0C0C0C0C0C0C0C77
:1089400008080808080808080C0C0C0C0C0C0C0C87
:108950000C0C0C0C0C0C0C0C0C0C0C0C0C0C0C0C57
:108960000C0C0C0C0C0C0C0C0C0C0C0C0C0C0C0C47
:108970000C0C0C0C0C0C0C0C0C0C0C0C0C0C0C0C37
:1089800008080808080808080C0C0C0C0C0C0C0C47
:108990000C0C0C0C0C0C0C0C0C0C0C0C0C0C0C0C17
:1089A0000C0C0C0C0C0C0C0C0C0C0C0C0C0C0C0C07
:1089B0000C0C0C0C0C0C0C0C0C0C0C0C0C0C0C0CF7
:1089C00008080808080808080C0C0C0C0C0C0C0C07
:1089D0000C0C0C0C0C0C0C0C0C0C0C0C0C0C0C0CD7
:1089E0000C0C0C0C0C0C0C0C0C0C0C0C0C0C0C0CC7
:1089F0000C0C0C0C0C0C0C0C0C0C0C0C0C0C0C0CB7
:108A000008080808080808080C0C0C0C0C0C0C0CC6
:108A10000C0C0C0C0C0C0C0C0C0C0C0C0C0C0C0C96
:108A20000C0C0C0C0C0C0C0C0C0C0C0C0C0C0C0C86
:108A30000C0C0C0C0C0C0C0C0C0C0C0C0C0C0C0C76
:108A400008080808080808080C0C0C0C0C0C0C0C86
:108A50000C0C0C0C0C0C0C0C0C0C0C0C0C0C0C0C56
:108A60000C0C0C0C0C0C0C0C0C0C0C0C0C0C0C0C46
:108A70000C0C0C0C0C0C0C0C0C0C0C0C0C0C0C0C36
:108A800008080808080808080C0C0C0C0C0C0C0C46
:108A90000C0C0C0C0C0C0C0C0C0C0C0C0C0C0C0C16
:108AA0000C0C0C0C0C0C0C0C0C0C0C0C0C0C0C0C06
:108AB0000C0C0C0C0C0C0C0C0C0C0C0C0C0C0C0CF6
:108AC00008080808080808080C0C0C0C0C0C0C0C06
:108AD0000C0C0C0C0C0C0C0C0C0C0C0C0C0C0C0CD6
:108AE0000C0C0C0C0C0C0C0C0C0C0C0C0C0C0C0CC6
:108AF0000C0C0C0C0C0C0C0C0C0C0C0C0C0C0C0CB6
:108B000008080808080808080C0C0C0C0C0C0C0CC5
:108B10000C0C0C0C0C0C0C0C0C0C0C0C0C0C0C0C95
:108B20000C0C0C0C0C0C0C0C0C0C0C0C0C0C0C0C85
:108B30000C0C0C0C0C0C0C0C0C0C0C0C0C0C0C0C75
:108B400008080808080808080C0C0C0C0C0C0C0C85
:108B50000C0C0C0C0C0C0C0C0C0C0C0C0C0C0C0C55
:108B60000C0C0C0C0C0C0C0C0C0C0C0C0C0C0C0C45
:108B70000C0C0C0C0C0C0C0C0C0C0C0C0C0C0C0C35
:108B800008080808080808080C0C0C0C0C0C0C0C45
:108B90000C0C0C0C0C0C0C0C0C0C0C0C0C0C0C0C15
:108BA0000C0C0C0C0C0C0C0C0C0C0C0C0C0C0C0C05
:108BB0000C0C0C0C0C0C0C0C0C0C0C0C0C0C0C0CF5
:108BC00008080808080808080C0C0C0C0C0C0C0C05
:108BD0000C0C0C0C0C0C0C0C0C0C0C0C0C0C0C0CD5
:108BE0000C0C0C0C0C0C0C0C0C0C0C0C0C0C0C0CC5
:108BF0000C0C0C0C0C0C0C0C0C0C0C0C0C0C0C0CB5
:108C000008080808080808080C0C0C0C0C0C0C0CC4
:108C10000C0C0C0C0C0C0C0C0C0C0C0C0C0C0C0C94
:108C20000C0C0C0C0C0C0C0C0C0C0C0C0C0C0C0C84
:108C30000C0C0C0C0C0C0C0C0C0C0C0C0C0C0C0C74
:108C400008080808080808080C0C0C0C0C0C0C0C84
:108C50000C0C0C0C0C0C0C0C0C0C0C0C0C0C0C0C54
:108C60000C0C0C0C0C0C0C0C0C0C0C0C0C0C0C0C44
:108C70000C0C0C0C0C0C0C0C0C0C0C0C0C0C0C0C34
:108C800008080808080808080C0C0C0C0C0C0C0C44
:108C90000C0C0C0C0C0C0C0C0C0C0C0C0C0C0C0C14
:108CA0000C0C0C0C0C0C0C0C0C0C0C0C0C0C0C0C04
:108CB0000C0C0C0C0C0C0C0C0C0C0C0C0C0C0C0CF4
:108CC00008080808080808080C0C0C0C0C0C0C0C04
:108CD0000C0C0C0C0C0C0C0C0C0C0C0C0C0C0C0CD4
:108CE0000C0C0C0C0C0C0C0C0C0C0C0C0C0C0C0CC4
:108CF0000C0C0C0C0C0C0C0C0C0C0C0C0C0C0C0CB4
:108D000008080808080808080C0C0C0C0C0C0C0CC3
:108D10000C0C0C0C0C0C0C0C0C0C0C0C0C0C0C0C93
:108D20000C0C0C0C0C0C0C0C0C0C0C0C0C0C0C0C83
:108D30000C0C0C0C0C0C0C0C0C0C0C0C0C0C0C0C73
:108D400008080808080808080C0C0C0C0C0C0C0C83
:108D50000C0C0C0C0C0C0C0C0C0C0C0C0C0C0C0C53
:108D60000C0C0C0C0C0C0C0C0C0C0C0C0C0C0C0C43
:108D70000C0C0C0C0C0C0C0C0C0C0C0C0C0C0C0C33
:108D800008080808080808080C0C0C0C0C0C0C0C43
:108D90000C0C0C0C0C0C0C0C0C0C0C0C0C0C0C0C13
:108DA0000C0C0C0C0C0C0C0C0C0C0C0C0C0C0C0C03
:108DB0000C0C0C0C0C0C0C0C0C0C0C0C0C0C0C0CF3
:108DC00008080808080808080C0C0C0C0C0C0C0C03
:108DD0000C0C0C0C0C0C0C0C0C0C0C0C0C0C0C0CD3
:108DE0000C0C0C0C0C0C0C0C0C0C0C0C0C0C0C0CC3
:108DF0000C0C0C0C0C0C0C0C0C0C0C0C0C0C0C0CB3
:108E000008080808080808080C0C0C0C0C0C0C0CC2
:108E10000C0C0C0C0C0C0C0C0C0C0C0C0C0C0C0C92
:108E20000C0C0C0C0C0C0C0C0C0C0C0C0C0C0C0C82
:108E30000C0C0C0C0C0C0C0C0C0C0C0C0C0C0C0C72
:108E400008080808080808080C0C0C0C0C0C0C0C82
:108E50000C0C0C0C0C0C0C0C0C0C0C0C0C0C0C0C52
:108E60000C0C0C0C0C0C0C0C0C0C0C0C0C0C0C0C42
:108E70000C0C0C0C0C0C0C0C0C0C0C0C0C0C0C0C32
:108E800008080808080808080C0C0C0C0C0C0C0C42
:108E90000C0C0C0C0C0C0C0C0C0C0C0C0C0C0C0C12
:108EA0000C0C0C0C0C0C0C0C0C0C0C0C0C0C0C0C02
:108EB0000C0C0C0C0C0C0C0C0C0C0C0C0C0C0C0CF2
:108EC00008080808080808080C0C0C0C0C0C0C0C02
:108ED0000C0C0C0C0C0C0C0C0C0C0C0C0C0C0C0CD2
:108EE0000C0C0C0C0C0C0C0C0C0C0C0C0C0C0C0CC2
:108EF0000C0C0C0C0C0C0C0C0C0C0C0C0C0C0C0CB2
:108F000008080808080808080C0C0C0C0C0C0C0CC1
:108F10000C0C0C0C0C0C0C0C0C0C0C0C0C0C0C0C91
:108F20000C0C0C0C0C0C0C0C0C0C0C0C0C0C0C0C81
:108F30000C0C0C0C0C0C0C0C0C0C0C0C0C0C0C0C71
:108F400008080808080808080C0C0C0C0C0C0C0C81
:108F50000C0C0C0C0C0C0C0C0C0C0C0C0C0C0C0C51
:108F60000C0C0C0C0C0C0C0C0C0C0C0C0C0C0C0C41
:108F70000C0C0C0C0C0C0C0C0C0C0C0C0C0C0C0C31
:108F800008080808080808080C0C0C0C0C0C0C0C41
:108F90000C0C0C0C0C0C0C0C0C0C0C0C0C0C0C0C11
:108FA0000C0C0C0C0C0C0C0C0C0C0C0C0C0C0C0C01
:108FB0000C0C0C0C0C0C0C0C0C0C0C0C0C0C0C0CF1
:108FC00008080808080808080C0C0C0C0C0C0C0C01
:108FD0000C0C0C0C0C0C0C0C0C0C0C0C0C0C0C0CD1
:108FE0000C0C0C0C0C0C0C0C0C0C0C0C0C0C0C0CC1
:108FF0000C0C0C0C0C0C0C0C0C0C0C0C0C0C0C0CB1
:1090000008080808080808080C0C0C0C0C0C0C0CC0
:109010000C0C0C0C0C0C0C0C0C0C0C0C0C0C0C0C90
:109020000C0C0C0C0C0C0C0C0C0C0C0C0C0C0C0C80
:109030000C0C0C0C0C0C0C0C0C0C0C0C0C0C0C0C70
:1090400008080808080808080C0C0C0C0C0C0C0C80
:109050000C0C0C0C0C0C0C0C0C0C0C0C0C0C0C0C50
:109060000C0C0C0C0C0C0C0C0C0C0C0C0C0C0C0C40
:109070000C0C0C0C0C0C0C0C0C0C0C0C0C0C0C0C30
:1090800008080808080808080C0C0C0C0C0C0C0C40
:109090000C0C0C0C0C0C0C0C0C0C0C0C0C0C0C0C10
:1090A0000C0C0C0C0C0C0C0C0C0C0C0C0C0C0C0C00
:1090B0000C0C0C0C0C0C0C0C0C0C0C0C0C0C0C0CF0
:1090C00008080808080808080C0C0C0C0C0C0C0C00
:1090D0000C0C0C0C0C0C0C0C0C0C0C0C0C0C0C0CD0
:1090E0000C0C0C0C0C0C0C0C0C0C0C0C0C0C0C0CC0
:1090F0000C0C0C0C0C0C0C0C0C0C0C0C0C0C0C0CB0
:1091000008080808080808080C0C0C0C0C0C0C0CBF
:109110000C0C0C0C0C0C0C0C0C0C0C0C0C0C0C0C8F
:109120000C0C0C0C0C0C0C0C0C0C0C0C0C0C0C0C7F
:109130000C0C0C0C0C0C0C0C0C0C0C0C0C0C0C0C6F
:1091400008080808080808080C0C0C0C0C0C0C0C7F
:109150000C0C0C0C0C0C0C0C0C0C0C0C0C0C0C0C4F
:109160000C0C0C0C0C0C0C0C0C0C0C0C0C0C0C0C3F
:109170000C0C0C0C0C0C0C0C0C0C0C0C0C0C0C0C2F
:1091800008080808080808080C0C0C0C0C0C0C0C3F
:109190000C0C0C0C0C0C0C0C0C0C0C0C0C0C0C0C0F
:1091A0000C0C0C0C0C0C0C0C0C0C0C0C0C0C0C0CFF
:1091B0000C0C0C0C0C0C0C0C0C0C0C0C0C0C0C0CEF
:1091C00008080808080808080C0C0C0C0C0C0C0CFF
:1091D0000C0C0C0C0C0C0C0C0C0C0C0C0C0C0C0CCF
:1091E0000C0C0C0C0C0C0C0C0C0C0C0C0C0C0C0CBF
:1091F0000C0C0C0C0C0C0C0C0C0C0C0C0C0C0C0CAF
:1092000008080808080808080C0C0C0C0C0C0C0CBE
:109210000C0C0C0C0C0C0C0C0C0C0C0C0C0C0C0C8E
:109220000C0C0C0C0C0C0C0C0C0C0C0C0C0C0C0C7E
:109230000C0C0C0C0C0C0C0C0C0C0C0C0C0C0C0C6E
:1092400008080808080808080C0C0C0C0C0C0C0C7E
:109250000C0C0C0C0C0C0C0C0C0C0C0C0C0C0C0C4E
:109260000C0C0C0C0C0C0C0C0C0C0C0C0C0C0C0C3E
:109270000C0C0C0C0C0C0C0C0C0C0C0C0C0C0C0C2E
:1092800008080808080808080C0C0C0C0C0C0C0C3E
:109290000C0C0C0C0C0C0C0C0C0C0C0C0C0C0C0C0E
:1092A0000C0C0C0C0C0C0C0C0C0C0C0C0C0C0C0CFE
:1092B0000C0C0C0C0C0C0C0C0C0C0C0C0C0C0C0CEE
:1092C00008080808080808080C0C0C0C0C0C0C0CFE
:1092D0000C0C0C0C0C0C0C0C0C0C0C0C0C0C0C0CCE
:1092E0000C0C0C0C0C0C0C0C0C0C0C0C0C0C0C0CBE
:1092F0000C0C0C0C0C0C0C0C0C0C0C0C0C0C0C0CAE
:1093000008080808080808080C0C0C0C0C0C0C0CBD
:109310000C0C0C0C0C0C0C0C0C0C0C0C0C0C0C0C8D
:109320000C0C0C0C0C0C0C0C0C0C0C0C0C0C0C0C7D
:109330000C0C0C0C0C0C0C0C0C0C0C0C0C0C0C0C6D
:1093400008080808080808080C0C0C0C0C0C0C0C7D
:109350000C0C0C0C0C0C0C0C0C0C0C0C0C0C0C0C4D
:109360000C0C0C0C0C0C0C0C0C0C0C0C0C0C0C0C3D
:109370000C0C0C0C0C0C0C0C0C0C0C0C0C0C0C0C2D
:1093800008080808080808080C0C0C0C0C0C0C0C3D
:109390000C0C0C0C0C0C0C0C0C0C0C0C0C0C0C0C0D
:1093A0000C0C0C0C0C0C0C0C0C0C0C0C0C0C0C0CFD
:1093B0000C0C0C0C0C0C0C0C0C0C0C0C0C0C0C0CED
:1093C00008080808080808080C0C0C0C0C0C0C0CFD
:1093D0000C0C0C0C0C0C0C0C0C0C0C0C0C0C0C0CCD
:1093E0000C0C0C0C0C0C0C0C0C0C0C0C0C0C0C0CBD
:1093F0000C0C0C0C0C0C0C0C0C0C0C0C0C0C0C0CAD
:1094000008080808080808080C0C0C0C0C0C0C0CBC
:109410000C0C0C0C0C0C0C0C0C0C0C0C0C0C0C0C8C
:109420000C0C0C0C0C0C0C0C0C0C0C0C0C0C0C0C7C
:109430000C0C0C0C0C0C0C0C0C0C0C0C0C0C0C0C6C
:1094400008080808080808080C0C0C0C0C0C0C0C7C
:109450000C0C0C0C0C0C0C0C0C0C0C0C0C0C0C0C4C
:109460000C0C0C0C0C0C0C0C0C0C0C0C0C0C0C0C3C
:109470000C0C0C0C0C0C0C0C0C0C0C0C0C0C0C0C2C
:1094800008080808080808080C0C0C0C0C0C0C0C3C
:109490000C0C0C0C0C0C0C0C0C0C0C0C0C0C0C0C0C
:1094A0000C0C0C0C0C0C0C0C0C0C0C0C0C0C0C0CFC
:1094B0000C0C0C0C0C0C0C0C0C0C0C0C0C0C0C0CEC
:1094C00008080808080808080C0C0C0C0C0C0C0CFC
:1094D0000C0C0C0C0C0C0C0C0C0C0C0C0C0C0C0CCC
:1094E0000C0C0C0C0C0C0C0C0C0C0C0C0C0C0C0CBC
:1094F0000C0C0C0C0C0C0C0C0C0C0C0C0C0C0C0CAC
:1095000008080808080808080C0C0C0C0C0C0C0CBB
:109510000C0C0C0C0C0C0C0C0C0C0C0C0C0C0C0C8B
:109520000C0C0C0C0C0C0C0C0C0C0C0C0C0C0C0C7B
:109530000C0C0C0C0C0C0C0C0C0C0C0C0C0C0C0C6B
:1095400008080808080808080C0C0C0C0C0C0C0C7B
:109550000C0C0C0C0C0C0C0C0C0C0C0C0C0C0C0C4B
:109560000C0C0C0C0C0C0C0C0C0C0C0C0C0C0C0C3B
:109570000C0C0C0C0C0C0C0C0C0C0C0C0C0C0C0C2B
:1095800008080808080808080C0C0C0C0C0C0C0C3B
:109590000C0C0C0C0C0C0C0C0C0C0C0C0C0C0C0C0B
:1095A0000C0C0C0C0C0C0C0C0C0C0C0C0C0C0C0CFB
:1095B0000C0C0C0C0C0C0C0C0C0C0C0C0C0C0C0CEB
:1095C00008080808080808080C0C0C0C0C0C0C0CFB
:1095D0000C0C0C0C0C0C0C0C0C0C0C0C0C0C0C0CCB
:1095E0000C0C0C0C0C0C0C0C0C0C0C0C0C0C0C0CBB
:1095F0000C0C0C0C0C0C0C0C0C0C0C0C0C0C0C0CAB
:1096000008080808080808080C0C0C0C0C0C0C0CBA
:109610000C0C0C0C0C0C0C0C0C0C0C0C0C0C0C0C8A
:109620000C0C0C0C0C0C0C0C0C0C0C0C0C0C0C0C7A
:109630000C0C0C0C0C0C0C0C0C0C0C0C0C0C0C0C6A
:1096400008080808080808080C0C0C0C0C0C0C0C7A
:109650000C0C0C0C0C0C0C0C0C0C0C0C0C0C0C0C4A
:109660000C0C0C0C0C0C0C0C0C0C0C0C0C0C0C0C3A
:109670000C0C0C0C0C0C0C0C0C0C0C0C0C0C0C0C2A
:1096800008080808080808080C0C0C0C0C0C0C0C3A
:109690000C0C0C0C0C0C0C0C0C0C0C0C0C0C0C0C0A
:1096A0000C0C0C0C0C0C0C0C0C0C0C0C0C0C0C0CFA
:1096B0000C0C0C0C0C0C0C0C0C0C0C0C0C0C0C0CEA
:1096C00008080808080808080C0C0C0C0C0C0C0CFA
:1096D0000C0C0C0C0C0C0C0C0C0C0C0C0C0C0C0CCA
:1096E0000C0C0C0C0C0C0C0C0C0C0C0C0C0C0C0CBA
:1096F0000C0C0C0C0C0C0C0C0C0C0C0C0C0C0C0CAA
:1097000008080808080808080C0C0C0C0C0C0C0CB9
:109710000C0C0C0C0C0C0C0C0C0C0C0C0C0C0C0C89
:109720000C0C0C0C0C0C0C0C0C0C0C0C0C0C0C0C79
:109730000C0C0C0C0C0C0C0C0C0C0C0C0C0C0C0C69
:1097400008080808080808080C0C0C0C0C0C0C0C79
:109750000C0C0C0C0C0C0C0C0C0C0C0C0C0C0C0C49
:109760000C0C0C0C0C0C0C0C0C0C0C0C0C0C0C0C39
:109770000C0C0C0C0C0C0C0C0C0C0C0C0C0C0C0C29
:1097800008080808080808080C0C0C0C0C0C0C0C39
:109790000C0C0C0C0C0C0C0C0C0C0C0C0C0C0C0C09
:1097A0000C0C0C0C0C0C0C0C0C0C0C0C0C0C0C0CF9
:1097B0000C0C0C0C0C0C0C0C0C0C0C0C0C0C0C0CE9
:1097C00008080808080808080C0C0C0C0C0C0C0CF9
:1097D0000C0C0C0C0C0C0C0C0C0C0C0C0C0C0C0CC9
:1097E0000C0C0C0C0C0C0C0C0C0C0C0C0C0C0C0CB9
:1097F0000C0C0C0C0C0C0C0C0C0C0C0C0C0C0C0CA9
:1098000008080808080808080C0C0C0C0C0C0C0CB8
:109810000C0C0C0C0C0C0C0C0C0C0C0C0C0C0C0C88
:109820000C0C0C0C0C0C0C0C0C0C0C0C0C0C0C0C78
:109830000C0C0C0C0C0C0C0C0C0C0C0C0C0C0C0C68
:1098400008080808080808080C0C0C0C0C0C0C0C78
:109850000C0C0C0C0C0C0C0C0C0C0C0C0C0C0C0C48
:109860000C0C0C0C0C0C0C0C0C0C0C0C0C0C0C0C38
:109870000C0C0C0C0C0C0C0C0C0C0C0C0C0C0C0C28
:1098800008080808080808080C0C0C0C0C0C0C0C38
:109890000C0C0C0C0C0C0C0C0C0C0C0C0C0C0C0C08
:1098A0000C0C0C0C0C0C0C0C0C0C0C0C0C0C0C0CF8
:1098B0000C0C0C0C0C0C0C0C0C0C0C0C0C0C0C0CE8
:1098C00008080808080808080C0C0C0C0C0C0C0CF8
:1098D0000C0C0C0C0C0C0C0C0C0C0C0C0C0C0C0CC8
:1098E0000C0C0C0C0C0C0C0C0C0C0C0C0C0C0C0CB8
:1098F0000C0C0C0C0C0C0C0C0C0C0C0C0C0C0C0CA8
:1099000008080808080808080C0C0C0C0C0C0C0CB7
:109910000C0C0C0C0C0C0C0C0C0C0C0C0C0C0C0C87
:109920000C0C0C0C0C0C0C0C0C0C0C0C0C0C0C0C77
:109930000C0C0C0C0C0C0C0C0C0C0C0C0C0C0C0C67
:1099400008080808080808080C0C0C0C0C0C0C0C77
:109950000C0C0C0C0C0C0C0C0C0C0C0C0C0C0C0C47
:109960000C0C0C0C0C0C0C0C0C0C0C0C0C0C0C0C37
:109970000C0C0C0C0C0C0C0C0C0C0C0C0C0C0C0C27
:1099800008080808080808080C0C0C0C0C0C0C0C37
:109990000C0C0C0C0C0C0C0C0C0C0C0C0C0C0C0C07
:1099A0000C0C0C0C0C0C0C0C0C0C0C0C0C0C0C0CF7
:1099B0000C0C0C0C0C0C0C0C0C0C0C0C0C0C0C0CE7
:1099C00008080808080808080C0C0C0C0C0C0C0CF7
:1099D0000C0C0C0C0C0C0C0C0C0C0C0C0C0C0C0CC7
:1099E0000C0C0C0C0C0C0C0C0C0C0C0C0C0C0C0CB7
:1099F0000C0C0C0C0C0C0C0C0C0C0C0C0C0C0C0CA7
:109A000008080808080808080C0C0C0C0C0C0C0CB6
:109A10000C0C0C0C0C0C0C0C0C0C0C0C0C0C0C0C86
:109A20000C0C0C0C0C0C0C0C0C0C0C0C0C0C0C0C76
:109A30000C0C0C0C0C0C0C0C0C0C0C0C0C0C0C0C66
:109A400008080808080808080C0C0C0C0C0C0C0C76
:109A50000C0C0C0C0C0C0C0C0C0C0C0C0C0C0C0C46
:109A60000C0C0C0C0C0C0C0C0C0C0C0C0C0C0C0C36
:109A70000C0C0C0C0C0C0C0C0C0C0C0C0C0C0C0C26
:109A800008080808080808080C0C0C0C0C0C0C0C36
:109A90000C0C0C0C0C0C0C0C0C0C0C0C0C0C0C0C06
:109AA0000C0C0C0C0C0C0C0C0C0C0C0C0C0C0C0CF6
:109AB0000C0C0C0C0C0C0C0C0C0C0C0C0C0C0C0CE6
:109AC00008080808080808080C0C0C0C0C0C0C0CF6
:109AD0000C0C0C0C0C0C0C0C0C0C0C0C0C0C0C0CC6
:109AE0000C0C0C0C0C0C0C0C0C0C0C0C0C0C0C0CB6
:109AF0000C0C0C0C0C0C0C0C0C0C0C0C0C0C0C0CA6
:109B000008080808080808080C0C0C0C0C0C0C0CB5
:109B10000C0C0C0C0C0C0C0C0C0C0C0C0C0C0C0C85
:109B20000C0C0C0C0C0C0C0C0C0C0C0C0C0C0C0C75
:109B30000C0C0C0C0C0C0C0C0C0C0C0C0C0C0C0C65
:109B400008080808080808080C0C0C0C0C0C0C0C75
:109B50000C0C0C0C0C0C0C0C0C0C0C0C0C0C0C0C45
:109B60000C0C0C0C0C0C0C0C0C0C0C0C0C0C0C0C35
:109B70000C0C0C0C0C0C0C0C0C0C0C0C0C0C0C0C25
:109B800008080808080808080C0C0C0C0C0C0C0C35
:109B90000C0C0C0C0C0C0C0C0C0C0C0C0C0C0C0C05
:109BA0000C0C0C0C0C0C0C0C0C0C0C0C0C0C0C0CF5
:109BB0000C0C0C0C0C0C0C0C0C0C0C0C0C0C0C0CE5
:109BC00008080808080808080C0C0C0C0C0C0C0CF5
:109BD0000C0C0C0C0C0C0C0C0C0C0C0C0C0C0C0CC5
:109BE0000C0C0C0C0C0C0C0C0C0C0C0C0C0C0C0CB5
:109BF0000C0C0C0C0C0C0C0C0C0C0C0C0C0C0C0CA5
:109C000008080808080808080C0C0C0C0C0C0C0CB4
:109C10000C0C0C0C0C0C0C0C0C0C0C0C0C0C0C0C84
:109C20000C0C0C0C0C0C0C0C0C0C0C0C0C0C0C0C74
:109C30000C0C0C0C0C0C0C0C0C0C0C0C0C0C0C0C64
:109C400008080808080808080C0C0C0C0C0C0C0C74
:109C50000C0C0C0C0C0C0C0C0C0C0C0C0C0C0C0C44
:109C60000C0C0C0C0C0C0C0C0C0C0C0C0C0C0C0C34
:109C70000C0C0C0C0C0C0C0C0C0C0C0C0C0C0C0C24
:109C800008080808080808080C0C0C0C0C0C0C0C34
:109C90000C0C0C0C0C0C0C0C0C0C0C0C0C0C0C0C04
:109CA0000C0C0C0C0C0C0C0C0C0C0C0C0C0C0C0CF4
:109CB0000C0C0C0C0C0C0C0C0C0C0C0C0C0C0C0CE4
:109CC00008080808080808080C0C0C0C0C0C0C0CF4
:109CD0000C0C0C0C0C0C0C0C0C0C0C0C0C0C0C0CC4
:109CE0000C0C0C0C0C0C0C0C0C0C0C0C0C0C0C0CB4
:109CF0000C0C0C0C0C0C0C0C0C0C0C0C0C0C0C0CA4
:109D000008080808080808080C0C0C0C0C0C0C0CB3
:109D10000C0C0C0C0C0C0C0C0C0C0C0C0C0C0C0C83
:109D20000C0C0C0C0C0C0C0C0C0C0C0C0C0C0C0C73
:109D30000C0C0C0C0C0C0C0C0C0C0C0C0C0C0C0C63
:109D400008080808080808080C0C0C0C0C0C0C0C73
:109D50000C0C0C0C0C0C0C0C0C0C0C0C0C0C0C0C43
:109D60000C0C0C0C0C0C0C0C0C0C0C0C0C0C0C0C33
:109D70000C0C0C0C0C0C0C0C0C0C0C0C0C0C0C0C23
:109D800008080808080808080C0C0C0C0C0C0C0C33
:109D90000C0C0C0C0C0C0C0C0C0C0C0C0C0C0C0C03
:109DA0000C0C0C0C0C0C0C0C0C0C0C0C0C0C0C0CF3
:109DB0000C0C0C0C0C0C0C0C0C0C0C0C0C0C0C0CE3
:109DC00008080808080808080C0C0C0C0C0C0C0CF3
:109DD0000C0C0C0C0C0C0C0C0C0C0C0C0C0C0C0CC3
:109DE0000C0C0C0C0C0C0C0C0C0C0C0C0C0C0C0CB3
:109DF0000C0C0C0C0C0C0C0C0C0C0C0C0C0C0C0CA3
:109E000008080808080808080C0C0C0C0C0C0C0CB2
:109E10000C0C0C0C0C0C0C0C0C0C0C0C0C0C0C0C82
:109E20000C0C0C0C0C0C0C0C0C0C0C0C0C0C0C0C72
:109E30000C0C0C0C0C0C0C0C0C0C0C0C0C0C0C0C62
:109E400008080808080808080C0C0C0C0C0C0C0C72
:109E50000C0C0C0C0C0C0C0C0C0C0C0C0C0C0C0C42
:109E60000C0C0C0C0C0C0C0C0C0C0C0C0C0C0C0C32
:109E70000C0C0C0C0C0C0C0C0C0C0C0C0C0C0C0C22
:109E800008080808080808080C0C0C0C0C0C0C0C32
:109E90000C0C0C0C0C0C0C0C0C0C0C0C0C0C0C0C02
:109EA0000C0C0C0C0C0C0C0C0C0C0C0C0C0C0C0CF2
:109EB0000C0C0C0C0C0C0C0C0C0C0C0C0C0C0C0CE2
:109EC00008080808080808080C0C0C0C0C0C0C0CF2
:109ED0000C0C0C0C0C0C0C0C0C0C0C0C0C0C0C0CC2
:109EE0000C0C0C0C0C0C0C0C0C0C0C0C0C0C0C0CB2
:109EF0000C0C0C0C0C0C0C0C0C0C0C0C0C0C0C0CA2
:109F000008080808080808080C0C0C0C0C0C0C0CB1
:109F10000C0C0C0C0C0C0C0C0C0C0C0C0C0C0C0C81
:109F20000C0C0C0C0C0C0C0C0C0C0C0C0C0C0C0C71
:109F30000C0C0C0C0C0C0C0C0C0C0C0C0C0C0C0C61
:109F400008080808080808080C0C0C0C0C0C0C0C71
:109F50000C0C0C0C0C0C0C0C0C0C0C0C0C0C0C0C41
:109F60000C0C0C0C0C0C0C0C0C0C0C0C0C0C0C0C31
:109F70000C0C0C0C0C0C0C0C0C0C0C0C0C0C0C0C21
:109F800008080808080808080C0C0C0C0C0C0C0C31
:109F90000C0C0C0C0C0C0C0C0C0C0C0C0C0C0C0C01
:109FA0000C0C0C0C0C0C0C0C0C0C0C0C0C0C0C0CF1
:109FB0000C0C0C0C0C0C0C0C0C0C0C0C0C0C0C0CE1
:109FC00008080808080808080C0C0C0C0C0C0C0CF1
:109FD0000C0C0C0C0C0C0C0C0C0C0C0C0C0C0C0CC1
:109FE0000C0C0C0C0C0C0C0C0C0C0C0C0C0C0C0CB1
:109FF0000C0C0C0C0C0C0C0C0C0C0C0C0C0C0C0CA1
:10A0000008080808080808080C0C0C0C0C0C0C0CB0
:10A010000C0C0C0C0C0C0C0C0C0C0C0C0C0C0C0C80
:10A020000C0C0C0C0C0C0C0C0C0C0C0C0C0C0C0C70
:10A030000C0C0C0C0C0C0C0C0C0C0C0C0C0C0C0C60
:10A0400008080808080808080C0C0C0C0C0C0C0C70
:10A050000C0C0C0C0C0C0C0C0C0C0C0C0C0C0C0C40
:10A060000C0C0C0C0C0C0C0C0C0C0C0C0C0C0C0C30
:10A070000C0C0C0C0C0C0C0C0C0C0C0C0C0C0C0C20
:10A0800008080808080808080C0C0C0C0C0C0C0C30
:10A090000C0C0C0C0C0C0C0C0C0C0C0C0C0C0C0C00
:10A0A0000C0C0C0C0C0C0C0C0C0C0C0C0C0C0C0CF0
:10A0B0000C0C0C0C0C0C0C0C0C0C0C0C0C0C0C0CE0
:10A0C00008080808080808080C0C0C0C0C0C0C0CF0
:10A0D0000C0C0C0C0C0C0C0C0C0C0C0C0C0C0C0CC0
:10A0E0000C0C0C0C0C0C0C0C0C0C0C0C0C0C0C0CB0
:10A0F0000C0C0C0C0C0C0C0C0C0C0C0C0C0C0C0CA0
:10A1000008080808080808080C0C0C0C0C0C0C0CAF
:10A110000C0C0C0C0C0C0C0C0C0C0C0C0C0C0C0C7F
:10A120000C0C0C0C0C0C0C0C0C0C0C0C0C0C0C0C6F
:10A130000C0C0C0C0C0C0C0C0C0C0C0C0C0C0C0C5F
:10A1400008080808080808080C0C0C0C0C0C0C0C6F
:10A150000C0C0C0C0C0C0C0C0C0C0C0C0C0C0C0C3F
:10A160000C0C0C0C0C0C0C0C0C0C0C0C0C0C0C0C2F
:10A170000C0C0C0C0C0C0C0C0C0C0C0C0C0C0C0C1F
:10A1800008080808080808080C0C0C0C0C0C0C0C2F
:10A190000C0C0C0C0C0C0C0C0C0C0C0C0C0C0C0CFF
:10A1A0000C0C0C0C0C0C0C0C0C0C0C0C0C0C0C0CEF
:10A1B0000C0C0C0C0C0C0C0C0C0C0C0C0C0C0C0CDF
:10A1C00008080808080808080C0C0C0C0C0C0C0CEF
:10A1D0000C0C0C0C0C0C0C0C0C0C0C0C0C0C0C0CBF
:10A1E0000C0C0C0C0C0C0C0C0C0C0C0C0C0C0C0CAF
:10A1F0000C0C0C0C0C0C0C0C0C0C0C0C0C0C0C0C9F
:10A2000008080808080808080C0C0C0C0C0C0C0CAE
:10A210000C0C0C0C0C0C0C0C0C0C0C0C0C0C0C0C7E
:10A220000C0C0C0C0C0C0C0C0C0C0C0C0C0C0C0C6E
:10A230000C0C0C0C0C0C0C0C0C0C0C0C0C0C0C0C5E
:10A2400008080808080808080C0C0C0C0C0C0C0C6E
:10A250000C0C0C0C0C0C0C0C0C0C0C0C0C0C0C0C3E
:10A260000C0C0C0C0C0C0C0C0C0C0C0C0C0C0C0C2E
:10A270000C0C0C0C0C0C0C0C0C0C0C0C0C0C0C0C1E
:10A2800008080808080808080C0C0C0C0C0C0C0C2E
:10A290000C0C0C0C0C0C0C0C0C0C0C0C0C0C0C0CFE
:10A2A0000C0C0C0C0C0C0C0C0C0C0C0C0C0C0C0CEE
:10A2B0000C0C0C0C0C0C0C0C0C0C0C0C0C0C0C0CDE
:10A2C00008080808080808080C0C0C0C0C0C0C0CEE
:10A2D0000C0C0C0C0C0C0C0C0C0C0C0C0C0C0C0CBE
:10A2E0000C0C0C0C0C0C0C0C0C0C0C0C0C0C0C0CAE
:10A2F0000C0C0C0C0C0C0C0C0C0C0C0C0C0C0C0C9E
:10A3000008080808080808080C0C0C0C0C0C0C0CAD
:10A310000C0C0C0C0C0C0C0C0C0C0C0C0C0C0C0C7D
:10A320000C0C0C0C0C0C0C0C0C0C0C0C0C0C0C0C6D
:10A330000C0C0C0C0C0C0C0C0C0C0C0C0C0C0C0C5D
:10A3400008080808080808080C0C0C0C0C0C0C0C6D
:10A350000C0C0C0C0C0C0C0C0C0C0C0C0C0C0C0C3D
:10A360000C0C0C0C0C0C0C0C0C0C0C0C0C0C0C0C2D
:10A370000C0C0C0C0C0C0C0C0C0C0C0C0C0C0C0C1D
:10A3800008080808080808080C0C0C0C0C0C0C0C2D
:10A390000C0C0C0C0C0C0C0C0C0C0C0C0C0C0C0CFD
:10A3A0000C0C0C0C0C0C0C0C0C0C0C0C0C0C0C0CED
:10A3B0000C0C0C0C0C0C0C0C0C0C0C0C0C0C0C0CDD
:10A3C00008080808080808080C0C0C0C0C0C0C0CED
:10A3D0000C0C0C0C0C0C0C0C0C0C0C0C0C0C0C0CBD
:10A3E0000C0C0C0C0C0C0C0C0C0C0C0C0C0C0C0CAD
:10A3F0000C0C0C0C0C0C0C0C0C0C0C0C0C0C0C0C9D
:10A4000008080808080808080C0C0C0C0C0C0C0CAC
:10A410000C0C0C0C0C0C0C0C0C0C0C0C0C0C0C0C7C
:10A420000C0C0C0C0C0C0C0C0C0C0C0C0C0C0C0C6C
:10A430000C0C0C0C0C0C0C0C0C0C0C0C0C0C0C0C5C
:10A4400008080808080808080C0C0C0C0C0C0C0C6C
:10A450000C0C0C0C0C0C0C0C0C0C0C0C0C0C0C0C3C
:10A460000C0C0C0C0C0C0C0C0C0C0C0C0C0C0C0C2C
:10A470000C0C0C0C0C0C0C0C0C0C0C0C0C0C0C0C1C
:10A4800008080808080808080C0C0C0C0C0C0C0C2C
:10A490000C0C0C0C0C0C0C0C0C0C0C0C0C0C0C0CFC
:10A4A0000C0C0C0C0C0C0C0C0C0C0C0C0C0C0C0CEC
:10A4B0000C0C0C0C0C0C0C0C0C0C0C0C0C0C0C0CDC
:10A4C00008080808080808080C0C0C0C0C0C0C0CEC
:10A4D0000C0C0C0C0C0C0C0C0C0C0C0C0C0C0C0CBC
:10A4E0000C0C0C0C0C0C0C0C0C0C0C0C0C0C0C0CAC
:10A4F0000C0C0C0C0C0C0C0C0C0C0C0C0C0C0C0C9C
:10A5000008080808080808080C0C0C0C0C0C0C0CAB
:10A510000C0C0C0C0C0C0C0C0C0C0C0C0C0C0C0C7B
:10A520000C0C0C0C0C0C0C0C0C0C0C0C0C0C0C0C6B
:10A530000C0C0C0C0C0C0C0C0C0C0C0C0C0C0C0C5B
:10A5400008080808080808080C0C0C0C0C0C0C0C6B
:10A550000C0C0C0C0C0C0C0C0C0C0C0C0C0C0C0C3B
:10A560000C0C0C0C0C0C0C0C0C0C0C0C0C0C0C0C2B
:10A570000C0C0C0C0C0C0C0C0C0C0C0C0C0C0C0C1B
:10A5800008080808080808080C0C0C0C0C0C0C0C2B
:10A590000C0C0C0C0C0C0C0C0C0C0C0C0C0C0C0CFB
:10A5A0000C0C0C0C0C0C0C0C0C0C0C0C0C0C0C0CEB
:10A5B0000C0C0C0C0C0C0C0C0C0C0C0C0C0C0C0CDB
:10A5C00008080808080808080C0C0C0C0C0C0C0CEB
:10A5D0000C0C0C0C0C0C0C0C0C0C0C0C0C0C0C0CBB
:10A5E0000C0C0C0C0C0C0C0C0C0C0C0C0C0C0C0CAB
:10A5F0000C0C0C0C0C0C0C0C0C0C0C0C0C0C0C0C9B
:10A6000008080808080808080C0C0C0C0C0C0C0CAA
:10A610000C0C0C0C0C0C0C0C0C0C0C0C0C0C0C0C7A
:10A620000C0C0C0C0C0C0C0C0C0C0C0C0C0C0C0C6A
:10A630000C0C0C0C0C0C0C0C0C0C0C0C0C0C0C0C5A
:10A6400008080808080808080C0C0C0C0C0C0C0C6A
:10A650000C0C0C0C0C0C0C0C0C0C0C0C0C0C0C0C3A
:10A660000C0C0C0C0C0C0C0C0C0C0C0C0C0C0C0C2A
:10A670000C0C0C0C0C0C0C0C0C0C0C0C0C0C0C0C1A
:10A6800008080808080808080C0C0C0C0C0C0C0C2A
:10A690000C0C0C0C0C0C0C0C0C0C0C0C0C0C0C0CFA
:10A6A0000C0C0C0C0C0C0C0C0C0C0C0C0C0C0C0CEA
:10A6B0000C0C0C0C0C0C0C0C0C0C0C0C0C0C0C0CDA
:10A6C00008080808080808080C0C0C0C0C0C0C0CEA
:10A6D0000C0C0C0C0C0C0C0C0C0C0C0C0C0C0C0CBA
:10A6E0000C0C0C0C0C0C0C0C0C0C0C0C0C0C0C0CAA
:10A6F0000C0C0C0C0C0C0C0C0C0C0C0C0C0C0C0C9A
:10A7000008080808080808080C0C0C0C0C0C0C0CA9
:10A710000C0C0C0C0C0C0C0C0C0C0C0C0C0C0C0C79
:10A720000C0C0C0C0C0C0C0C0C0C0C0C0C0C0C0C69
:10A730000C0C0C0C0C0C0C0C0C0C0C0C0C0C0C0C59
:10A7400008080808080808080C0C0C0C0C0C0C0C69
:10A750000C0C0C0C0C0C0C0C0C0C0C0C0C0C0C0C39
:10A760000C0C0C0C0C0C0C0C0C0C0C0C0C0C0C0C29
:10A770000C0C0C0C0C0C0C0C0C0C0C0C0C0C0C0C19
:10A7800008080808080808080C0C0C0C0C0C0C0C29
:10A790000C0C0C0C0C0C0C0C0C0C0C0C0C0C0C0CF9
:10A7A0000C0C0C0C0C0C0C0C0C0C0C0C0C0C0C0CE9
:10A7B0000C0C0C0C0C0C0C0C0C0C0C0C0C0C0C0CD9
:10A7C00008080808080808080C0C0C0C0C0C0C0CE9
:10A7D0000C0C0C0C0C0C0C0C0C0C0C0C0C0C0C0CB9
:10A7E0000C0C0C0C0C0C0C0C0C0C0C0C0C0C0C0CA9
:10A7F0000C0C0C0C0C0C0C0C0C0C0C0C0C0C0C0C99
:10A8000008080808080808080C0C0C0C0C0C0C0CA8
:10A810000C0C0C0C0C0C0C0C0C0C0C0C0C0C0C0C78
:10A820000C0C0C0C0C0C0C0C0C0C0C0C0C0C0C0C68
:10A830000C0C0C0C0C0C0C0C0C0C0C0C0C0C0C0C58
:10A8400008080808080808080C0C0C0C0C0C0C0C68
:10A850000C0C0C0C0C0C0C0C0C0C0C0C0C0C0C0C38
:10A860000C0C0C0C0C0C0C0C0C0C0C0C0C0C0C0C28
:10A870000C0C0C0C0C0C0C0C0C0C0C0C0C0C0C0C18
:10A8800008080808080808080C0C0C0C0C0C0C0C28
:10A890000C0C0C0C0C0C0C0C0C0C0C0C0C0C0C0CF8
:10A8A0000C0C0C0C0C0C0C0C0C0C0C0C0C0C0C0CE8
:10A8B0000C0C0C0C0C0C0C0C0C0C0C0C0C0C0C0CD8
:10A8C00008080808080808080C0C0C0C0C0C0C0CE8
:10A8D0000C0C0C0C0C0C0C0C0C0C0C0C0C0C0C0CB8
:10A8E0000C0C0C0C0C0C0C0C0C0C0C0C0C0C0C0CA8
:10A8F0000C0C0C0C0C0C0C0C0C0C0C0C0C0C0C0C98
:10A9000008080808080808080C0C0C0C0C0C0C0CA7
:10A910000C0C0C0C0C0C0C0C0C0C0C0C0C0C0C0C77
:10A920000C0C0C0C0C0C0C0C0C0C0C0C0C0C0C0C67
:10A930000C0C0C0C0C0C0C0C0C0C0C0C0C0C0C0C57
:10A9400008080808080808080C0C0C0C0C0C0C0C67
:10A950000C0C0C0C0C0C0C0C0C0C0C0C0C0C0C0C37
:10A960000C0C0C0C0C0C0C0C0C0C0C0C0C0C0C0C27
:10A970000C0C0C0C0C0C0C0C0C0C0C0C0C0C0C0C17
:10A9800008080808080808080C0C0C0C0C0C0C0C27
:10A990000C0C0C0C0C0C0C0C0C0C0C0C0C0C0C0CF7
:10A9A0000C0C0C0C0C0C0C0C0C0C0C0C0C0C0C0CE7
:10A9B0000C0C0C0C0C0C0C0C0C0C0C0C0C0C0C0CD7
:10A9C00008080808080808080C0C0C0C0C0C0C0CE7
:10A9D0000C0C0C0C0C0C0C0C0C0C0C0C0C0C0C0CB7
:10A9E0000C0C0C0C0C0C0C0C0C0C0C0C0C0C0C0CA7
:10A9F0000C0C0C0C0C0C0C0C0C0C0C0C0C0C0C0C97
:10AA000008080808080808080C0C0C0C0C0C0C0CA6
:10AA10000C0C0C0C0C0C0C0C0C0C0C0C0C0C0C0C76
:10AA20000C0C0C0C0C0C0C0C0C0C0C0C0C0C0C0C66
:10AA30000C0C0C0C0C0C0C0C0C0C0C0C0C0C0C0C56
:10AA400008080808080808080C0C0C0C0C0C0C0C66
:10AA50000C0C0C0C0C0C0C0C0C0C0C0C0C0C0C0C36
:10AA60000C0C0C0C0C0C0C0C0C0C0C0C0C0C0C0C26
:10AA70000C0C0C0C0C0C0C0C0C0C0C0C0C0C0C0C16
:10AA800008080808080808080C0C0C0C0C0C0C0C26
:10AA90000C0C0C0C0C0C0C0C0C0C0C0C0C0C0C0CF6
:10AAA0000C0C0C0C0C0C0C0C0C0C0C0C0C0C0C0CE6
:10AAB0000C0C0C0C0C0C0C0C0C0C0C0C0C0C0C0CD6
:10AAC00008080808080808080C0C0C0C0C0C0C0CE6
:10AAD0000C0C0C0C0C0C0C0C0C0C0C0C0C0C0C0CB6
:10AAE0000C0C0C0C0C0C0C0C0C0C0C0C0C0C0C0CA6
:10AAF0000C0C0C0C0C0C0C0C0C0C0C0C0C0C0C0C96
:10AB000008080808080808080C0C0C0C0C0C0C0CA5
:10AB10000C0C0C0C0C0C0C0C0C0C0C0C0C0C0C0C75
:10AB20000C0C0C0C0C0C0C0C0C0C0C0C0C0C0C0C65
:10AB30000C0C0C0C0C0C0C0C0C0C0C0C0C0C0C0C55
:10AB400008080808080808080C0C0C0C0C0C0C0C65
:10AB50000C0C0C0C0C0C0C0C0C0C0C0C0C0C0C0C35
:10AB60000C0C0C0C0C0C0C0C0C0C0C0C0C0C0C0C25
:10AB70000C0C0C0C0C0C0C0C0C0C0C0C0C0C0C0C15
:10AB800008080808080808080C0C0C0C0C0C0C0C25
:10AB90000C0C0C0C0C0C0C0C0C0C0C0C0C0C0C0CF5
:10ABA0000C0C0C0C0C0C0C0C0C0C0C0C0C0C0C0CE5
:10ABB0000C0C0C0C0C0C0C0C0C0C0C0C0C0C0C0CD5
:10ABC00008080808080808080C0C0C0C0C0C0C0CE5
:10ABD0000C0C0C0C0C0C0C0C0C0C0C0C0C0C0C0CB5
:10ABE0000C0C0C0C0C0C0C0C0C0C0C0C0C0C0C0CA5
:10ABF0000C0C0C0C0C0C0C0C0C0C0C0C0C0C0C0C95
:10AC000008080808080808080C0C0C0C0C0C0C0CA4
:10AC10000C0C0C0C0C0C0C0C0C0C0C0C0C0C0C0C74
:10AC20000C0C0C0C0C0C0C0C0C0C0C0C0C0C0C0C64
:10AC30000C0C0C0C0C0C0C0C0C0C0C0C0C0C0C0C54
:10AC400008080808080808080C0C0C0C0C0C0C0C64
:10AC50000C0C0C0C0C0C0C0C0C0C0C0C0C0C0C0C34
:10AC60000C0C0C0C0C0C0C0C0C0C0C0C0C0C0C0C24
:10AC70000C0C0C0C0C0C0C0C0C0C0C0C0C0C0C0C14
:10AC800008080808080808080C0C0C0C0C0C0C0C24
:10AC90000C0C0C0C0C0C0C0C0C0C0C0C0C0C0C0CF4
:10ACA0000C0C0C0C0C0C0C0C0C0C0C0C0C0C0C0CE4
:10ACB0000C0C0C0C0C0C0C0C0C0C0C0C0C0C0C0CD4
:10ACC00008080808080808080C0C0C0C0C0C0C0CE4
:10ACD0000C0C0C0C0C0C0C0C0C0C0C0C0C0C0C0CB4
:10ACE0000C0C0C0C0C0C0C0C0C0C0C0C0C0C0C0CA4
:10ACF0000C0C0C0C0C0C0C0C0C0C0C0C0C0C0C0C94
:10AD000008080808080808080C0C0C0C0C0C0C0CA3
:10AD10000C0C0C0C0C0C0C0C0C0C0C0C0C0C0C0C73
:10AD20000C0C0C0C0C0C0C0C0C0C0C0C0C0C0C0C63
:10AD30000C0C0C0C0C0C0C0C0C0C0C0C0C0C0C0C53
:10AD400008080808080808080C0C0C0C0C0C0C0C63
:10AD50000C0C0C0C0C0C0C0C0C0C0C0C0C0C0C0C33
:10AD60000C0C0C0C0C0C0C0C0C0C0C0C0C0C0C0C23
:10AD70000C0C0C0C0C0C0C0C0C0C0C0C0C0C0C0C13
:10AD800008080808080808080C0C0C0C0C0C0C0C23
:10AD90000C0C0C0C0C0C0C0C0C0C0C0C0C0C0C0CF3
:10ADA0000C0C0C0C0C0C0C0C0C0C0C0C0C0C0C0CE3
:10ADB0000C0C0C0C0C0C0C0C0C0C0C0C0C0C0C0CD3
:10ADC00008080808080808080C0C0C0C0C0C0C0CE3
:10ADD0000C0C0C0C0C0C0C0C0C0C0C0C0C0C0C0CB3
:10ADE0000C0C0C0C0C0C0C0C0C0C0C0C0C0C0C0CA3
:10ADF0000C0C0C0C0C0C0C0C0C0C0C0C0C0C0C0C93
:10AE000008080808080808080C0C0C0C0C0C0C0CA2
:10AE10000C0C0C0C0C0C0C0C0C0C0C0C0C0C0C0C72
:10AE20000C0C0C0C0C0C0C0C0C0C0C0C0C0C0C0C62
:10AE30000C0C0C0C0C0C0C0C0C0C0C0C0C0C0C0C52
:10AE400008080808080808080C0C0C0C0C0C0C0C62
:10AE50000C0C0C0C0C0C0C0C0C0C0C0C0C0C0C0C32
:10AE60000C0C0C0C0C0C0C0C0C0C0C0C0C0C0C0C22
:10AE70000C0C0C0C0C0C0C0C0C0C0C0C0C0C0C0C12
:10AE800008080808080808080C0C0C0C0C0C0C0C22
:10AE90000C0C0C0C0C0C0C0C0C0C0C0C0C0C0C0CF2
:10AEA0000C0C0C0C0C0C0C0C0C0C0C0C0C0C0C0CE2
:10AEB0000C0C0C0C0C0C0C0C0C0C0C0C0C0C0C0CD2
:10AEC00008080808080808080C0C0C0C0C0C0C0CE2
:10AED0000C0C0C0C0C0C0C0C0C0C0C0C0C0C0C0CB2
:10AEE0000C0C0C0C0C0C0C0C0C0C0C0C0C0C0C0CA2
:10AEF0000C0C0C0C0C0C0C0C0C0C0C0C0C0C0C0C92
:10AF000008080808080808080C0C0C0C0C0C0C0CA1
:10AF10000C0C0C0C0C0C0C0C0C0C0C0C0C0C0C0C71
:10AF20000C0C0C0C0C0C0C0C0C0C0C0C0C0C0C0C61
:10AF30000C0C0C0C0C0C0C0C0C0C0C0C0C0C0C0C51
:10AF400008080808080808080C0C0C0C0C0C0C0C61
:10AF50000C0C0C0C0C0C0C0C0C0C0C0C0C0C0C0C31
:10AF60000C0C0C0C0C0C0C0C0C0C0C0C0C0C0C0C21
:10AF70000C0C0C0C0C0C0C0C0C0C0C0C0C0C0C0C11
:10AF800008080808080808080C0C0C0C0C0C0C0C21
:10AF90000C0C0C0C0C0C0C0C0C0C0C0C0C0C0C0CF1
:10AFA0000C0C0C0C0C0C0C0C0C0C0C0C0C0C0C0CE1
:10AFB0000C0C0C0C0C0C0C0C0C0C0C0C0C0C0C0CD1
:10AFC00008080808080808080C0C0C0C0C0C0C0CE1
:10AFD0000C0C0C0C0C0C0C0C0C0C0C0C0C0C0C0CB1
:10AFE0000C0C0C0C0C0C0C0C0C0C0C0C0C0C0C0CA1
:10AFF0000C0C0C0C0C0C0C0C0C0C0C0C0C0C0C0C91
:10B0000008080808080808080C0C0C0C0C0C0C0CA0
:10B010000C0C0C0C0C0C0C0C0C0C0C0C0C0C0C0C70
:10B020000C0C0C0C0C0C0C0C0C0C0C0C0C0C0C0C60
:10B030000C0C0C0C0C0C0C0C0C0C0C0C0C0C0C0C50
:10B0400008080808080808080C0C0C0C0C0C0C0C60
:10B050000C0C0C0C0C0C0C0C0C0C0C0C0C0C0C0C30
:10B060000C0C0C0C0C0C0C0C0C0C0C0C0C0C0C0C20
:10B070000C0C0C0C0C0C0C0C0C0C0C0C0C0C0C0C10
:10B0800008080808080808080C0C0C0C0C0C0C0C20
:10B090000C0C0C0C0C0C0C0C0C0C0C0C0C0C0C0CF0
:10B0A0000C0C0C0C0C0C0C0C0C0C0C0C0C0C0C0CE0
:10B0B0000C0C0C0C0C0C0C0C0C0C0C0C0C0C0C0CD0
:10B0C00008080808080808080C0C0C0C0C0C0C0CE0
:10B0D0000C0C0C0C0C0C0C0C0C0C0C0C0C0C0C0CB0
:10B0E0000C0C0C0C0C0C0C0C0C0C0C0C0C0C0C0CA0
:10B0F0000C0C0C0C0C0C0C0C0C0C0C0C0C0C0C0C90
:10B1000008080808080808080C0C0C0C0C0C0C0C9F
:10B110000C0C0C0C0C0C0C0C0C0C0C0C0C0C0C0C6F
:10B120000C0C0C0C0C0C0C0C0C0C0C0C0C0C0C0C5F
:10B130000C0C0C0C0C0C0C0C0C0C0C0C0C0C0C0C4F
:10B1400008080808080808080C0C0C0C0C0C0C0C5F
:10B150000C0C0C0C0C0C0C0C0C0C0C0C0C0C0C0C2F
:10B160000C0C0C0C0C0C0C0C0C0C0C0C0C0C0C0C1F
:10B170000C0C0C0C0C0C0C0C0C0C0C0C0C0C0C0C0F
:10B1800008080808080808080C0C0C0C0C0C0C0C1F
:10B190000C0C0C0C0C0C0C0C0C0C0C0C0C0C0C0CEF
:10B1A0000C0C0C0C0C0C0C0C0C0C0C0C0C0C0C0CDF
:10B1B0000C0C0C0C0C0C0C0C0C0C0C0C0C0C0C0CCF
:10B1C00008080808080808080C0C0C0C0C0C0C0CDF
:10B1D0000C0C0C0C0C0C0C0C0C0C0C0C0C0C0C0CAF
:10B1E0000C0C0C0C0C0C0C0C0C0C0C0C0C0C0C0C9F
:10B1F0000C0C0C0C0C0C0C0C0C0C0C0C0C0C0C0C8F
:10B2000008080808080808080C0C0C0C0C0C0C0C9E
:10B210000C0C0C0C0C0C0C0C0C0C0C0C0C0C0C0C6E
:10B220000C0C0C0C0C0C0C0C0C0C0C0C0C0C0C0C5E
:10B230000C0C0C0C0C0C0C0C0C0C0C0C0C0C0C0C4E
:10B2400008080808080808080C0C0C0C0C0C0C0C5E
:10B250000C0C0C0C0C0C0C0C0C0C0C0C0C0C0C0C2E
:10B260000C0C0C0C0C0C0C0C0C0C0C0C0C0C0C0C1E
:10B270000C0C0C0C0C0C0C0C0C0C0C0C0C0C0C0C0E
:10B2800008080808080808080C0C0C0C0C0C0C0C1E
:10B290000C0C0C0C0C0C0C0C0C0C0C0C0C0C0C0CEE
:10B2A0000C0C0C0C0C0C0C0C0C0C0C0C0C0C0C0CDE
:10B2B0000C0C0C0C0C0C0C0C0C0C0C0C0C0C0C0CCE
:10B2C00008080808080808080C0C0C0C0C0C0C0CDE
:10B2D0000C0C0C0C0C0C0C0C0C0C0C0C0C0C0C0CAE
:10B2E0000C0C0C0C0C0C0C0C0C0C0C0C0C0C0C0C9E
:10B2F0000C0C0C0C0C0C0C0C0C0C0C0C0C0C0C0C8E
:10B3000008080808080808080C0C0C0C0C0C0C0C9D
:10B310000C0C0C0C0C0C0C0C0C0C0C0C0C0C0C0C6D
:10B320000C0C0C0C0C0C0C0C0C0C0C0C0C0C0C0C5D
:10B330000C0C0C0C0C0C0C0C0C0C0C0C0C0C0C0C4D
:10B3400008080808080808080C0C0C0C0C0C0C0C5D
:10B350000C0C0C0C0C0C0C0C0C0C0C0C0C0C0C0C2D
:10B360000C0C0C0C0C0C0C0C0C0C0C0C0C0C0C0C1D
:10B370000C0C0C0C0C0C0C0C0C0C0C0C0C0C0C0C0D
:10B3800008080808080808080C0C0C0C0C0C0C0C1D
:10B390000C0C0C0C0C0C0C0C0C0C0C0C0C0C0C0CED
:10B3A0000C0C0C0C0C0C0C0C0C0C0C0C0C0C0C0CDD
:10B3B0000C0C0C0C0C0C0C0C0C0C0C0C0C0C0C0CCD
:10B3C00008080808080808080C0C0C0C0C0C0C0CDD
:10B3D0000C0C0C0C0C0C0C0C0C0C0C0C0C0C0C0CAD
:10B3E0000C0C0C0C0C0C0C0C0C0C0C0C0C0C0C0C9D
:10B3F0000C0C0C0C0C0C0C0C0C0C0C0C0C0C0C0C8D
:10B4000008080808080808080C0C0C0C0C0C0C0C9C
:10B410000C0C0C0C0C0C0C0C0C0C0C0C0C0C0C0C6C
:10B420000C0C0C0C0C0C0C0C0C0C0C0C0C0C0C0C5C
:10B430000C0C0C0C0C0C0C0C0C0C0C0C0C0C0C0C4C
:10B4400008080808080808080C0C0C0C0C0C0C0C5C
:10B450000C0C0C0C0C0C0C0C0C0C0C0C0C0C0C0C2C
:10B460000C0C0C0C0C0C0C0C0C0C0C0C0C0C0C0C1C
:10B470000C0C0C0C0C0C0C0C0C0C0C0C0C0C0C0C0C
:10B4800008080808080808080C0C0C0C0C0C0C0C1C
:10B490000C0C0C0C0C0C0C0C0C0C0C0C0C0C0C0CEC
:10B4A0000C0C0C0C0C0C0C0C0C0C0C0C0C0C0C0CDC
:10B4B0000C0C0C0C0C0C0C0C0C0C0C0C0C0C0C0CCC
:10B4C00008080808080808080C0C0C0C0C0C0C0CDC
:10B4D0000C0C0C0C0C0C0C0C0C0C0C0C0C0C0C0CAC
:10B4E0000C0C0C0C0C0C0C0C0C0C0C0C0C0C0C0C9C
:10B4F0000C0C0C0C0C0C0C0C0C0C0C0C0C0C0C0C8C
:10B5000008080808080808080C0C0C0C0C0C0C0C9B
:10B510000C0C0C0C0C0C0C0C0C0C0C0C0C0C0C0C6B
:10B520000C0C0C0C0C0C0C0C0C0C0C0C0C0C0C0C5B
:10B530000C0C0C0C0C0C0C0C0C0C0C0C0C0C0C0C4B
:10B5400008080808080808080C0C0C0C0C0C0C0C5B
:10B550000C0C0C0C0C0C0C0C0C0C0C0C0C0C0C0C2B
:10B560000C0C0C0C0C0C0C0C0C0C0C0C0C0C0C0C1B
:10B570000C0C0C0C0C0C0C0C0C0C0C0C0C0C0C0C0B
:10B5800008080808080808080C0C0C0C0C0C0C0C1B
:10B590000C0C0C0C0C0C0C0C0C0C0C0C0C0C0C0CEB
:10B5A0000C0C0C0C0C0C0C0C0C0C0C0C0C0C0C0CDB
:10B5B0000C0C0C0C0C0C0C0C0C0C0C0C0C0C0C0CCB
:10B5C00008080808080808080C0C0C0C0C0C0C0CDB
:10B5D0000C0C0C0C0C0C0C0C0C0C0C0C0C0C0C0CAB
:10B5E0000C0C0C0C0C0C0C0C0C0C0C0C0C0C0C0C9B
:10B5F0000C0C0C0C0C0C0C0C0C0C0C0C0C0C0C0C8B
:10B6000008080808080808080C0C0C0C0C0C0C0C9A
:10B610000C0C0C0C0C0C0C0C0C0C0C0C0C0C0C0C6A
:10B620000C0C0C0C0C0C0C0C0C0C0C0C0C0C0C0C5A
:10B630000C0C0C0C0C0C0C0C0C0C0C0C0C0C0C0C4A
:10B6400008080808080808080C0C0C0C0C0C0C0C5A
:10B650000C0C0C0C0C0C0C0C0C0C0C0C0C0C0C0C2A
:10B660000C0C0C0C0C0C0C0C0C0C0C0C0C0C0C0C1A
:10B670000C0C0C0C0C0C0C0C0C0C0C0C0C0C0C0C0A
:10B6800008080808080808080C0C0C0C0C0C0C0C1A
:10B690000C0C0C0C0C0C0C0C0C0C0C0C0C0C0C0CEA
:10B6A0000C0C0C0C0C0C0C0C0C0C0C0C0C0C0C0CDA
:10B6B0000C0C0C0C0C0C0C0C0C0C0C0C0C0C0C0CCA
:10B6C00008080808080808080C0C0C0C0C0C0C0CDA
:10B6D0000C0C0C0C0C0C0C0C0C0C0C0C0C0C0C0CAA
:10B6E0000C0C0C0C0C0C0C0C0C0C0C0C0C0C0C0C9A
:10B6F0000C0C0C0C0C0C0C0C0C0C0C0C0C0C0C0C8A
:10B7000008080808080808080C0C0C0C0C0C0C0C99
:10B710000C0C0C0C0C0C0C0C0C0C0C0C0C0C0C0C69
:10B720000C0C0C0C0C0C0C0C0C0C0C0C0C0C0C0C59
:10B730000C0C0C0C0C0C0C0C0C0C0C0C0C0C0C0C49
:10B7400008080808080808080C0C0C0C0C0C0C0C59
:10B750000C0C0C0C0C0C0C0C0C0C0C0C0C0C0C0C29
:10B760000C0C0C0C0C0C0C0C0C0C0C0C0C0C0C0C19
:10B770000C0C0C0C0C0C0C0C0C0C0C0C0C0C0C0C09
:10B7800008080808080808080C0C0C0C0C0C0C0C19
:10B790000C0C0C0C0C0C0C0C0C0C0C0C0C0C0C0CE9
:10B7A0000C0C0C0C0C0C0C0C0C0C0C0C0C0C0C0CD9
:10B7B0000C0C0C0C0C0C0C0C0C0C0C0C0C0C0C0CC9
:10B7C00008080808080808080C0C0C0C0C0C0C0CD9
:10B7D0000C0C0C0C0C0C0C0C0C0C0C0C0C0C0C0CA9
:10B7E0000C0C0C0C0C0C0C0C0C0C0C0C0C0C0C0C99
:10B7F0000C0C0C0C0C0C0C0C0C0C0C0C0C0C0C0C89
:10B8000008080808080808080C0C0C0C0C0C0C0C98
:10B810000C0C0C0C0C0C0C0C0C0C0C0C0C0C0C0C68
:10B820000C0C0C0C0C0C0C0C0C0C0C0C0C0C0C0C58
:10B830000C0C0C0C0C0C0C0C0C0C0C0C0C0C0C0C48
:10B8400008080808080808080C0C0C0C0C0C0C0C58
:10B850000C0C0C0C0C0C0C0C0C0C0C0C0C0C0C0C28
:10B860000C0C0C0C0C0C0C0C0C0C0C0C0C0C0C0C18
:10B870000C0C0C0C0C0C0C0C0C0C0C0C0C0C0C0C08
:10B8800008080808080808080C0C0C0C0C0C0C0C18
:10B890000C0C0C0C0C0C0C0C0C0C0C0C0C0C0C0CE8
:10B8A0000C0C0C0C0C0C0C0C0C0C0C0C0C0C0C0CD8
:10B8B0000C0C0C0C0C0C0C0C0C0C0C0C0C0C0C0CC8
:10B8C00008080808080808080C0C0C0C0C0C0C0CD8
:10B8D0000C0C0C0C0C0C0C0C0C0C0C0C0C0C0C0CA8
:10B8E0000C0C0C0C0C0C0C0C0C0C0C0C0C0C0C0C98
:10B8F0000C0C0C0C0C0C0C0C0C0C0C0C0C0C0C0C88
:10B9000008080808080808080C0C0C0C0C0C0C0C97
:10B910000C0C0C0C0C0C0C0C0C0C0C0C0C0C0C0C67
:10B920000C0C0C0C0C0C0C0C0C0C0C0C0C0C0C0C57
:10B930000C0C0C0C0C0C0C0C0C0C0C0C0C0C0C0C47
:10B9400008080808080808080C0C0C0C0C0C0C0C57
:10B950000C0C0C0C0C0C0C0C0C0C0C0C0C0C0C0C27
:10B960000C0C0C0C0C0C0C0C0C0C0C0C0C0C0C0C17
:10B970000C0C0C0C0C0C0C0C0C0C0C0C0C0C0C0C07
:10B9800008080808080808080C0C0C0C0C0C0C0C17
:10B990000C0C0C0C0C0C0C0C0C0C0C0C0C0C0C0CE7
:10B9A0000C0C0C0C0C0C0C0C0C0C0C0C0C0C0C0CD7
:10B9B0000C0C0C0C0C0C0C0C0C0C0C0C0C0C0C0CC7
:10B9C00008080808080808080C0C0C0C0C0C0C0CD7
:10B9D0000C0C0C0C0C0C0C0C0C0C0C0C0C0C0C0CA7
:10B9E0000C0C0C0C0C0C0C0C0C0C0C0C0C0C0C0C97
:10B9F0000C0C0C0C0C0C0C0C0C0C0C0C0C0C0C0C87
:10BA000008080808080808080C0C0C0C0C0C0C0C96
:10BA10000C0C0C0C0C0C0C0C0C0C0C0C0C0C0C0C66
:10BA20000C0C0C0C0C0C0C0C0C0C0C0C0C0C0C0C56
:10BA30000C0C0C0C0C0C0C0C0C0C0C0C0C0C0C0C46
:10BA400008080808080808080C0C0C0C0C0C0C0C56
:10BA50000C0C0C0C0C0C0C0C0C0C0C0C0C0C0C0C26
:10BA60000C0C0C0C0C0C0C0C0C0C0C0C0C0C0C0C16
:10BA70000C0C0C0C0C0C0C0C0C0C0C0C0C0C0C0C06
:10BA800008080808080808080C0C0C0C0C0C0C0C16
:10BA90000C0C0C0C0C0C0C0C0C0C0C0C0C0C0C0CE6
:10BAA0000C0C0C0C0C0C0C0C0C0C0C0C0C0C0C0CD6
:10BAB0000C0C0C0C0C0C0C0C0C0C0C0C0C0C0C0CC6
:10BAC00008080808080808080C0C0C0C0C0C0C0CD6
:10BAD0000C0C0C0C0C0C0C0C0C0C0C0C0C0C0C0CA6
:10BAE0000C0C0C0C0C0C0C0C0C0C0C0C0C0C0C0C96
:10BAF0000C0C0C0C0C0C0C0C0C0C0C0C0C0C0C0C86
:10BB000008080808080808080C0C0C0C0C0C0C0C95
:10BB10000C0C0C0C0C0C0C0C0C0C0C0C0C0C0C0C65
:10BB20000C0C0C0C0C0C0C0C0C0C0C0C0C0C0C0C55
:10BB30000C0C0C0C0C0C0C0C0C0C0C0C0C0C0C0C45
:10BB400008080808080808080C0C0C0C0C0C0C0C55
:10BB50000C0C0C0C0C0C0C0C0C0C0C0C0C0C0C0C25
:10BB60000C0C0C0C0C0C0C0C0C0C0C0C0C0C0C0C15
:10BB70000C0C0C0C0C0C0C0C0C0C0C0C0C0C0C0C05
:10BB800008080808080808080C0C0C0C0C0C0C0C15
:10BB90000C0C0C0C0C0C0C0C0C0C0C0C0C0C0C0CE5
:10BBA0000C0C0C0C0C0C0C0C0C0C0C0C0C0C0C0CD5
:10BBB0000C0C0C0C0C0C0C0C0C0C0C0C0C0C0C0CC5
:10BBC00008080808080808080C0C0C0C0C0C0C0CD5
:10BBD0000C0C0C0C0C0C0C0C0C0C0C0C0C0C0C0CA5
:10BBE0000C0C0C0C0C0C0C0C0C0C0C0C0C0C0C0C95
:10BBF0000C0C0C0C0C0C0C0C0C0C0C0C0C0C0C0C85
:10BC000008080808080808080C0C0C0C0C0C0C0C94
:10BC10000C0C0C0C0C0C0C0C0C0C0C0C0C0C0C0C64
:10BC20000C0C0C0C0C0C0C0C0C0C0C0C0C0C0C0C54
:10BC30000C0C0C0C0C0C0C0C0C0C0C0C0C0C0C0C44
:10BC400008080808080808080C0C0C0C0C0C0C0C54
:10BC50000C0C0C0C0C0C0C0C0C0C0C0C0C0C0C0C24
:10BC60000C0C0C0C0C0C0C0C0C0C0C0C0C0C0C0C14
:10BC70000C0C0C0C0C0C0C0C0C0C0C0C0C0C0C0C04
:10BC800008080808080808080C0C0C0C0C0C0C0C14
:10BC90000C0C0C0C0C0C0C0C0C0C0C0C0C0C0C0CE4
:10BCA0000C0C0C0C0C0C0C0C0C0C0C0C0C0C0C0CD4
:10BCB0000C0C0C0C0C0C0C0C0C0C0C0C0C0C0C0CC4
:10BCC00008080808080808080C0C0C0C0C0C0C0CD4
:10BCD0000C0C0C0C0C0C0C0C0C0C0C0C0C0C0C0CA4
:10BCE0000C0C0C0C0C0C0C0C0C0C0C0C0C0C0C0C94
:10BCF0000C0C0C0C0C0C0C0C0C0C0C0C0C0C0C0C84
:10BD000008080808080808080C0C0C0C0C0C0C0C93
:10BD10000C0C0C0C0C0C0C0C0C0C0C0C0C0C0C0C63
:10BD20000C0C0C0C0C0C0C0C0C0C0C0C0C0C0C0C53
:10BD30000C0C0C0C0C0C0C0C0C0C0C0C0C0C0C0C43
:10BD400008080808080808080C0C0C0C0C0C0C0C53
:10BD50000C0C0C0C0C0C0C0C0C0C0C0C0C0C0C0C23
:10BD60000C0C0C0C0C0C0C0C0C0C0C0C0C0C0C0C13
:10BD70000C0C0C0C0C0C0C0C0C0C0C0C0C0C0C0C03
:10BD800008080808080808080C0C0C0C0C0C0C0C13
:10BD90000C0C0C0C0C0C0C0C0C0C0C0C0C0C0C0CE3
:10BDA0000C0C0C0C0C0C0C0C0C0C0C0C0C0C0C0CD3
:10BDB0000C0C0C0C0C0C0C0C0C0C0C0C0C0C0C0CC3
:10BDC00008080808080808080C0C0C0C0C0C0C0CD3
:10BDD0000C0C0C0C0C0C0C0C0C0C0C0C0C0C0C0CA3
:10BDE0000C0C0C0C0C0C0C0C0C0C0C0C0C0C0C0C93
:10BDF0000C0C0C0C0C0C0C0C0C0C0C0C0C0C0C0C83
:10BE000008080808080808080C0C0C0C0C0C0C0C92
:10BE10000C0C0C0C0C0C0C0C0C0C0C0C0C0C0C0C62
:10BE20000C0C0C0C0C0C0C0C0C0C0C0C0C0C0C0C52
:10BE30000C0C0C0C0C0C0C0C0C0C0C0C0C0C0C0C42
:10BE400008080808080808080C0C0C0C0C0C0C0C52
:10BE50000C0C0C0C0C0C0C0C0C0C0C0C0C0C0C0C22
:10BE60000C0C0C0C0C0C0C0C0C0C0C0C0C0C0C0C12
:10BE70000C0C0C0C0C0C0C0C0C0C0C0C0C0C0C0C02
:10BE800008080808080808080C0C0C0C0C0C0C0C12
:10BE90000C0C0C0C0C0C0C0C0C0C0C0C0C0C0C0CE2
:10BEA0000C0C0C0C0C0C0C0C0C0C0C0C0C0C0C0CD2
:10BEB0000C0C0C0C0C0C0C0C0C0C0C0C0C0C0C0CC2
:10BEC00008080808080808080C0C0C0C0C0C0C0CD2
:10BED0000C0C0C0C0C0C0C0C0C0C0C0C0C0C0C0CA2
:10BEE0000C0C0C0C0C0C0C0C0C0C0C0C0C0C0C0C92
:10BEF0000C0C0C0C0C0C0C0C0C0C0C0C0C0C0C0C82
:10BF000008080808080808080C0C0C0C0C0C0C0C91
:10BF10000C0C0C0C0C0C0C0C0C0C0C0C0C0C0C0C61
:10BF20000C0C0C0C0C0C0C0C0C0C0C0C0C0C0C0C51
:10BF30000C0C0C0C0C0C0C0C0C0C0C0C0C0C0C0C41
:10BF400008080808080808080C0C0C0C0C0C0C0C51
:10BF50000C0C0C0C0C0C0C0C0C0C0C0C0C0C0C0C21
:10BF60000C0C0C0C0C0C0C0C0C0C0C0C0C0C0C0C11
:10BF70000C0C0C0C0C0C0C0C0C0C0C0C0C0C0C0C01
:10BF800008080808080808080C0C0C0C0C0C0C0C11
:10BF90000C0C0C0C0C0C0C0C0C0C0C0C0C0C0C0CE1
:10BFA0000C0C0C0C0C0C0C0C0C0C0C0C0C0C0C0CD1
:10BFB0000C0C0C0C0C0C0C0C0C0C0C0C0C0C0C0CC1
:10BFC00008080808080808080C0C0C0C0C0C0C0CD1
:10BFD0000C0C0C0C0C0C0C0C0C0C0C0C0C0C0C0CA1
:10BFE0000C0C0C0C0C0C0C0C0C0C0C0C0C0C0C0C91
:10BFF0000C0C0C0C0C0C0C0C0C0C0C0C0C0C0C0C81
:10C0000008080808080808080C0C0C0C0C0C0C0C90
:10C010000C0C0C0C0C0C0C0C0C0C0C0C0C0C0C0C60
:10C020000C0C0C0C0C0C0C0C0C0C0C0C0C0C0C0C50
:10C030000C0C0C0C0C0C0C0C0C0C0C0C0C0C0C0C40
:10C0400008080808080808080C0C0C0C0C0C0C0C50
:10C050000C0C0C0C0C0C0C0C0C0C0C0C0C0C0C0C20
:10C060000C0C0C0C0C0C0C0C0C0C0C0C0C0C0C0C10
:10C070000C0C0C0C0C0C0C0C0C0C0C0C0C0C0C0C00
:10C0800008080808080808080C0C0C0C0C0C0C0C10
:10C090000C0C0C0C0C0C0C0C0C0C0C0C0C0C0C0CE0
:10C0A0000C0C0C0C0C0C0C0C0C0C0C0C0C0C0C0CD0
:10C0B0000C0C0C0C0C0C0C0C0C0C0C0C0C0C0C0CC0
:10C0C00008080808080808080C0C0C0C0C0C0C0CD0
:10C0D0000C0C0C0C0C0C0C0C0C0C0C0C0C0C0C0CA0
:10C0E0000C0C0C0C0C0C0C0C0C0C0C0C0C0C0C0C90
:10C0F0000C0C0C0C0C0C0C0C0C0C0C0C0C0C0C0C80
:10C1000008080808080808080C0C0C0C0C0C0C0C8F
:10C110000C0C0C0C0C0C0C0C0C0C0C0C0C0C0C0C5F
:10C120000C0C0C0C0C0C0C0C0C0C0C0C0C0C0C0C4F
:10C130000C0C0C0C0C0C0C0C0C0C0C0C0C0C0C0C3F
:10C1400008080808080808080C0C0C0C0C0C0C0C4F
:10C150000C0C0C0C0C0C0C0C0C0C0C0C0C0C0C0C1F
:10C160000C0C0C0C0C0C0C0C0C0C0C0C0C0C0C0C0F
:10C170000C0C0C0C0C0C0C0C0C0C0C0C0C0C0C0CFF
:10C1800008080808080808080C0C0C0C0C0C0C0C0F
:10C190000C0C0C0C0C0C0C0C0C0C0C0C0C0C0C0CDF
:10C1A0000C0C0C0C0C0C0C0C0C0C0C0C0C0C0C0CCF
:10C1B0000C0C0C0C0C0C0C0C0C0C0C0C0C0C0C0CBF
:10C1C00008080808080808080C0C0C0C0C0C0C0CCF
:10C1D0000C0C0C0C0C0C0C0C0C0C0C0C0C0C0C0C9F
:10C1E0000C0C0C0C0C0C0C0C0C0C0C0C0C0C0C0C8F
:10C1F0000C0C0C0C0C0C0C0C0C0C0C0C0C0C0C0C7F
:10C2000008080808080808080C0C0C0C0C0C0C0C8E
:10C210000C0C0C0C0C0C0C0C0C0C0C0C0C0C0C0C5E
:10C220000C0C0C0C0C0C0C0C0C0C0C0C0C0C0C0C4E
:10C230000C0C0C0C0C0C0C0C0C0C0C0C0C0C0C0C3E
:10C2400008080808080808080C0C0C0C0C0C0C0C4E
:10C250000C0C0C0C0C0C0C0C0C0C0C0C0C0C0C0C1E
:10C260000C0C0C0C0C0C0C0C0C0C0C0C0C0C0C0C0E
:10C270000C0C0C0C0C0C0C0C0C0C0C0C0C0C0C0CFE
:10C2800008080808080808080C0C0C0C0C0C0C0C0E
:10C290000C0C0C0C0C0C0C0C0C0C0C0C0C0C0C0CDE
:10C2A0000C0C0C0C0C0C0C0C0C0C0C0C0C0C0C0CCE
:10C2B0000C0C0C0C0C0C0C0C0C0C0C0C0C0C0C0CBE
:10C2C00008080808080808080C0C0C0C0C0C0C0CCE
:10C2D0000C0C0C0C0C0C0C0C0C0C0C0C0C0C0C0C9E
:10C2E0000C0C0C0C0C0C0C0C0C0C0C0C0C0C0C0C8E
:10C2F0000C0C0C0C0C0C0C0C0C0C0C0C0C0C0C0C7E
:10C3000008080808080808080C0C0C0C0C0C0C0C8D
:10C310000C0C0C0C0C0C0C0C0C0C0C0C0C0C0C0C5D
:10C320000C0C0C0C0C0C0C0C0C0C0C0C0C0C0C0C4D
:10C330000C0C0C0C0C0C0C0C0C0C0C0C0C0C0C0C3D
:10C3400008080808080808080C0C0C0C0C0C0C0C4D
:10C350000C0C0C0C0C0C0C0C0C0C0C0C0C0C0C0C1D
:10C360000C0C0C0C0C0C0C0C0C0C0C0C0C0C0C0C0D
:10C370000C0C0C0C0C0C0C0C0C0C0C0C0C0C0C0CFD
:10C3800008080808080808080C0C0C0C0C0C0C0C0D
:10C390000C0C0C0C0C0C0C0C0C0C0C0C0C0C0C0CDD
:10C3A0000C0C0C0C0C0C0C0C0C0C0C0C0C0C0C0CCD
:10C3B0000C0C0C0C0C0C0C0C0C0C0C0C0C0C0C0CBD
:10C3C00008080808080808080C0C0C0C0C0C0C0CCD
:10C3D0000C0C0C0C0C0C0C0C0C0C0C0C0C0C0C0C9D
:10C3E0000C0C0C0C0C0C0C0C0C0C0C0C0C0C0C0C8D
:10C3F0000C0C0C0C0C0C0C0C0C0C0C0C0C0C0C0C7D
:10C4000008080808080808080C0C0C0C0C0C0C0C8C
:10C410000C0C0C0C0C0C0C0C0C0C0C0C0C0C0C0C5C
:10C420000C0C0C0C0C0C0C0C0C0C0C0C0C0C0C0C4C
:10C430000C0C0C0C0C0C0C0C0C0C0C0C0C0C0C0C3C
:10C4400008080808080808080C0C0C0C0C0C0C0C4C
:10C450000C0C0C0C0C0C0C0C0C0C0C0C0C0C0C0C1C
:10C460000C0C0C0C0C0C0C0C0C0C0C0C0C0C0C0C0C
:10C470000C0C0C0C0C0C0C0C0C0C0C0C0C0C0C0CFC
:10C4800008080808080808080C0C0C0C0C0C0C0C0C
:10C490000C0C0C0C0C0C0C0C0C0C0C0C0C0C0C0CDC
:10C4A0000C0C0C0C0C0C0C0C0C0C0C0C0C0C0C0CCC
:10C4B0000C0C0C0C0C0C0C0C0C0C0C0C0C0C0C0CBC
:10C4C00008080808080808080C0C0C0C0C0C0C0CCC
:10C4D0000C0C0C0C0C0C0C0C0C0C0C0C0C0C0C0C9C
:10C4E0000C0C0C0C0C0C0C0C0C0C0C0C0C0C0C0C8C
:10C4F0000C0C0C0C0C0C0C0C0C0C0C0C0C0C0C0C7C
:10C5000008080808080808080C0C0C0C0C0C0C0C8B
:10C510000C0C0C0C0C0C0C0C0C0C0C0C0C0C0C0C5B
:10C520000C0C0C0C0C0C0C0C0C0C0C0C0C0C0C0C4B
:10C530000C0C0C0C0C0C0C0C0C0C0C0C0C0C0C0C3B
:10C5400008080808080808080C0C0C0C0C0C0C0C4B
:10C550000C0C0C0C0C0C0C0C0C0C0C0C0C0C0C0C1B
:10C560000C0C0C0C0C0C0C0C0C0C0C0C0C0C0C0C0B
:10C570000C0C0C0C0C0C0C0C0C0C0C0C0C0C0C0CFB
:10C5800008080808080808080C0C0C0C0C0C0C0C0B
:10C590000C0C0C0C0C0C0C0C0C0C0C0C0C0C0C0CDB
:10C5A0000C0C0C0C0C0C0C0C0C0C0C0C0C0C0C0CCB
:10C5B0000C0C0C0C0C0C0C0C0C0C0C0C0C0C0C0CBB
:10C5C00008080808080808080C0C0C0C0C0C0C0CCB
:10C5D0000C0C0C0C0C0C0C0C0C0C0C0C0C0C0C0C9B
:10C5E0000C0C0C0C0C0C0C0C0C0C0C0C0C0C0C0C8B
:10C5F0000C0C0C0C0C0C0C0C0C0C0C0C0C0C0C0C7B
:10C6000008080808080808080C0C0C0C0C0C0C0C8A
:10C610000C0C0C0C0C0C0C0C0C0C0C0C0C0C0C0C5A
:10C620000C0C0C0C0C0C0C0C0C0C0C0C0C0C0C0C4A
:10C630000C0C0C0C0C0C0C0C0C0C0C0C0C0C0C0C3A
:10C6400008080808080808080C0C0C0C0C0C0C0C4A
:10C650000C0C0C0C0C0C0C0C0C0C0C0C0C0C0C0C1A
:10C660000C0C0C0C0C0C0C0C0C0C0C0C0C0C0C0C0A
:10C670000C0C0C0C0C0C0C0C0C0C0C0C0C0C0C0CFA
:10C6800008080808080808080C0C0C0C0C0C0C0C0A
:10C690000C0C0C0C0C0C0C0C0C0C0C0C0C0C0C0CDA
:10C6A0000C0C0C0C0C0C0C0C0C0C0C0C0C0C0C0CCA
:10C6B0000C0C0C0C0C0C0C0C0C0C0C0C0C0C0C0CBA
:10C6C00008080808080808080C0C0C0C0C0C0C0CCA
:10C6D0000C0C0C0C0C0C0C0C0C0C0C0C0C0C0C0C9A
:10C6E0000C0C0C0C0C0C0C0C0C0C0C0C0C0C0C0C8A
:10C6F0000C0C0C0C0C0C0C0C0C0C0C0C0C0C0C0C7A
:10C7000008080808080808080C0C0C0C0C0C0C0C89
:10C710000C0C0C0C0C0C0C0C0C0C0C0C0C0C0C0C59
:10C720000C0C0C0C0C0C0C0C0C0C0C0C0C0C0C0C49
:10C730000C0C0C0C0C0C0C0C0C0C0C0C0C0C0C0C39
:10C7400008080808080808080C0C0C0C0C0C0C0C49
:10C750000C0C0C0C0C0C0C0C0C0C0C0C0C0C0C0C19
:10C760000C0C0C0C0C0C0C0C0C0C0C0C0C0C0C0C09
:10C770000C0C0C0C0C0C0C0C0C0C0C0C0C0C0C0CF9
:10C7800008080808080808080C0C0C0C0C0C0C0C09
:10C790000C0C0C0C0C0C0C0C0C0C0C0C0C0C0C0CD9
:10C7A0000C0C0C0C0C0C0C0C0C0C0C0C0C0C0C0CC9
:10C7B0000C0C0C0C0C0C0C0C0C0C0C0C0C0C0C0CB9
:10C7C00008080808080808080C0C0C0C0C0C0C0CC9
:10C7D0000C0C0C0C0C0C0C0C0C0C0C0C0C0C0C0C99
:10C7E0000C0C0C0C0C0C0C0C0C0C0C0C0C0C0C0C89
:10C7F0000C0C0C0C0C0C0C0C0C0C0C0C0C0C0C0C79
:10C8000008080808080808080C0C0C0C0C0C0C0C88
:10C810000C0C0C0C0C0C0C0C0C0C0C0C0C0C0C0C58
:10C820000C0C0C0C0C0C0C0C0C0C0C0C0C0C0C0C48
:10C830000C0C0C0C0C0C0C0C0C0C0C0C0C0C0C0C38
:10C8400008080808080808080C0C0C0C0C0C0C0C48
:10C850000C0C0C0C0C0C0C0C0C0C0C0C0C0C0C0C18
:10C860000C0C0C0C0C0C0C0C0C0C0C0C0C0C0C0C08
:10C870000C0C0C0C0C0C0C0C0C0C0C0C0C0C0C0CF8
:10C8800008080808080808080C0C0C0C0C0C0C0C08
:10C890000C0C0C0C0C0C0C0C0C0C0C0C0C0C0C0CD8
:10C8A0000C0C0C0C0C0C0C0C0C0C0C0C0C0C0C0CC8
:10C8B0000C0C0C0C0C0C0C0C0C0C0C0C0C0C0C0CB8
:10C8C00008080808080808080C0C0C0C0C0C0C0CC8
:10C8D0000C0C0C0C0C0C0C0C0C0C0C0C0C0C0C0C98
:10C8E0000C0C0C0C0C0C0C0C0C0C0C0C0C0C0C0C88
:10C8F0000C0C0C0C0C0C0C0C0C0C0C0C0C0C0C0C78
:10C9000008080808080808080C0C0C0C0C0C0C0C87
:10C910000C0C0C0C0C0C0C0C0C0C0C0C0C0C0C0C57
:10C920000C0C0C0C0C0C0C0C0C0C0C0C0C0C0C0C47
:10C930000C0C0C0C0C0C0C0C0C0C0C0C0C0C0C0C37
:10C9400008080808080808080C0C0C0C0C0C0C0C47
:10C950000C0C0C0C0C0C0C0C0C0C0C0C0C0C0C0C17
:10C960000C0C0C0C0C0C0C0C0C0C0C0C0C0C0C0C07
:10C970000C0C0C0C0C0C0C0C0C0C0C0C0C0C0C0CF7
:10C9800008080808080808080C0C0C0C0C0C0C0C07
:10C990000C0C0C0C0C0C0C0C0C0C0C0C0C0C0C0CD7
:10C9A0000C0C0C0C0C0C0C0C0C0C0C0C0C0C0C0CC7
:10C9B0000C0C0C0C0C0C0C0C0C0C0C0C0C0C0C0CB7
:10C9C00008080808080808080C0C0C0C0C0C0C0CC7
:10C9D0000C0C0C0C0C0C0C0C0C0C0C0C0C0C0C0C97
:10C9E0000C0C0C0C0C0C0C0C0C0C0C0C0C0C0C0C87
:10C9F0000C0C0C0C0C0C0C0C0C0C0C0C0C0C0C0C77
:10CA000008080808080808080C0C0C0C0C0C0C0C86
:10CA10000C0C0C0C0C0C0C0C0C0C0C0C0C0C0C0C56
:10CA20000C0C0C0C0C0C0C0C0C0C0C0C0C0C0C0C46
:10CA30000C0C0C0C0C0C0C0C0C0C0C0C0C0C0C0C36
:10CA400008080808080808080C0C0C0C0C0C0C0C46
:10CA50000C0C0C0C0C0C0C0C0C0C0C0C0C0C0C0C16
:10CA60000C0C0C0C0C0C0C0C0C0C0C0C0C0C0C0C06
:10CA70000C0C0C0C0C0C0C0C0C0C0C0C0C0C0C0CF6
:10CA800008080808080808080C0C0C0C0C0C0C0C06
:10CA90000C0C0C0C0C0C0C0C0C0C0C0C0C0C0C0CD6
:10CAA0000C0C0C0C0C0C0C0C0C0C0C0C0C0C0C0CC6
:10CAB0000C0C0C0C0C0C0C0C0C0C0C0C0C0C0C0CB6
:10CAC00008080808080808080C0C0C0C0C0C0C0CC6
:10CAD0000C0C0C0C0C0C0C0C0C0C0C0C0C0C0C0C96
:10CAE0000C0C0C0C0C0C0C0C0C0C0C0C0C0C0C0C86
:10CAF0000C0C0C0C0C0C0C0C0C0C0C0C0C0C0C0C76
:10CB000008080808080808080C0C0C0C0C0C0C0C85
:10CB10000C0C0C0C0C0C0C0C0C0C0C0C0C0C0C0C55
:10CB20000C0C0C0C0C0C0C0C0C0C0C0C0C0C0C0C45
:10CB30000C0C0C0C0C0C0C0C0C0C0C0C0C0C0C0C35
:10CB400008080808080808080C0C0C0C0C0C0C0C45
:10CB50000C0C0C0C0C0C0C0C0C0C0C0C0C0C0C0C15
:10CB60000C0C0C0C0C0C0C0C0C0C0C0C0C0C0C0C05
:10CB70000C0C0C0C0C0C0C0C0C0C0C0C0C0C0C0CF5
:10CB800008080808080808080C0C0C0C0C0C0C0C05
:10CB90000C0C0C0C0C0C0C0C0C0C0C0C0C0C0C0CD5
:10CBA0000C0C0C0C0C0C0C0C0C0C0C0C0C0C0C0CC5
:10CBB0000C0C0C0C0C0C0C0C0C0C0C0C0C0C0C0CB5
:10CBC00008080808080808080C0C0C0C0C0C0C0CC5
:10CBD0000C0C0C0C0C0C0C0C0C0C0C0C0C0C0C0C95
:10CBE0000C0C0C0C0C0C0C0C0C0C0C0C0C0C0C0C85
:10CBF0000C0C0C0C0C0C0C0C0C0C0C0C0C0C0C0C75
:10CC000008080808080808080C0C0C0C0C0C0C0C84
:10CC10000C0C0C0C0C0C0C0C0C0C0C0C0C0C0C0C54
:10CC20000C0C0C0C0C0C0C0C0C0C0C0C0C0C0C0C44
:10CC30000C0C0C0C0C0C0C0C0C0C0C0C0C0C0C0C34
:10CC400008080808080808080C0C0C0C0C0C0C0C44
:10CC50000C0C0C0C0C0C0C0C0C0C0C0C0C0C0C0C14
:10CC60000C0C0C0C0C0C0C0C0C0C0C0C0C0C0C0C04
:10CC70000C0C0C0C0C0C0C0C0C0C0C0C0C0C0C0CF4
:10CC800008080808080808080C0C0C0C0C0C0C0C04
:10CC90000C0C0C0C0C0C0C0C0C0C0C0C0C0C0C0CD4
:10CCA0000C0C0C0C0C0C0C0C0C0C0C0C0C0C0C0CC4
:10CCB0000C0C0C0C0C0C0C0C0C0C0C0C0C0C0C0CB4
:10CCC00008080808080808080C0C0C0C0C0C0C0CC4
:10CCD0000C0C0C0C0C0C0C0C0C0C0C0C0C0C0C0C94
:10CCE0000C0C0C0C0C0C0C0C0C0C0C0C0C0C0C0C84
:10CCF0000C0C0C0C0C0C0C0C0C0C0C0C0C0C0C0C74
:10CD000008080808080808080C0C0C0C0C0C0C0C83
:10CD10000C0C0C0C0C0C0C0C0C0C0C0C0C0C0C0C53
:10CD20000C0C0C0C0C0C0C0C0C0C0C0C0C0C0C0C43
:10CD30000C0C0C0C0C0C0C0C0C0C0C0C0C0C0C0C33
:10CD400008080808080808080C0C0C0C0C0C0C0C43
:10CD50000C0C0C0C0C0C0C0C0C0C0C0C0C0C0C0C13
:10CD60000C0C0C0C0C0C0C0C0C0C0C0C0C0C0C0C03
:10CD70000C0C0C0C0C0C0C0C0C0C0C0C0C0C0C0CF3
:10CD800008080808080808080C0C0C0C0C0C0C0C03
:10CD90000C0C0C0C0C0C0C0C0C0C0C0C0C0C0C0CD3
:10CDA0000C0C0C0C0C0C0C0C0C0C0C0C0C0C0C0CC3
:10CDB0000C0C0C0C0C0C0C0C0C0C0C0C0C0C0C0CB3
:10CDC00008080808080808080C0C0C0C0C0C0C0CC3
:10CDD0000C0C0C0C0C0C0C0C0C0C0C0C0C0C0C0C93
:10CDE0000C0C0C0C0C0C0C0C0C0C0C0C0C0C0C0C83
:10CDF0000C0C0C0C0C0C0C0C0C0C0C0C0C0C0C0C73
:10CE000008080808080808080C0C0C0C0C0C0C0C82
:10CE10000C0C0C0C0C0C0C0C0C0C0C0C0C0C0C0C52
:10CE20000C0C0C0C0C0C0C0C0C0C0C0C0C0C0C0C42
:10CE30000C0C0C0C0C0C0C0C0C0C0C0C0C0C0C0C32
:10CE400008080808080808080C0C0C0C0C0C0C0C42
:10CE50000C0C0C0C0C0C0C0C0C0C0C0C0C0C0C0C12
:10CE60000C0C0C0C0C0C0C0C0C0C0C0C0C0C0C0C02
:10CE70000C0C0C0C0C0C0C0C0C0C0C0C0C0C0C0CF2
:10CE800008080808080808080C0C0C0C0C0C0C0C02
:10CE90000C0C0C0C0C0C0C0C0C0C0C0C0C0C0C0CD2
:10CEA0000C0C0C0C0C0C0C0C0C0C0C0C0C0C0C0CC2
:10CEB0000C0C0C0C0C0C0C0C0C0C0C0C0C0C0C0CB2
:10CEC00008080808080808080C0C0C0C0C0C0C0CC2
:10CED0000C0C0C0C0C0C0C0C0C0C0C0C0C0C0C0C92
:10CEE0000C0C0C0C0C0C0C0C0C0C0C0C0C0C0C0C82
:10CEF0000C0C0C0C0C0C0C0C0C0C0C0C0C0C0C0C72
:10CF000008080808080808080C0C0C0C0C0C0C0C81
:10CF10000C0C0C0C0C0C0C0C0C0C0C0C0C0C0C0C51
:10CF20000C0C0C0C0C0C0C0C0C0C0C0C0C0C0C0C41
:10CF30000C0C0C0C0C0C0C0C0C0C0C0C0C0C0C0C31
:10CF400008080808080808080C0C0C0C0C0C0C0C41
:10CF50000C0C0C0C0C0C0C0C0C0C0C0C0C0C0C0C11
:10CF60000C0C0C0C0C0C0C0C0C0C0C0C0C0C0C0C01
:10CF70000C0C0C0C0C0C0C0C0C0C0C0C0C0C0C0CF1
:10CF800008080808080808080C0C0C0C0C0C0C0C01
:10CF90000C0C0C0C0C0C0C0C0C0C0C0C0C0C0C0CD1
:10CFA0000C0C0C0C0C0C0C0C0C0C0C0C0C0C0C0CC1
:10CFB0000C0C0C0C0C0C0C0C0C0C0C0C0C0C0C0CB1
:10CFC00008080808080808080C0C0C0C0C0C0C0CC1
:10CFD0000C0C0C0C0C0C0C0C0C0C0C0C0C0C0C0C91
:10CFE0000C0C0C0C0C0C0C0C0C0C0C0C0C0C0C0C81
:10CFF0000C0C0C0C0C0C0C0C0C0C0C0C0C0C0C0C71
:10D0000008080808080808080C0C0C0C0C0C0C0C80
:10D010000C0C0C0C0C0C0C0C0C0C0C0C0C0C0C0C50
:10D020000C0C0C0C0C0C0C0C0C0C0C0C0C0C0C0C40
:10D030000C0C0C0C0C0C0C0C0C0C0C0C0C0C0C0C30
:10D0400008080808080808080C0C0C0C0C0C0C0C40
:10D050000C0C0C0C0C0C0C0C0C0C0C0C0C0C0C0C10
:10D060000C0C0C0C0C0C0C0C0C0C0C0C0C0C0C0C00
:10D070000C0C0C0C0C0C0C0C0C0C0C0C0C0C0C0CF0
:10D0800008080808080808080C0C0C0C0C0C0C0C00
:10D090000C0C0C0C0C0C0C0C0C0C0C0C0C0C0C0CD0
:10D0A0000C0C0C0C0C0C0C0C0C0C0C0C0C0C0C0CC0
:10D0B0000C0C0C0C0C0C0C0C0C0C0C0C0C0C0C0CB0
:10D0C00008080808080808080C0C0C0C0C0C0C0CC0
:10D0D0000C0C0C0C0C0C0C0C0C0C0C0C0C0C0C0C90
:10D0E0000C0C0C0C0C0C0C0C0C0C0C0C0C0C0C0C80
:10D0F0000C0C0C0C0C0C0C0C0C0C0C0C0C0C0C0C70
:10D1000008080808080808080C0C0C0C0C0C0C0C7F
:10D110000C0C0C0C0C0C0C0C0C0C0C0C0C0C0C0C4F
:10D120000C0C0C0C0C0C0C0C0C0C0C0C0C0C0C0C3F
:10D130000C0C0C0C0C0C0C0C0C0C0C0C0C0C0C0C2F
:10D1400008080808080808080C0C0C0C0C0C0C0C3F
:10D150000C0C0C0C0C0C0C0C0C0C0C0C0C0C0C0C0F
:10D160000C0C0C0C0C0C0C0C0C0C0C0C0C0C0C0CFF
:10D170000C0C0C0C0C0C0C0C0C0C0C0C0C0C0C0CEF
:10D1800008080808080808080C0C0C0C0C0C0C0CFF
:10D190000C0C0C0C0C0C0C0C0C0C0C0C0C0C0C0CCF
:10D1A0000C0C0C0C0C0C0C0C0C0C0C0C0C0C0C0CBF
:10D1B0000C0C0C0C0C0C0C0C0C0C0C0C0C0C0C0CAF
:10D1C00008080808080808080C0C0C0C0C0C0C0CBF
:10D1D0000C0C0C0C0C0C0C0C0C0C0C0C0C0C0C0C8F
:10D1E0000C0C0C0C0C0C0C0C0C0C0C0C0C0C0C0C7F
:10D1F0000C0C0C0C0C0C0C0C0C0C0C0C0C0C0C0C6F
:10D2000008080808080808080C0C0C0C0C0C0C0C7E
:10D210000C0C0C0C0C0C0C0C0C0C0C0C0C0C0C0C4E
:10D220000C0C0C0C0C0C0C0C0C0C0C0C0C0C0C0C3E
:10D230000C0C0C0C0C0C0C0C0C0C0C0C0C0C0C0C2E
:10D2400008080808080808080C0C0C0C0C0C0C0C3E
:10D250000C0C0C0C0C0C0C0C0C0C0C0C0C0C0C0C0E
:10D260000C0C0C0C0C0C0C0C0C0C0C0C0C0C0C0CFE
:10D270000C0C0C0C0C0C0C0C0C0C0C0C0C0C0C0CEE
:10D2800008080808080808080C0C0C0C0C0C0C0CFE
:10D290000C0C0C0C0C0C0C0C0C0C0C0C0C0C0C0CCE
:10D2A0000C0C0C0C0C0C0C0C0C0C0C0C0C0C0C0CBE
:10D2B0000C0C0C0C0C0C0C0C0C0C0C0C0C0C0C0CAE
:10D2C00008080808080808080C0C0C0C0C0C0C0CBE
:10D2D0000C0C0C0C0C0C0C0C0C0C0C0C0C0C0C0C8E
:10D2E0000C0C0C0C0C0C0C0C0C0C0C0C0C0C0C0C7E
:10D2F0000C0C0C0C0C0C0C0C0C0C0C0C0C0C0C0C6E
:10D3000008080808080808080C0C0C0C0C0C0C0C7D
:10D310000C0C0C0C0C0C0C0C0C0C0C0C0C0C0C0C4D
:10D320000C0C0C0C0C0C0C0C0C0C0C0C0C0C0C0C3D
:10D330000C0C0C0C0C0C0C0C0C0C0C0C0C0C0C0C2D
:10D3400008080808080808080C0C0C0C0C0C0C0C3D
:10D350000C0C0C0C0C0C0C0C0C0C0C0C0C0C0C0C0D
:10D360000C0C0C0C0C0C0C0C0C0C0C0C0C0C0C0CFD
:10D370000C0C0C0C0C0C0C0C0C0C0C0C0C0C0C0CED
:10D3800008080808080808080C0C0C0C0C0C0C0CFD
:10D390000C0C0C0C0C0C0C0C0C0C0C0C0C0C0C0CCD
:10D3A0000C0C0C0C0C0C0C0C0C0C0C0C0C0C0C0CBD
:10D3B0000C0C0C0C0C0C0C0C0C0C0C0C0C0C0C0CAD
:10D3C00008080808080808080C0C0C0C0C0C0C0CBD
:10D3D0000C0C0C0C0C0C0C0C0C0C0C0C0C0C0C0C8D
:10D3E0000C0C0C0C0C0C0C0C0C0C0C0C0C0C0C0C7D
:10D3F0000C0C0C0C0C0C0C0C0C0C0C0C0C0C0C0C6D
:10D4000008080808080808080C0C0C0C0C0C0C0C7C
:10D410000C0C0C0C0C0C0C0C0C0C0C0C0C0C0C0C4C
:10D420000C0C0C0C0C0C0C0C0C0C0C0C0C0C0C0C3C
:10D430000C0C0C0C0C0C0C0C0C0C0C0C0C0C0C0C2C
:10D4400008080808080808080C0C0C0C0C0C0C0C3C
:10D450000C0C0C0C0C0C0C0C0C0C0C0C0C0C0C0C0C
:10D460000C0C0C0C0C0C0C0C0C0C0C0C0C0C0C0CFC
:10D470000C0C0C0C0C0C0C0C0C0C0C0C0C0C0C0CEC
:10D4800008080808080808080C0C0C0C0C0C0C0CFC
:10D490000C0C0C0C0C0C0C0C0C0C0C0C0C0C0C0CCC
:10D4A0000C0C0C0C0C0C0C0C0C0C0C0C0C0C0C0CBC
:10D4B0000C0C0C0C0C0C0C0C0C0C0C0C0C0C0C0CAC
:10D4C00008080808080808080C0C0C0C0C0C0C0CBC
:10D4D0000C0C0C0C0C0C0C0C0C0C0C0C0C0C0C0C8C
:10D4E0000C0C0C0C0C0C0C0C0C0C0C0C0C0C0C0C7C
:10D4F0000C0C0C0C0C0C0C0C0C0C0C0C0C0C0C0C6C
:10D5000008080808080808080C0C0C0C0C0C0C0C7B
:10D510000C0C0C0C0C0C0C0C0C0C0C0C0C0C0C0C4B
:10D520000C0C0C0C0C0C0C0C0C0C0C0C0C0C0C0C3B
:10D530000C0C0C0C0C0C0C0C0C0C0C0C0C0C0C0C2B
:10D5400008080808080808080C0C0C0C0C0C0C0C3B
:10D550000C0C0C0C0C0C0C0C0C0C0C0C0C0C0C0C0B
:10D560000C0C0C0C0C0C0C0C0C0C0C0C0C0C0C0CFB
:10D570000C0C0C0C0C0C0C0C0C0C0C0C0C0C0C0CEB
:10D5800008080808080808080C0C0C0C0C0C0C0CFB
:10D590000C0C0C0C0C0C0C0C0C0C0C0C0C0C0C0CCB
:10D5A0000C0C0C0C0C0C0C0C0C0C0C0C0C0C0C0CBB
:10D5B0000C0C0C0C0C0C0C0C0C0C0C0C0C0C0C0CAB
:10D5C00008080808080808080C0C0C0C0C0C0C0CBB
:10D5D0000C0C0C0C0C0C0C0C0C0C0C0C0C0C0C0C8B
:10D5E0000C0C0C0C0C0C0C0C0C0C0C0C0C0C0C0C7B
:10D5F0000C0C0C0C0C0C0C0C0C0C0C0C0C0C0C0C6B
:10D6000008080808080808080C0C0C0C0C0C0C0C7A
:10D610000C0C0C0C0C0C0C0C0C0C0C0C0C0C0C0C4A
:10D620000C0C0C0C0C0C0C0C0C0C0C0C0C0C0C0C3A
:10D630000C0C0C0C0C0C0C0C0C0C0C0C0C0C0C0C2A
:10D6400008080808080808080C0C0C0C0C0C0C0C3A
:10D650000C0C0C0C0C0C0C0C0C0C0C0C0C0C0C0C0A
:10D660000C0C0C0C0C0C0C0C0C0C0C0C0C0C0C0CFA
:10D670000C0C0C0C0C0C0C0C0C0C0C0C0C0C0C0CEA
:10D6800008080808080808080C0C0C0C0C0C0C0CFA
:10D690000C0C0C0C0C0C0C0C0C0C0C0C0C0C0C0CCA
:10D6A0000C0C0C0C0C0C0C0C0C0C0C0C0C0C0C0CBA
:10D6B0000C0C0C0C0C0C0C0C0C0C0C0C0C0C0C0CAA
:10D6C00008080808080808080C0C0C0C0C0C0C0CBA
:10D6D0000C0C0C0C0C0C0C0C0C0C0C0C0C0C0C0C8A
:10D6E0000C0C0C0C0C0C0C0C0C0C0C0C0C0C0C0C7A
:10D6F0000C0C0C0C0C0C0C0C0C0C0C0C0C0C0C0C6A
:10D7000008080808080808080C0C0C0C0C0C0C0C79
:10D710000C0C0C0C0C0C0C0C0C0C0C0C0C0C0C0C49
:10D720000C0C0C0C0C0C0C0C0C0C0C0C0C0C0C0C39
:10D730000C0C0C0C0C0C0C0C0C0C0C0C0C0C0C0C29
:10D7400008080808080808080C0C0C0C0C0C0C0C39
:10D750000C0C0C0C0C0C0C0C0C0C0C0C0C0C0C0C09
:10D760000C0C0C0C0C0C0C0C0C0C0C0C0C0C0C0CF9
:10D770000C0C0C0C0C0C0C0C0C0C0C0C0C0C0C0CE9
:10D7800008080808080808080C0C0C0C0C0C0C0CF9
:10D790000C0C0C0C0C0C0C0C0C0C0C0C0C0C0C0CC9
:10D7A0000C0C0C0C0C0C0C0C0C0C0C0C0C0C0C0CB9
:10D7B0000C0C0C0C0C0C0C0C0C0C0C0C0C0C0C0CA9
:10D7C00008080808080808080C0C0C0C0C0C0C0CB9
:10D7D0000C0C0C0C0C0C0C0C0C0C0C0C0C0C0C0C89
:10D7E0000C0C0C0C0C0C0C0C0C0C0C0C0C0C0C0C79
:10D7F0000C0C0C0C0C0C0C0C0C0C0C0C0C0C0C0C69
:10D8000008080808080808080C0C0C0C0C0C0C0C78
:10D810000C0C0C0C0C0C0C0C0C0C0C0C0C0C0C0C48
:10D820000C0C0C0C0C0C0C0C0C0C0C0C0C0C0C0C38
:10D830000C0C0C0C0C0C0C0C0C0C0C0C0C0C0C0C28
:10D8400008080808080808080C0C0C0C0C0C0C0C38
:10D850000C0C0C0C0C0C0C0C0C0C0C0C0C0C0C0C08
:10D860000C0C0C0C0C0C0C0C0C0C0C0C0C0C0C0CF8
:10D870000C0C0C0C0C0C0C0C0C0C0C0C0C0C0C0CE8
:10D8800008080808080808080C0C0C0C0C0C0C0CF8
:10D890000C0C0C0C0C0C0C0C0C0C0C0C0C0C0C0CC8
:10D8A0000C0C0C0C0C0C0C0C0C0C0C0C0C0C0C0CB8
:10D8B0000C0C0C0C0C0C0C0C0C0C0C0C0C0C0C0CA8
:10D8C00008080808080808080C0C0C0C0C0C0C0CB8
:10D8D0000C0C0C0C0C0C0C0C0C0C0C0C0C0C0C0C88
:10D8E0000C0C0C0C0C0C0C0C0C0C0C0C0C0C0C0C78
:10D8F0000C0C0C0C0C0C0C0C0C0C0C0C0C0C0C0C68
:10D9000008080808080808080C0C0C0C0C0C0C0C77
:10D910000C0C0C0C0C0C0C0C0C0C0C0C0C0C0C0C47
:10D920000C0C0C0C0C0C0C0C0C0C0C0C0C0C0C0C37
:10D930000C0C0C0C0C0C0C0C0C0C0C0C0C0C0C0C27
:10D9400008080808080808080C0C0C0C0C0C0C0C37
:10D950000C0C0C0C0C0C0C0C0C0C0C0C0C0C0C0C07
:10D960000C0C0C0C0C0C0C0C0C0C0C0C0C0C0C0CF7
:10D970000C0C0C0C0C0C0C0C0C0C0C0C0C0C0C0CE7
:10D9800008080808080808080C0C0C0C0C0C0C0CF7
:10D990000C0C0C0C0C0C0C0C0C0C0C0C0C0C0C0CC7
:10D9A0000C0C0C0C0C0C0C0C0C0C0C0C0C0C0C0CB7
:10D9B0000C0C0C0C0C0C0C0C0C0C0C0C0C0C0C0CA7
:10D9C00008080808080808080C0C0C0C0C0C0C0CB7
:10D9D0000C0C0C0C0C0C0C0C0C0C0C0C0C0C0C0C87
:10D9E0000C0C0C0C0C0C0C0C0C0C0C0C0C0C0C0C77
:10D9F0000C0C0C0C0C0C0C0C0C0C0C0C0C0C0C0C67
:10DA000008080808080808080C0C0C0C0C0C0C0C76
:10DA10000C0C0C0C0C0C0C0C0C0C0C0C0C0C0C0C46
:10DA20000C0C0C0C0C0C0C0C0C0C0C0C0C0C0C0C36
:10DA30000C0C0C0C0C0C0C0C0C0C0C0C0C0C0C0C26
:10DA400008080808080808080C0C0C0C0C0C0C0C36
:10DA50000C0C0C0C0C0C0C0C0C0C0C0C0C0C0C0C06
:10DA60000C0C0C0C0C0C0C0C0C0C0C0C0C0C0C0CF6
:10DA70000C0C0C0C0C0C0C0C0C0C0C0C0C0C0C0CE6
:10DA800008080808080808080C0C0C0C0C0C0C0CF6
:10DA90000C0C0C0C0C0C0C0C0C0C0C0C0C0C0C0CC6
:10DAA0000C0C0C0C0C0C0C0C0C0C0C0C0C0C0C0CB6
:10DAB0000C0C0C0C0C0C0C0C0C0C0C0C0C0C0C0CA6
:10DAC00008080808080808080C0C0C0C0C0C0C0CB6
:10DAD0000C0C0C0C0C0C0C0C0C0C0C0C0C0C0C0C86
:10DAE0000C0C0C0C0C0C0C0C0C0C0C0C0C0C0C0C76
:10DAF0000C0C0C0C0C0C0C0C0C0C0C0C0C0C0C0C66
:10DB000008080808080808080C0C0C0C0C0C0C0C75
:10DB10000C0C0C0C0C0C0C0C0C0C0C0C0C0C0C0C45
:10DB20000C0C0C0C0C0C0C0C0C0C0C0C0C0C0C0C35
:10DB30000C0C0C0C0C0C0C0C0C0C0C0C0C0C0C0C25
:10DB400008080808080808080C0C0C0C0C0C0C0C35
:10DB50000C0C0C0C0C0C0C0C0C0C0C0C0C0C0C0C05
:10DB60000C0C0C0C0C0C0C0C0C0C0C0C0C0C0C0CF5
:10DB70000C0C0C0C0C0C0C0C0C0C0C0C0C0C0C0CE5
:10DB800008080808080808080C0C0C0C0C0C0C0CF5
:10DB90000C0C0C0C0C0C0C0C0C0C0C0C0C0C0C0CC5
:10DBA0000C0C0C0C0C0C0C0C0C0C0C0C0C0C0C0CB5
:10DBB0000C0C0C0C0C0C0C0C0C0C0C0C0C0C0C0CA5
:10DBC00008080808080808080C0C0C0C0C0C0C0CB5
:10DBD0000C0C0C0C0C0C0C0C0C0C0C0C0C0C0C0C85
:10DBE0000C0C0C0C0C0C0C0C0C0C0C0C0C0C0C0C75
:10DBF0000C0C0C0C0C0C0C0C0C0C0C0C0C0C0C0C65
:10DC000008080808080808080C0C0C0C0C0C0C0C74
:10DC10000C0C0C0C0C0C0C0C0C0C0C0C0C0C0C0C44
:10DC20000C0C0C0C0C0C0C0C0C0C0C0C0C0C0C0C34
:10DC30000C0C0C0C0C0C0C0C0C0C0C0C0C0C0C0C24
:10DC400008080808080808080C0C0C0C0C0C0C0C34
:10DC50000C0C0C0C0C0C0C0C0C0C0C0C0C0C0C0C04
:10DC60000C0C0C0C0C0C0C0C0C0C0C0C0C0C0C0CF4
:10DC70000C0C0C0C0C0C0C0C0C0C0C0C0C0C0C0CE4
:10DC800008080808080808080C0C0C0C0C0C0C0CF4
:10DC90000C0C0C0C0C0C0C0C0C0C0C0C0C0C0C0CC4
:10DCA0000C0C0C0C0C0C0C0C0C0C0C0C0C0C0C0CB4
:10DCB0000C0C0C0C0C0C0C0C0C0C0C0C0C0C0C0CA4
:10DCC00008080808080808080C0C0C0C0C0C0C0CB4
:10DCD0000C0C0C0C0C0C0C0C0C0C0C0C0C0C0C0C84
:10DCE0000C0C0C0C0C0C0C0C0C0C0C0C0C0C0C0C74
:10DCF0000C0C0C0C0C0C0C0C0C0C0C0C0C0C0C0C64
:10DD000008080808080808080C0C0C0C0C0C0C0C73
:10DD10000C0C0C0C0C0C0C0C0C0C0C0C0C0C0C0C43
:10DD20000C0C0C0C0C0C0C0C0C0C0C0C0C0C0C0C33
:10DD30000C0C0C0C0C0C0C0C0C0C0C0C0C0C0C0C23
:10DD400008080808080808080C0C0C0C0C0C0C0C33
:10DD50000C0C0C0C0C0C0C0C0C0C0C0C0C0C0C0C03
:10DD60000C0C0C0C0C0C0C0C0C0C0C0C0C0C0C0CF3
:10DD70000C0C0C0C0C0C0C0C0C0C0C0C0C0C0C0CE3
:10DD800008080808080808080C0C0C0C0C0C0C0CF3
:10DD90000C0C0C0C0C0C0C0C0C0C0C0C0C0C0C0CC3
:10DDA0000C0C0C0C0C0C0C0C0C0C0C0C0C0C0C0CB3
:10DDB0000C0C0C0C0C0C0C0C0C0C0C0C0C0C0C0CA3
:10DDC00008080808080808080C0C0C0C0C0C0C0CB3
:10DDD0000C0C0C0C0C0C0C0C0C0C0C0C0C0C0C0C83
:10DDE0000C0C0C0C0C0C0C0C0C0C0C0C0C0C0C0C73
:10DDF0000C0C0C0C0C0C0C0C0C0C0C0C0C0C0C0C63
:10DE000008080808080808080C0C0C0C0C0C0C0C72
:10DE10000C0C0C0C0C0C0C0C0C0C0C0C0C0C0C0C42
:10DE20000C0C0C0C0C0C0C0C0C0C0C0C0C0C0C0C32
:10DE30000C0C0C0C0C0C0C0C0C0C0C0C0C0C0C0C22
:10DE400008080808080808080C0C0C0C0C0C0C0C32
:10DE50000C0C0C0C0C0C0C0C0C0C0C0C0C0C0C0C02
:10DE60000C0C0C0C0C0C0C0C0C0C0C0C0C0C0C0CF2
:10DE70000C0C0C0C0C0C0C0C0C0C0C0C0C0C0C0CE2
:10DE800008080808080808080C0C0C0C0C0C0C0CF2
:10DE90000C0C0C0C0C0C0C0C0C0C0C0C0C0C0C0CC2
:10DEA0000C0C0C0C0C0C0C0C0C0C0C0C0C0C0C0CB2
:10DEB0000C0C0C0C0C0C0C0C0C0C0C0C0C0C0C0CA2
:10DEC00008080808080808080C0C0C0C0C0C0C0CB2
:10DED0000C0C0C0C0C0C0C0C0C0C0C0C0C0C0C0C82
:10DEE0000C0C0C0C0C0C0C0C0C0C0C0C0C0C0C0C72
:10DEF0000C0C0C0C0C0C0C0C0C0C0C0C0C0C0C0C62
:10DF000008080808080808080C0C0C0C0C0C0C0C71
:10DF10000C0C0C0C0C0C0C0C0C0C0C0C0C0C0C0C41
:10DF20000C0C0C0C0C0C0C0C0C0C0C0C0C0C0C0C31
:10DF30000C0C0C0C0C0C0C0C0C0C0C0C0C0C0C0C21
:10DF400008080808080808080C0C0C0C0C0C0C0C31
:10DF50000C0C0C0C0C0C0C0C0C0C0C0C0C0C0C0C01
:10DF60000C0C0C0C0C0C0C0C0C0C0C0C0C0C0C0CF1
:10DF70000C0C0C0C0C0C0C0C0C0C0C0C0C0C0C0CE1
:10DF800008080808080808080C0C0C0C0C0C0C0CF1
:10DF90000C0C0C0C0C0C0C0C0C0C0C0C0C0C0C0CC1
:10DFA0000C0C0C0C0C0C0C0C0C0C0C0C0C0C0C0CB1
:10DFB0000C0C0C0C0C0C0C0C0C0C0C0C0C0C0C0CA1
:10DFC00008080808080808080C0C0C0C0C0C0C0CB1
:10DFD0000C0C0C0C0C0C0C0C0C0C0C0C0C0C0C0C81
:10DFE0000C0C0C0C0C0C0C0C0C0C0C0C0C0C0C0C71
:10DFF0000C0C0C0C0C0C0C0C0C0C0C0C0C0C0C0C61
:10E0000008080808080808080C0C0C0C0C0C0C0C70
:10E010000C0C0C0C0C0C0C0C0C0C0C0C0C0C0C0C40
:10E020000C0C0C0C0C0C0C0C0C0C0C0C0C0C0C0C30
:10E030000C0C0C0C0C0C0C0C0C0C0C0C0C0C0C0C20
:10E0400008080808080808080C0C0C0C0C0C0C0C30
:10E050000C0C0C0C0C0C0C0C0C0C0C0C0C0C0C0C00
:10E060000C0C0C0C0C0C0C0C0C0C0C0C0C0C0C0CF0
:10E070000C0C0C0C0C0C0C0C0C0C0C0C0C0C0C0CE0
:10E0800008080808080808080C0C0C0C0C0C0C0CF0
:10E090000C0C0C0C0C0C0C0C0C0C0C0C0C0C0C0CC0
:10E0A0000C0C0C0C0C0C0C0C0C0C0C0C0C0C0C0CB0
:10E0B0000C0C0C0C0C0C0C0C0C0C0C0C0C0C0C0CA0
:10E0C00008080808080808080C0C0C0C0C0C0C0CB0
:10E0D0000C0C0C0C0C0C0C0C0C0C0C0C0C0C0C0C80
:10E0E0000C0C0C0C0C0C0C0C0C0C0C0C0C0C0C0C70
:10E0F0000C0C0C0C0C0C0C0C0C0C0C0C0C0C0C0C60
:10E1000008080808080808080C0C0C0C0C0C0C0C6F
:10E110000C0C0C0C0C0C0C0C0C0C0C0C0C0C0C0C3F
:10E120000C0C0C0C0C0C0C0C0C0C0C0C0C0C0C0C2F
:10E130000C0C0C0C0C0C0C0C0C0C0C0C0C0C0C0C1F
:10E1400008080808080808080C0C0C0C0C0C0C0C2F
:10E150000C0C0C0C0C0C0C0C0C0C0C0C0C0C0C0CFF
:10E160000C0C0C0C0C0C0C0C0C0C0C0C0C0C0C0CEF
:10E170000C0C0C0C0C0C0C0C0C0C0C0C0C0C0C0CDF
:10E1800008080808080808080C0C0C0C0C0C0C0CEF
:10E190000C0C0C0C0C0C0C0C0C0C0C0C0C0C0C0CBF
:10E1A0000C0C0C0C0C0C0C0C0C0C0C0C0C0C0C0CAF
:10E1B0000C0C0C0C0C0C0C0C0C0C0C0C0C0C0C0C9F
:10E1C00008080808080808080C0C0C0C0C0C0C0CAF
:10E1D0000C0C0C0C0C0C0C0C0C0C0C0C0C0C0C0C7F
:10E1E0000C0C0C0C0C0C0C0C0C0C0C0C0C0C0C0C6F
:10E1F0000C0C0C0C0C0C0C0C0C0C0C0C0C0C0C0C5F
:10E2000008080808080808080C0C0C0C0C0C0C0C6E
:10E210000C0C0C0C0C0C0C0C0C0C0C0C0C0C0C0C3E
:10E220000C0C0C0C0C0C0C0C0C0C0C0C0C0C0C0C2E
:10E230000C0C0C0C0C0C0C0C0C0C0C0C0C0C0C0C1E
:10E2400008080808080808080C0C0C0C0C0C0C0C2E
:10E250000C0C0C0C0C0C0C0C0C0C0C0C0C0C0C0CFE
:10E260000C0C0C0C0C0C0C0C0C0C0C0C0C0C0C0CEE
:10E270000C0C0C0C0C0C0C0C0C0C0C0C0C0C0C0CDE
:10E2800008080808080808080C0C0C0C0C0C0C0CEE
:10E290000C0C0C0C0C0C0C0C0C0C0C0C0C0C0C0CBE
:10E2A0000C0C0C0C0C0C0C0C0C0C0C0C0C0C0C0CAE
:10E2B0000C0C0C0C0C0C0C0C0C0C0C0C0C0C0C0C9E
:10E2C00008080808080808080C0C0C0C0C0C0C0CAE
:10E2D0000C0C0C0C0C0C0C0C0C0C0C0C0C0C0C0C7E
:10E2E0000C0C0C0C0C0C0C0C0C0C0C0C0C0C0C0C6E
:10E2F0000C0C0C0C0C0C0C0C0C0C0C0C0C0C0C0C5E
:10E3000008080808080808080C0C0C0C0C0C0C0C6D
:10E310000C0C0C0C0C0C0C0C0C0C0C0C0C0C0C0C3D
:10E320000C0C0C0C0C0C0C0C0C0C0C0C0C0C0C0C2D
:10E330000C0C0C0C0C0C0C0C0C0C0C0C0C0C0C0C1D
:10E3400008080808080808080C0C0C0C0C0C0C0C2D
:10E350000C0C0C0C0C0C0C0C0C0C0C0C0C0C0C0CFD
:10E360000C0C0C0C0C0C0C0C0C0C0C0C0C0C0C0CED
:10E370000C0C0C0C0C0C0C0C0C0C0C0C0C0C0C0CDD
:10E3800008080808080808080C0C0C0C0C0C0C0CED
:10E390000C0C0C0C0C0C0C0C0C0C0C0C0C0C0C0CBD
:10E3A0000C0C0C0C0C0C0C0C0C0C0C0C0C0C0C0CAD
:10E3B0000C0C0C0C0C0C0C0C0C0C0C0C0C0C0C0C9D
:10E3C00008080808080808080C0C0C0C0C0C0C0CAD
:10E3D0000C0C0C0C0C0C0C0C0C0C0C0C0C0C0C0C7D
:10E3E0000C0C0C0C0C0C0C0C0C0C0C0C0C0C0C0C6D
:10E3F0000C0C0C0C0C0C0C0C0C0C0C0C0C0C0C0C5D
:10E4000008080808080808080C0C0C0C0C0C0C0C6C
:10E410000C0C0C0C0C0C0C0C0C0C0C0C0C0C0C0C3C
:10E420000C0C0C0C0C0C0C0C0C0C0C0C0C0C0C0C2C
:10E430000C0C0C0C0C0C0C0C0C0C0C0C0C0C0C0C1C
:10E4400008080808080808080C0C0C0C0C0C0C0C2C
:10E450000C0C0C0C0C0C0C0C0C0C0C0C0C0C0C0CFC
:10E460000C0C0C0C0C0C0C0C0C0C0C0C0C0C0C0CEC
:10E470000C0C0C0C0C0C0C0C0C0C0C0C0C0C0C0CDC
:10E4800008080808080808080C0C0C0C0C0C0C0CEC
:10E490000C0C0C0C0C0C0C0C0C0C0C0C0C0C0C0CBC
:10E4A0000C0C0C0C0C0C0C0C0C0C0C0C0C0C0C0CAC
:10E4B0000C0C0C0C0C0C0C0C0C0C0C0C0C0C0C0C9C
:10E4C00008080808080808080C0C0C0C0C0C0C0CAC
:10E4D0000C0C0C0C0C0C0C0C0C0C0C0C0C0C0C0C7C
:10E4E0000C0C0C0C0C0C0C0C0C0C0C0C0C0C0C0C6C
:10E4F0000C0C0C0C0C0C0C0C0C0C0C0C0C0C0C0C5C
:10E5000008080808080808080C0C0C0C0C0C0C0C6B
:10E510000C0C0C0C0C0C0C0C0C0C0C0C0C0C0C0C3B
:10E520000C0C0C0C0C0C0C0C0C0C0C0C0C0C0C0C2B
:10E530000C0C0C0C0C0C0C0C0C0C0C0C0C0C0C0C1B
:10E5400008080808080808080C0C0C0C0C0C0C0C2B
:10E550000C0C0C0C0C0C0C0C0C0C0C0C0C0C0C0CFB
:10E560000C0C0C0C0C0C0C0C0C0C0C0C0C0C0C0CEB
:10E570000C0C0C0C0C0C0C0C0C0C0C0C0C0C0C0CDB
:10E5800008080808080808080C0C0C0C0C0C0C0CEB
:10E590000C0C0C0C0C0C0C0C0C0C0C0C0C0C0C0CBB
:10E5A0000C0C0C0C0C0C0C0C0C0C0C0C0C0C0C0CAB
:10E5B0000C0C0C0C0C0C0C0C0C0C0C0C0C0C0C0C9B
:10E5C00008080808080808080C0C0C0C0C0C0C0CAB
:10E5D0000C0C0C0C0C0C0C0C0C0C0C0C0C0C0C0C7B
:10E5E0000C0C0C0C0C0C0C0C0C0C0C0C0C0C0C0C6B
:10E5F0000C0C0C0C0C0C0C0C0C0C0C0C0C0C0C0C5B
:10E6000008080808080808080C0C0C0C0C0C0C0C6A
:10E610000C0C0C0C0C0C0C0C0C0C0C0C0C0C0C0C3A
:10E620000C0C0C0C0C0C0C0C0C0C0C0C0C0C0C0C2A
:10E630000C0C0C0C0C0C0C0C0C0C0C0C0C0C0C0C1A
:10E6400008080808080808080C0C0C0C0C0C0C0C2A
:10E650000C0C0C0C0C0C0C0C0C0C0C0C0C0C0C0CFA
:10E660000C0C0C0C0C0C0C0C0C0C0C0C0C0C0C0CEA
:10E670000C0C0C0C0C0C0C0C0C0C0C0C0C0C0C0CDA
:10E6800008080808080808080C0C0C0C0C0C0C0CEA
:10E690000C0C0C0C0C0C0C0C0C0C0C0C0C0C0C0CBA
:10E6A0000C0C0C0C0C0C0C0C0C0C0C0C0C0C0C0CAA
:10E6B0000C0C0C0C0C0C0C0C0C0C0C0C0C0C0C0C9A
:10E6C00008080808080808080C0C0C0C0C0C0C0CAA
:10E6D0000C0C0C0C0C0C0C0C0C0C0C0C0C0C0C0C7A
:10E6E0000C0C0C0C0C0C0C0C0C0C0C0C0C0C0C0C6A
:10E6F0000C0C0C0C0C0C0C0C0C0C0C0C0C0C0C0C5A
:10E7000008080808080808080C0C0C0C0C0C0C0C69
:10E710000C0C0C0C0C0C0C0C0C0C0C0C0C0C0C0C39
:10E720000C0C0C0C0C0C0C0C0C0C0C0C0C0C0C0C29
:10E730000C0C0C0C0C0C0C0C0C0C0C0C0C0C0C0C19
:10E7400008080808080808080C0C0C0C0C0C0C0C29
:10E750000C0C0C0C0C0C0C0C0C0C0C0C0C0C0C0CF9
:10E760000C0C0C0C0C0C0C0C0C0C0C0C0C0C0C0CE9
:10E770000C0C0C0C0C0C0C0C0C0C0C0C0C0C0C0CD9
:10E7800008080808080808080C0C0C0C0C0C0C0CE9
:10E790000C0C0C0C0C0C0C0C0C0C0C0C0C0C0C0CB9
:10E7A0000C0C0C0C0C0C0C0C0C0C0C0C0C0C0C0CA9
:10E7B0000C0C0C0C0C0C0C0C0C0C0C0C0C0C0C0C99
:10E7C00008080808080808080C0C0C0C0C0C0C0CA9
:10E7D0000C0C0C0C0C0C0C0C0C0C0C0C0C0C0C0C79
:10E7E0000C0C0C0C0C0C0C0C0C0C0C0C0C0C0C0C69
:10E7F0000C0C0C0C0C0C0C0C0C0C0C0C0C0C0C0C59
:10E8000008080808080808080C0C0C0C0C0C0C0C68
:10E810000C0C0C0C0C0C0C0C0C0C0C0C0C0C0C0C38
:10E820000C0C0C0C0C0C0C0C0C0C0C0C0C0C0C0C28
:10E830000C0C0C0C0C0C0C0C0C0C0C0C0C0C0C0C18
:10E8400008080808080808080C0C0C0C0C0C0C0C28
:10E850000C0C0C0C0C0C0C0C0C0C0C0C0C0C0C0CF8
:10E860000C0C0C0C0C0C0C0C0C0C0C0C0C0C0C0CE8
:10E870000C0C0C0C0C0C0C0C0C0C0C0C0C0C0C0CD8
:10E8800008080808080808080C0C0C0C0C0C0C0CE8
:10E890000C0C0C0C0C0C0C0C0C0C0C0C0C0C0C0CB8
:10E8A0000C0C0C0C0C0C0C0C0C0C0C0C0C0C0C0CA8
:10E8B0000C0C0C0C0C0C0C0C0C0C0C0C0C0C0C0C98
:10E8C00008080808080808080C0C0C0C0C0C0C0CA8
:10E8D0000C0C0C0C0C0C0C0C0C0C0C0C0C0C0C0C78
:10E8E0000C0C0C0C0C0C0C0C0C0C0C0C0C0C0C0C68
:10E8F0000C0C0C0C0C0C0C0C0C0C0C0C0C0C0C0C58
:10E9000008080808080808080C0C0C0C0C0C0C0C67
:10E910000C0C0C0C0C0C0C0C0C0C0C0C0C0C0C0C37
:10E920000C0C0C0C0C0C0C0C0C0C0C0C0C0C0C0C27
:10E930000C0C0C0C0C0C0C0C0C0C0C0C0C0C0C0C17
:10E9400008080808080808080C0C0C0C0C0C0C0C27
:10E950000C0C0C0C0C0C0C0C0C0C0C0C0C0C0C0CF7
:10E960000C0C0C0C0C0C0C0C0C0C0C0C0C0C0C0CE7
:10E970000C0C0C0C0C0C0C0C0C0C0C0C0C0C0C0CD7
:10E9800008080808080808080C0C0C0C0C0C0C0CE7
:10E990000C0C0C0C0C0C0C0C0C0C0C0C0C0C0C0CB7
:10E9A0000C0C0C0C0C0C0C0C0C0C0C0C0C0C0C0CA7
:10E9B0000C0C0C0C0C0C0C0C0C0C0C0C0C0C0C0C97
:10E9C00008080808080808080C0C0C0C0C0C0C0CA7
:10E9D0000C0C0C0C0C0C0C0C0C0C0C0C0C0C0C0C77
:10E9E0000C0C0C0C0C0C0C0C0C0C0C0C0C0C0C0C67
:10E9F0000C0C0C0C0C0C0C0C0C0C0C0C0C0C0C0C57
:10EA000008080808080808080C0C0C0C0C0C0C0C66
:10EA10000C0C0C0C0C0C0C0C0C0C0C0C0C0C0C0C36
:10EA20000C0C0C0C0C0C0C0C0C0C0C0C0C0C0C0C26
:10EA30000C0C0C0C0C0C0C0C0C0C0C0C0C0C0C0C16
:10EA400008080808080808080C0C0C0C0C0C0C0C26
:10EA50000C0C0C0C0C0C0C0C0C0C0C0C0C0C0C0CF6
:10EA60000C0C0C0C0C0C0C0C0C0C0C0C0C0C0C0CE6
:10EA70000C0C0C0C0C0C0C0C0C0C0C0C0C0C0C0CD6
:10EA800008080808080808080C0C0C0C0C0C0C0CE6
:10EA90000C0C0C0C0C0C0C0C0C0C0C0C0C0C0C0CB6
:10EAA0000C0C0C0C0C0C0C0C0C0C0C0C0C0C0C0CA6
:10EAB0000C0C0C0C0C0C0C0C0C0C0C0C0C0C0C0C96
:10EAC00008080808080808080C0C0C0C0C0C0C0CA6
:10EAD0000C0C0C0C0C0C0C0C0C0C0C0C0C0C0C0C76
:10EAE0000C0C0C0C0C0C0C0C0C0C0C0C0C0C0C0C66
:10EAF0000C0C0C0C0C0C0C0C0C0C0C0C0C0C0C0C56
:10EB000008080808080808080C0C0C0C0C0C0C0C65
:10EB10000C0C0C0C0C0C0C0C0C0C0C0C0C0C0C0C35
:10EB20000C0C0C0C0C0C0C0C0C0C0C0C0C0C0C0C25
:10EB30000C0C0C0C0C0C0C0C0C0C0C0C0C0C0C0C15
:10EB400008080808080808080C0C0C0C0C0C0C0C25
:10EB50000C0C0C0C0C0C0C0C0C0C0C0C0C0C0C0CF5
:10EB60000C0C0C0C0C0C0C0C0C0C0C0C0C0C0C0CE5
:10EB70000C0C0C0C0C0C0C0C0C0C0C0C0C0C0C0CD5
:10EB800008080808080808080C0C0C0C0C0C0C0CE5
:10EB90000C0C0C0C0C0C0C0C0C0C0C0C0C0C0C0CB5
:10EBA0000C0C0C0C0C0C0C0C0C0C0C0C0C0C0C0CA5
:10EBB0000C0C0C0C0C0C0C0C0C0C0C0C0C0C0C0C95
:10EBC00008080808080808080C0C0C0C0C0C0C0CA5
:10EBD0000C0C0C0C0C0C0C0C0C0C0C0C0C0C0C0C75
:10EBE0000C0C0C0C0C0C0C0C0C0C0C0C0C0C0C0C65
:10EBF0000C0C0C0C0C0C0C0C0C0C0C0C0C0C0C0C55
:10EC000008080808080808080C0C0C0C0C0C0C0C64
:10EC10000C0C0C0C0C0C0C0C0C0C0C0C0C0C0C0C34
:10EC20000C0C0C0C0C0C0C0C0C0C0C0C0C0C0C0C24
:10EC30000C0C0C0C0C0C0C0C0C0C0C0C0C0C0C0C14
:10EC400008080808080808080C0C0C0C0C0C0C0C24
:10EC50000C0C0C0C0C0C0C0C0C0C0C0C0C0C0C0CF4
:10EC60000C0C0C0C0C0C0C0C0C0C0C0C0C0C0C0CE4
:10EC70000C0C0C0C0C0C0C0C0C0C0C0C0C0C0C0CD4
:10EC800008080808080808080C0C0C0C0C0C0C0CE4
:10EC90000C0C0C0C0C0C0C0C0C0C0C0C0C0C0C0CB4
:10ECA0000C0C0C0C0C0C0C0C0C0C0C0C0C0C0C0CA4
:10ECB0000C0C0C0C0C0C0C0C0C0C0C0C0C0C0C0C94
:10ECC00008080808080808080C0C0C0C0C0C0C0CA4
:10ECD0000C0C0C0C0C0C0C0C0C0C0C0C0C0C0C0C74
:10ECE0000C0C0C0C0C0C0C0C0C0C0C0C0C0C0C0C64
:10ECF0000C0C0C0C0C0C0C0C0C0C0C0C0C0C0C0C54
:10ED000008080808080808080C0C0C0C0C0C0C0C63
:10ED10000C0C0C0C0C0C0C0C0C0C0C0C0C0C0C0C33
:10ED20000C0C0C0C0C0C0C0C0C0C0C0C0C0C0C0C23
:10ED30000C0C0C0C0C0C0C0C0C0C0C0C0C0C0C0C13
:10ED400008080808080808080C0C0C0C0C0C0C0C23
:10ED50000C0C0C0C0C0C0C0C0C0C0C0C0C0C0C0CF3
:10ED60000C0C0C0C0C0C0C0C0C0C0C0C0C0C0C0CE3
:10ED70000C0C0C0C0C0C0C0C0C0C0C0C0C0C0C0CD3
:10ED800008080808080808080C0C0C0C0C0C0C0CE3
:10ED90000C0C0C0C0C0C0C0C0C0C0C0C0C0C0C0CB3
:10EDA0000C0C0C0C0C0C0C0C0C0C0C0C0C0C0C0CA3
:10EDB0000C0C0C0C0C0C0C0C0C0C0C0C0C0C0C0C93
:10EDC00008080808080808080C0C0C0C0C0C0C0CA3
:10EDD0000C0C0C0C0C0C0C0C0C0C0C0C0C0C0C0C73
:10EDE0000C0C0C0C0C0C0C0C0C0C0C0C0C0C0C0C63
:10EDF0000C0C0C0C0C0C0C0C0C0C0C0C0C0C0C0C53
:10EE000008080808080808080C0C0C0C0C0C0C0C62
:10EE10000C0C0C0C0C0C0C0C0C0C0C0C0C0C0C0C32
:10EE20000C0C0C0C0C0C0C0C0C0C0C0C0C0C0C0C22
:10EE30000C0C0C0C0C0C0C0C0C0C0C0C0C0C0C0C12
:10EE400008080808080808080C0C0C0C0C0C0C0C22
:10EE50000C0C0C0C0C0C0C0C0C0C0C0C0C0C0C0CF2
:10EE60000C0C0C0C0C0C0C0C0C0C0C0C0C0C0C0CE2
:10EE70000C0C0C0C0C0C0C0C0C0C0C0C0C0C0C0CD2
:10EE800008080808080808080C0C0C0C0C0C0C0CE2
:10EE90000C0C0C0C0C0C0C0C0C0C0C0C0C0C0C0CB2
:10EEA0000C0C0C0C0C0C0C0C0C0C0C0C0C0C0C0CA2
:10EEB0000C0C0C0C0C0C0C0C0C0C0C0C0C0C0C0C92
:10EEC00008080808080808080C0C0C0C0C0C0C0CA2
:10EED0000C0C0C0C0C0C0C0C0C0C0C0C0C0C0C0C72
:10EEE0000C0C0C0C0C0C0C0C0C0C0C0C0C0C0C0C62
:10EEF0000C0C0C0C0C0C0C0C0C0C0C0C0C0C0C0C52
:10EF000008080808080808080C0C0C0C0C0C0C0C61
:10EF10000C0C0C0C0C0C0C0C0C0C0C0C0C0C0C0C31
:10EF20000C0C0C0C0C0C0C0C0C0C0C0C0C0C0C0C21
:10EF30000C0C0C0C0C0C0C0C0C0C0C0C0C0C0C0C11
:10EF400008080808080808080C0C0C0C0C0C0C0C21
:10EF50000C0C0C0C0C0C0C0C0C0C0C0C0C0C0C0CF1
:10EF60000C0C0C0C0C0C0C0C0C0C0C0C0C0C0C0CE1
:10EF70000C0C0C0C0C0C0C0C0C0C0C0C0C0C0C0CD1
:10EF800008080808080808080C0C0C0C0C0C0C0CE1
:10EF90000C0C0C0C0C0C0C0C0C0C0C0C0C0C0C0CB1
:10EFA0000C0C0C0C0C0C0C0C0C0C0C0C0C0C0C0CA1
:10EFB0000C0C0C0C0C0C0C0C0C0C0C0C0C0C0C0C91
:10EFC00008080808080808080C0C0C0C0C0C0C0CA1
:10EFD0000C0C0C0C0C0C0C0C0C0C0C0C0C0C0C0C71
:10EFE0000C0C0C0C0C0C0C0C0C0C0C0C0C0C0C0C61
:10EFF0000C0C0C0C0C0C0C0C0C0C0C0C0C0C0C0C51
:10F0000008080808080808080C0C0C0C0C0C0C0C60
:10F010000C0C0C0C0C0C0C0C0C0C0C0C0C0C0C0C30
:10F020000C0C0C0C0C0C0C0C0C0C0C0C0C0C0C0C20
:10F030000C0C0C0C0C0C0C0C0C0C0C0C0C0C0C0C10
:10F0400008080808080808080C0C0C0C0C0C0C0C20
:10F050000C0C0C0C0C0C0C0C0C0C0C0C0C0C0C0CF0
:10F060000C0C0C0C0C0C0C0C0C0C0C0C0C0C0C0CE0
:10F070000C0C0C0C0C0C0C0C0C0C0C0C0C0C0C0CD0
:10F0800008080808080808080C0C0C0C0C0C0C0CE0
:10F090000C0C0C0C0C0C0C0C0C0C0C0C0C0C0C0CB0
:10F0A0000C0C0C0C0C0C0C0C0C0C0C0C0C0C0C0CA0
:10F0B0000C0C0C0C0C0C0C0C0C0C0C0C0C0C0C0C90
:10F0C00008080808080808080C0C0C0C0C0C0C0CA0
:10F0D0000C0C0C0C0C0C0C0C0C0C0C0C0C0C0C0C70
:10F0E0000C0C0C0C0C0C0C0C0C0C0C0C0C0C0C0C60
:10F0F0000C0C0C0C0C0C0C0C0C0C0C0C0C0C0C0C50
:10F1000008080808080808080C0C0C0C0C0C0C0C5F
:10F110000C0C0C0C0C0C0C0C0C0C0C0C0C0C0C0C2F
:10F120000C0C0C0C0C0C0C0C0C0C0C0C0C0C0C0C1F
:10F130000C0C0C0C0C0C0C0C0C0C0C0C0C0C0C0C0F
:10F1400008080808080808080C0C0C0C0C0C0C0C1F
:10F150000C0C0C0C0C0C0C0C0C0C0C0C0C0C0C0CEF
:10F160000C0C0C0C0C0C0C0C0C0C0C0C0C0C0C0CDF
:10F170000C0C0C0C0C0C0C0C0C0C0C0C0C0C0C0CCF
:10F1800008080808080808080C0C0C0C0C0C0C0CDF
:10F190000C0C0C0C0C0C0C0C0C0C0C0C0C0C0C0CAF
:10F1A0000C0C0C0C0C0C0C0C0C0C0C0C0C0C0C0C9F
:10F1B0000C0C0C0C0C0C0C0C0C0C0C0C0C0C0C0C8F
:10F1C00008080808080808080C0C0C0C0C0C0C0C9F
:10F1D0000C0C0C0C0C0C0C0C0C0C0C0C0C0C0C0C6F
:10F1E0000C0C0C0C0C0C0C0C0C0C0C0C0C0C0C0C5F
:10F1F0000C0C0C0C0C0C0C0C0C0C0C0C0C0C0C0C4F
:10F2000008080808080808080C0C0C0C0C0C0C0C5E
:10F210000C0C0C0C0C0C0C0C0C0C0C0C0C0C0C0C2E
:10F220000C0C0C0C0C0C0C0C0C0C0C0C0C0C0C0C1E
:10F230000C0C0C0C0C0C0C0C0C0C0C0C0C0C0C0C0E
:10F2400008080808080808080C0C0C0C0C0C0C0C1E
:10F250000C0C0C0C0C0C0C0C0C0C0C0C0C0C0C0CEE
:10F260000C0C0C0C0C0C0C0C0C0C0C0C0C0C0C0CDE
:10F270000C0C0C0C0C0C0C0C0C0C0C0C0C0C0C0CCE
:10F2800008080808080808080C0C0C0C0C0C0C0CDE
:10F290000C0C0C0C0C0C0C0C0C0C0C0C0C0C0C0CAE
:10F2A0000C0C0C0C0C0C0C0C0C0C0C0C0C0C0C0C9E
:10F2B0000C0C0C0C0C0C0C0C0C0C0C0C0C0C0C0C8E
:10F2C00008080808080808080C0C0C0C0C0C0C0C9E
:10F2D0000C0C0C0C0C0C0C0C0C0C0C0C0C0C0C0C6E
:10F2E0000C0C0C0C0C0C0C0C0C0C0C0C0C0C0C0C5E
:10F2F0000C0C0C0C0C0C0C0C0C0C0C0C0C0C0C0C4E
:10F3000008080808080808080C0C0C0C0C0C0C0C5D
:10F310000C0C0C0C0C0C0C0C0C0C0C0C0C0C0C0C2D
:10F320000C0C0C0C0C0C0C0C0C0C0C0C0C0C0C0C1D
:10F330000C0C0C0C0C0C0C0C0C0C0C0C0C0C0C0C0D
:10F3400008080808080808080C0C0C0C0C0C0C0C1D
:10F350000C0C0C0C0C0C0C0C0C0C0C0C0C0C0C0CED
:10F360000C0C0C0C0C0C0C0C0C0C0C0C0C0C0C0CDD
:10F370000C0C0C0C0C0C0C0C0C0C0C0C0C0C0C0CCD
:10F3800008080808080808080C0C0C0C0C0C0C0CDD
:10F390000C0C0C0C0C0C0C0C0C0C0C0C0C0C0C0CAD
:10F3A0000C0C0C0C0C0C0C0C0C0C0C0C0C0C0C0C9D
:10F3B0000C0C0C0C0C0C0C0C0C0C0C0C0C0C0C0C8D
:10F3C00008080808080808080C0C0C0C0C0C0C0C9D
:10F3D0000C0C0C0C0C0C0C0C0C0C0C0C0C0C0C0C6D
:10F3E0000C0C0C0C0C0C0C0C0C0C0C0C0C0C0C0C5D
:10F3F0000C0C0C0C0C0C0C0C0C0C0C0C0C0C0C0C4D
:10F4000008080808080808080C0C0C0C0C0C0C0C5C
:10F410000C0C0C0C0C0C0C0C0C0C0C0C0C0C0C0C2C
:10F420000C0C0C0C0C0C0C0C0C0C0C0C0C0C0C0C1C
:10F430000C0C0C0C0C0C0C0C0C0C0C0C0C0C0C0C0C
:10F4400008080808080808080C0C0C0C0C0C0C0C1C
:10F450000C0C0C0C0C0C0C0C0C0C0C0C0C0C0C0CEC
:10F460000C0C0C0C0C0C0C0C0C0C0C0C0C0C0C0CDC
:10F470000C0C0C0C0C0C0C0C0C0C0C0C0C0C0C0CCC
:10F4800008080808080808080C0C0C0C0C0C0C0CDC
:10F490000C0C0C0C0C0C0C0C0C0C0C0C0C0C0C0CAC
:10F4A0000C0C0C0C0C0C0C0C0C0C0C0C0C0C0C0C9C
:10F4B0000C0C0C0C0C0C0C0C0C0C0C0C0C0C0C0C8C
:10F4C00008080808080808080C0C0C0C0C0C0C0C9C
:10F4D0000C0C0C0C0C0C0C0C0C0C0C0C0C0C0C0C6C
:10F4E0000C0C0C0C0C0C0C0C0C0C0C0C0C0C0C0C5C
:10F4F0000C0C0C0C0C0C0C0C0C0C0C0C0C0C0C0C4C
:10F5000008080808080808080C0C0C0C0C0C0C0C5B
:10F510000C0C0C0C0C0C0C0C0C0C0C0C0C0C0C0C2B
:10F520000C0C0C0C0C0C0C0C0C0C0C0C0C0C0C0C1B
:10F530000C0C0C0C0C0C0C0C0C0C0C0C0C0C0C0C0B
:10F5400008080808080808080C0C0C0C0C0C0C0C1B
:10F550000C0C0C0C0C0C0C0C0C0C0C0C0C0C0C0CEB
:10F560000C0C0C0C0C0C0C0C0C0C0C0C0C0C0C0CDB
:10F570000C0C0C0C0C0C0C0C0C0C0C0C0C0C0C0CCB
:10F5800008080808080808080C0C0C0C0C0C0C0CDB
:10F590000C0C0C0C0C0C0C0C0C0C0C0C0C0C0C0CAB
:10F5A0000C0C0C0C0C0C0C0C0C0C0C0C0C0C0C0C9B
:10F5B0000C0C0C0C0C0C0C0C0C0C0C0C0C0C0C0C8B
:10F5C00008080808080808080C0C0C0C0C0C0C0C9B
:10F5D0000C0C0C0C0C0C0C0C0C0C0C0C0C0C0C0C6B
:10F5E0000C0C0C0C0C0C0C0C0C0C0C0C0C0C0C0C5B
:10F5F0000C0C0C0C0C0C0C0C0C0C0C0C0C0C0C0C4B
:10F6000008080808080808080C0C0C0C0C0C0C0C5A
:10F610000C0C0C0C0C0C0C0C0C0C0C0C0C0C0C0C2A
:10F620000C0C0C0C0C0C0C0C0C0C0C0C0C0C0C0C1A
:10F630000C0C0C0C0C0C0C0C0C0C0C0C0C0C0C0C0A
:10F6400008080808080808080C0C0C0C0C0C0C0C1A
:10F650000C0C0C0C0C0C0C0C0C0C0C0C0C0C0C0CEA
:10F660000C0C0C0C0C0C0C0C0C0C0C0C0C0C0C0CDA
:10F670000C0C0C0C0C0C0C0C0C0C0C0C0C0C0C0CCA
:10F6800008080808080808080C0C0C0C0C0C0C0CDA
:10F690000C0C0C0C0C0C0C0C0C0C0C0C0C0C0C0CAA
:10F6A0000C0C0C0C0C0C0C0C0C0C0C0C0C0C0C0C9A
:10F6B0000C0C0C0C0C0C0C0C0C0C0C0C0C0C0C0C8A
:10F6C00008080808080808080C0C0C0C0C0C0C0C9A
:10F6D0000C0C0C0C0C0C0C0C0C0C0C0C0C0C0C0C6A
:10F6E0000C0C0C0C0C0C0C0C0C0C0C0C0C0C0C0C5A
:10F6F0000C0C0C0C0C0C0C0C0C0C0C0C0C0C0C0C4A
:10F7000008080808080808080C0C0C0C0C0C0C0C59
:10F710000C0C0C0C0C0C0C0C0C0C0C0C0C0C0C0C29
:10F720000C0C0C0C0C0C0C0C0C0C0C0C0C0C0C0C19
:10F730000C0C0C0C0C0C0C0C0C0C0C0C0C0C0C0C09
:10F7400008080808080808080C0C0C0C0C0C0C0C19
:10F750000C0C0C0C0C0C0C0C0C0C0C0C0C0C0C0CE9
:10F760000C0C0C0C0C0C0C0C0C0C0C0C0C0C0C0CD9
:10F770000C0C0C0C0C0C0C0C0C0C0C0C0C0C0C0CC9
:10F7800008080808080808080C0C0C0C0C0C0C0CD9
:10F790000C0C0C0C0C0C0C0C0C0C0C0C0C0C0C0CA9
:10F7A0000C0C0C0C0C0C0C0C0C0C0C0C0C0C0C0C99
:10F7B0000C0C0C0C0C0C0C0C0C0C0C0C0C0C0C0C89
:10F7C00008080808080808080C0C0C0C0C0C0C0C99
:10F7D0000C0C0C0C0C0C0C0C0C0C0C0C0C0C0C0C69
:10F7E0000C0C0C0C0C0C0C0C0C0C0C0C0C0C0C0C59
:10F7F0000C0C0C0C0C0C0C0C0C0C0C0C0C0C0C0C49
:10F8000008080808080808080C0C0C0C0C0C0C0C58
:10F810000C0C0C0C0C0C0C0C0C0C0C0C0C0C0C0C28
:10F820000C0C0C0C0C0C0C0C0C0C0C0C0C0C0C0C18
:10F830000C0C0C0C0C0C0C0C0C0C0C0C0C0C0C0C08
:10F8400008080808080808080C0C0C0C0C0C0C0C18
:10F850000C0C0C0C0C0C0C0C0C0C0C0C0C0C0C0CE8
:10F860000C0C0C0C0C0C0C0C0C0C0C0C0C0C0C0CD8
:10F870000C0C0C0C0C0C0C0C0C0C0C0C0C0C0C0CC8
:10F8800008080808080808080C0C0C0C0C0C0C0CD8
:10F890000C0C0C0C0C0C0C0C0C0C0C0C0C0C0C0CA8
:10F8A0000C0C0C0C0C0C0C0C0C0C0C0C0C0C0C0C98
:10F8B0000C0C0C0C0C0C0C0C0C0C0C0C0C0C0C0C88
:10F8C00008080808080808080C0C0C0C0C0C0C0C98
:10F8D0000C0C0C0C0C0C0C0C0C0C0C0C0C0C0C0C68
:10F8E0000C0C0C0C0C0C0C0C0C0C0C0C0C0C0C0C58
:10F8F0000C0C0C0C0C0C0C0C0C0C0C0C0C0C0C0C48
:10F9000008080808080808080C0C0C0C0C0C0C0C57
:10F910000C0C0C0C0C0C0C0C0C0C0C0C0C0C0C0C27
:10F920000C0C0C0C0C0C0C0C0C0C0C0C0C0C0C0C17
:10F930000C0C0C0C0C0C0C0C0C0C0C0C0C0C0C0C07
:10F9400008080808080808080C0C0C0C0C0C0C0C17
:10F950000C0C0C0C0C0C0C0C0C0C0C0C0C0C0C0CE7
:10F960000C0C0C0C0C0C0C0C0C0C0C0C0C0C0C0CD7
:10F970000C0C0C0C0C0C0C0C0C0C0C0C0C0C0C0CC7
:10F9800008080808080808080C0C0C0C0C0C0C0CD7
:10F990000C0C0C0C0C0C0C0C0C0C0C0C0C0C0C0CA7
:10F9A0000C0C0C0C0C0C0C0C0C0C0C0C0C0C0C0C97
:10F9B0000C0C0C0C0C0C0C0C0C0C0C0C0C0C0C0C87
:10F9C00008080808080808080C0C0C0C0C0C0C0C97
:10F9D0000C0C0C0C0C0C0C0C0C0C0C0C0C0C0C0C67
:10F9E0000C0C0C0C0C0C0C0C0C0C0C0C0C0C0C0C57
:10F9F0000C0C0C0C0C0C0C0C0C0C0C0C0C0C0C0C47
:10FA000008080808080808080C0C0C0C0C0C0C0C56
:10FA10000C0C0C0C0C0C0C0C0C0C0C0C0C0C0C0C26
:10FA20000C0C0C0C0C0C0C0C0C0C0C0C0C0C0C0C16
:10FA30000C0C0C0C0C0C0C0C0C0C0C0C0C0C0C0C06
:10FA400008080808080808080C0C0C0C0C0C0C0C16
:10FA50000C0C0C0C0C0C0C0C0C0C0C0C0C0C0C0CE6
:10FA60000C0C0C0C0C0C0C0C0C0C0C0C0C0C0C0CD6
:10FA70000C0C0C0C0C0C0C0C0C0C0C0C0C0C0C0CC6
:10FA800008080808080808080C0C0C0C0C0C0C0CD6
:10FA90000C0C0C0C0C0C0C0C0C0C0C0C0C0C0C0CA6
:10FAA0000C0C0C0C0C0C0C0C0C0C0C0C0C0C0C0C96
:10FAB0000C0C0C0C0C0C0C0C0C0C0C0C0C0C0C0C86
:10FAC00008080808080808080C0C0C0C0C0C0C0C96
:10FAD0000C0C0C0C0C0C0C0C0C0C0C0C0C0C0C0C66
:10FAE0000C0C0C0C0C0C0C0C0C0C0C0C0C0C0C0C56
:10FAF0000C0C0C0C0C0C0C0C0C0C0C0C0C0C0C0C46
:10FB000008080808080808080C0C0C0C0C0C0C0C55
:10FB10000C0C0C0C0C0C0C0C0C0C0C0C0C0C0C0C25
:10FB20000C0C0C0C0C0C0C0C0C0C0C0C0C0C0C0C15
:10FB30000C0C0C0C0C0C0C0C0C0C0C0C0C0C0C0C05
:10FB400008080808080808080C0C0C0C0C0C0C0C15
:10FB50000C0C0C0C0C0C0C0C0C0C0C0C0C0C0C0CE5
:10FB60000C0C0C0C0C0C0C0C0C0C0C0C0C0C0C0CD5
:10FB70000C0C0C0C0C0C0C0C0C0C0C0C0C0C0C0CC5
:10FB800008080808080808080C0C0C0C0C0C0C0CD5
:10FB90000C0C0C0C0C0C0C0C0C0C0C0C0C0C0C0CA5
:10FBA0000C0C0C0C0C0C0C0C0C0C0C0C0C0C0C0C95
:10FBB0000C0C0C0C0C0C0C0C0C0C0C0C0C0C0C0C85
:10FBC00008080808080808080C0C0C0C0C0C0C0C95
:10FBD0000C0C0C0C0C0C0C0C0C0C0C0C0C0C0C0C65
:10FBE0000C0C0C0C0C0C0C0C0C0C0C0C0C0C0C0C55
:10FBF0000C0C0C0C0C0C0C0C0C0C0C0C0C0C0C0C45
:10FC000008080808080808080C0C0C0C0C0C0C0C54
:10FC10000C0C0C0C0C0C0C0C0C0C0C0C0C0C0C0C24
:10FC20000C0C0C0C0C0C0C0C0C0C0C0C0C0C0C0C14
:10FC30000C0C0C0C0C0C0C0C0C0C0C0C0C0C0C0C04
:10FC400008080808080808080C0C0C0C0C0C0C0C14
:10FC50000C0C0C0C0C0C0C0C0C0C0C0C0C0C0C0CE4
:10FC60000C0C0C0C0C0C0C0C0C0C0C0C0C0C0C0CD4
:10FC70000C0C0C0C0C0C0C0C0C0C0C0C0C0C0C0CC4
:10FC800008080808080808080C0C0C0C0C0C0C0CD4
:10FC90000C0C0C0C0C0C0C0C0C0C0C0C0C0C0C0CA4
:10FCA0000C0C0C0C0C0C0C0C0C0C0C0C0C0C0C0C94
:10FCB0000C0C0C0C0C0C0C0C0C0C0C0C0C0C0C0C84
:10FCC00008080808080808080C0C0C0C0C0C0C0C94
:10FCD0000C0C0C0C0C0C0C0C0C0C0C0C0C0C0C0C64
:10FCE0000C0C0C0C0C0C0C0C0C0C0C0C0C0C0C0C54
:10FCF0000C0C0C0C0C0C0C0C0C0C0C0C0C0C0C0C44
:10FD000008080808080808080C0C0C0C0C0C0C0C53
:10FD10000C0C0C0C0C0C0C0C0C0C0C0C0C0C0C0C23
:10FD20000C0C0C0C0C0C0C0C0C0C0C0C0C0C0C0C13
:10FD30000C0C0C0C0C0C0C0C0C0C0C0C0C0C0C0C03
:10FD400008080808080808080C0C0C0C0C0C0C0C13
:10FD50000C0C0C0C0C0C0C0C0C0C0C0C0C0C0C0CE3
:10FD60000C0C0C0C0C0C0C0C0C0C0C0C0C0C0C0CD3
:10FD70000C0C0C0C0C0C0C0C0C0C0C0C0C0C0C0CC3
:10FD800008080808080808080C0C0C0C0C0C0C0CD3
:10FD90000C0C0C0C0C0C0C0C0C0C0C0C0C0C0C0CA3
:10FDA0000C0C0C0C0C0C0C0C0C0C0C0C0C0C0C0C93
:10FDB0000C0C0C0C0C0C0C0C0C0C0C0C0C0C0C0C83
:10FDC00008080808080808080C0C0C0C0C0C0C0C93
:10FDD0000C0C0C0C0C0C0C0C0C0C0C0C0C0C0C0C63
:10FDE0000C0C0C0C0C0C0C0C0C0C0C0C0C0C0C0C53
:10FDF0000C0C0C0C0C0C0C0C0C0C0C0C0C0C0C0C43
:10FE000008080808080808080C0C0C0C0C0C0C0C52
:10FE10000C0C0C0C0C0C0C0C0C0C0C0C0C0C0C0C22
:10FE20000C0C0C0C0C0C0C0C0C0C0C0C0C0C0C0C12
:10FE30000C0C0C0C0C0C0C0C0C0C0C0C0C0C0C0C02
:10FE400008080808080808080C0C0C0C0C0C0C0C12
:10FE50000C0C0C0C0C0C0C0C0C0C0C0C0C0C0C0CE2
:10FE60000C0C0C0C0C0C0C0C0C0C0C0C0C0C0C0CD2
:10FE70000C0C0C0C0C0C0C0C0C0C0C0C0C0C0C0CC2
:10FE800008080808080808080C0C0C0C0C0C0C0CD2
:10FE90000C0C0C0C0C0C0C0C0C0C0C0C0C0C0C0CA2
:10FEA0000C0C0C0C0C0C0C0C0C0C0C0C0C0C0C0C92
:10FEB0000C0C0C0C0C0C0C0C0C0C0C0C0C0C0C0C82
:10FEC00008080808080808080C0C0C0C0C0C0C0C92
:10FED0000C0C0C0C0C0C0C0C0C0C0C0C0C0C0C0C62
:10FEE0000C0C0C0C0C0C0C0C0C0C0C0C0C0C0C0C52
:10FEF0000C0C0C0C0C0C0C0C0C0C0C0C0C0C0C0C42
:10FF000008080808080808080C0C0C0C0C0C0C0C51
:10FF10000C0C0C0C0C0C0C0C0C0C0C0C0C0C0C0C21
:10FF20000C0C0C0C0C0C0C0C0C0C0C0C0C0C0C0C11
:10FF30000C0C0C0C0C0C0C0C0C0C0C0C0C0C0C0C01
:10FF400008080808080808080C0C0C0C0C0C0C0C11
:10FF50000C0C0C0C0C0C0C0C0C0C0C0C0C0C0C0CE1
:10FF60000C0C0C0C0C0C0C0C0C0C0C0C0C0C0C0CD1
:10FF70000C0C0C0C0C0C0C0C0C0C0C0C0C0C0C0CC1
:10FF800008080808080808080C0C0C0C0C0C0C0CD1
:10FF90000C0C0C0C0C0C0C0C0C0C0C0C0C0C0C0CA1
:10FFA0000C0C0C0C0C0C0C0C0C0C0C0C0C0C0C0C91
:10FFB0000C0C0C0C0C0C0C0C0C0C0C0C0C0C0C0C81
:10FFC00008080808080808080C0C0C0C0C0C0C0C91
:10FFD0000C0C0C0C0C0C0C0C0C0C0C0C0C0C0C0C61
:10FFE0000C0C0C0C0C0C0C0C0C0C0C0C0C0C0C0C51
:10FFF0000C0C0C0C0C0C0C0C0C0C0C0C0C0C0C0C41
:020000040005F5
:100000000D0D0D0D0D0D0D0D0D0D0D0D0D0D0D0D20
:1010000008080808080808080C0C0C0C0C0C0C0C40
:101010000C0C0C0C0C0C0C0C0C0C0C0C0C0C0C0C10
:101020000C0C0C0C0C0C0C0C0C0C0C0C0C0C0C0C00
:101030000C0C0C0C0C0C0C0C0C0C0C0C0C0C0C0CF0
:1010400008080808080808080C0C0C0C0C0C0C0C00
:101050000C0C0C0C0C0C0C0C0C0C0C0C0C0C0C0CD0
:101060000C0C0C0C0C0C0C0C0C0C0C0C0C0C0C0CC0
:101070000C0C0C0C0C0C0C0C0C0C0C0C0C0C0C0CB0
:1010800008080808080808080C0C0C0C0C0C0C0CC0
:101090000C0C0C0C0C0C0C0C0C0C0C0C0C0C0C0C90
:1010A0000C0C0C0C0C0C0C0C0C0C0C0C0C0C0C0C80
:1010B0000C0C0C0C0C0C0C0C0C0C0C0C0C0C0C0C70
:1010C00008080808080808080C0C0C0C0C0C0C0C80
:1010D0000C0C0C0C0C0C0C0C0C0C0C0C0C0C0C0C50
:1010E0000C0C0C0C0C0C0C0C0C0C0C0C0C0C0C0C40
:1010F0000C0C0C0C0C0C0C0C0C0C0C0C0C0C0C0C30
:1011000008080808080808080C0C0C0C0C0C0C0C3F
:101110000C0C0C0C0C0C0C0C0C0C0C0C0C0C0C0C0F
:101120000C0C0C0C0C0C0C0C0C0C0C0C0C0C0C0CFF
:101130000C0C0C0C0C0C0C0C0C0C0C0C0C0C0C0CEF
:1011400008080808080808080C0C0C0C0C0C0C0CFF
:101150000C0C0C0C0C0C0C0C0C0C0C0C0C0C0C0CCF
:101160000C0C0C0C0C0C0C0C0C0C0C0C0C0C0C0CBF
:101170000C0C0C0C0C0C0C0C0C0C0C0C0C0C0C0CAF
:1011800008080808080808080C0C0C0C0C0C0C0CBF
:101190000C0C0C0C0C0C0C0C0C0C0C0C0C0C0C0C8F
:1011A0000C0C0C0C0C0C0C0C0C0C0C0C0C0C0C0C7F
:1011B0000C0C0C0C0C0C0C0C0C0C0C0C0C0C0C0C6F
:1011C00008080808080808080C0C0C0C0C0C0C0C7F
:1011D0000C0C0C0C0C0C0C0C0C0C0C0C0C0C0C0C4F
:1011E0000C0C0C0C0C0C0C0C0C0C0C0C0C0C0C0C3F
:1011F0000C0C0C0C0C0C0C0C0C0C0C0C0C0C0C0C2F
:101200000C0C0C0C0C0C0C0C0C0C0C0C0C0C0C0C1E
:1020000008080808080808080C0C0C0C0C0C0C0C30
:102010000C0C0C0C0C0C0C0C0C0C0C0C0C0C0C0C00
:102020000C0C0C0C0C0C0C0C0C0C0C0C0C0C0C0CF0
:102030000C0C0C0C0C0C0C0C0C0C0C0C0C0C0C0CE0
:1020400008080808080808080C0C0C0C0C0C0C0CF0
:102050000C0C0C0C0C0C0C0C0C0C0C0C0C0C0C0CC0
:102060000C0C0C0C0C0C0C0C0C0C0C0C0C0C0C0CB0
:102070000C0C0C0C0C0C0C0C0C0C0C0C0C0C0C0CA0
:1020800008080808080808080C0C0C0C0C0C0C0CB0
:102090000C0C0C0C0C0C0C0C0C0C0C0C0C0C0C0C80
:1020A0000C0C0C0C0C0C0C0C0C0C0C0C0C0C0C0C70
:1020B0000C0C0C0C0C0C0C0C0C0C0C0C0C0C0C0C60
:1020C00008080808080808080C0C0C0C0C0C0C0C70
:1020D0000C0C0C0C0C0C0C0C0C0C0C0C0C0C0C0C40
:1020E0000C0C0C0C0C0C0C0C0C0C0C0C0C0C0C0C30
:1020F0000C0C0C0C0C0C0C0C0C0C0C0C0C0C0C0C20
:1021000008080808080808080C0C0C0C0C0C0C0C2F
:102110000C0C0C0C0C0C0C0C0C0C0C0C0C0C0C0CFF
:102120000C0C0C0C0C0C0C0C0C0C0C0C0C0C0C0CEF
:102130000C0C0C0C0C0C0C0C0C0C0C0C0C0C0C0CDF
:1021400008080808080808080C0C0C0C0C0C0C0CEF
:102150000C0C0C0C0C0C0C0C0C0C0C0C0C0C0C0CBF
:102160000C0C0C0C0C0C0C0C0C0C0C0C0C0C0C0CAF
:102170000C0C0C0C0C0C0C0C0C0C0C0C0C0C0C0C9F
:1021800008080808080808080C0C0C0C0C0C0C0CAF
:102190000C0C0C0C0C0C0C0C0C0C0C0C0C0C0C0C7F
:1021A0000C0C0C0C0C0C0C0C0C0C0C0C0C0C0C0C6F
:1021B0000C0C0C0C0C0C0C0C0C0C0C0C0C0C0C0C5F
:1021C00008080808080808080C0C0C0C0C0C0C0C6F
:1021D0000C0C0C0C0C0C0C0C0C0C0C0C0C0C0C0C3F
:1021E0000C0C0C0C0C0C0C0C0C0C0C0C0C0C0C0C2F
:1021F0000C0C0C0C0C0C0C0C0C0C0C0C0C0C0C0C1F
:102200000C0C0C0C0C0C0C0C0C0C0C0C0C0C0C0C0E
:1030000008080808080808080C0C0C0C0C0C0C0C20
:103010000C0C0C0C0C0C0C0C0C0C0C0C0C0C0C0CF0
:103020000C0C0C0C0C0C0C0C0C0C0C0C0C0C0C0CE0
:103030000C0C0C0C0C0C0C0C0C0C0C0C0C0C0C0CD0
:1030400008080808080808080C0C0C0C0C0C0C0CE0
:103050000C0C0C0C0C0C0C0C0C0C0C0C0C0C0C0CB0
:103060000C0C0C0C0C0C0C0C0C0C0C0C0C0C0C0CA0
:103070000C0C0C0C0C0C0C0C0C0C0C0C0C0C0C0C90
:1030800008080808080808080C0C0C0C0C0C0C0CA0
:103090000C0C0C0C0C0C0C0C0C0C0C0C0C0C0C0C70
:1030A0000C0C0C0C0C0C0C0C0C0C0C0C0C0C0C0C60
:1030B0000C0C0C0C0C0C0C0C0C0C0C0C0C0C0C0C50
:1030C00008080808080808080C0C0C0C0C0C0C0C60
:1030D0000C0C0C0C0C0C0C0C0C0C0C0C0C0C0C0C30
:1030E0000C0C0C0C0C0C0C0C0C0C0C0C0C0C0C0C20
:1030F0000C0C0C0C0C0C0C0C0C0C0C0C0C0C0C0C10
:1031000008080808080808080C0C0C0C0C0C0C0C1F
:103110000C0C0C0C0C0C0C0C0C0C0C0C0C0C0C0CEF
:103120000C0C0C0C0C0C0C0C0C0C0C0C0C0C0C0CDF
:103130000C0C0C0C0C0C0C0C0C0C0C0C0C0C0C0CCF
:1031400008080808080808080C0C0C0C0C0C0C0CDF
:103150000C0C0C0C0C0C0C0C0C0C0C0C0C0C0C0CAF
:103160000C0C0C0C0C0C0C0C0C0C0C0C0C0C0C0C9F
:103170000C0C0C0C0C0C0C0C0C0C0C0C0C0C0C0C8F
:1031800008080808080808080C0C0C0C0C0C0C0C9F
:103190000C0C0C0C0C0C0C0C0C0C0C0C0C0C0C0C6F
:1031A0000C0C0C0C0C0C0C0C0C0C0C0C0C0C0C0C5F
:1031B0000C0C0C0C0C0C0C0C0C0C0C0C0C0C0C0C4F
:1031C00008080808080808080C0C0C0C0C0C0C0C5F
:1031D0000C0C0C0C0C0C0C0C0C0C0C0C0C0C0C0C2F
:1031E0000C0C0C0C0C0C0C0C0C0C0C0C0C0C0C0C1F
:1031F0000C0C0C0C0C0C0C0C0C0C0C0C0C0C0C0C0F
:103200000C0C0C0C0C0C0C0C0C0C0C0C0C0C0C0CFE
:1040000008080808080808080C0C0C0C0C0C0C0C10
:104010000C0C0C0C0C0C0C0C0C0C0C0C0C0C0C0CE0
:104020000C0C0C0C0C0C0C0C0C0C0C0C0C0C0C0CD0
:104030000C0C0C0C0C0C0C0C0C0C0C0C0C0C0C0CC0
:1040400008080808080808080C0C0C0C0C0C0C0CD0
:104050000C0C0C0C0C0C0C0C0C0C0C0C0C0C0C0CA0
:104060000C0C0C0C0C0C0C0C0C0C0C0C0C0C0C0C90
:104070000C0C0C0C0C0C0C0C0C0C0C0C0C0C0C0C80
:1040800008080808080808080C0C0C0C0C0C0C0C90
:104090000C0C0C0C0C0C0C0C0C0C0C0C0C0C0C0C60
:1040A0000C0C0C0C0C0C0C0C0C0C0C0C0C0C0C0C50
:1040B0000C0C0C0C0C0C0C0C0C0C0C0C0C0C0C0C40
:1040C00008080808080808080C0C0C0C0C0C0C0C50
:1040D0000C0C0C0C0C0C0C0C0C0C0C0C0C0C0C0C20
:1040E0000C0C0C0C0C0C0C0C0C0C0C0C0C0C0C0C10
:1040F0000C0C0C0C0C0C0C0C0C0C0C0C0C0C0C0C00
:1041000008080808080808080C0C0C0C0C0C0C0C0F
:104110000C0C0C0C0C0C0C0C0C0C0C0C0C0C0C0CDF
:104120000C0C0C0C0C0C0C0C0C0C0C0C0C0C0C0CCF
:104130000C0C0C0C0C0C0C0C0C0C0C0C0C0C0C0CBF
:1041400008080808080808080C0C0C0C0C0C0C0CCF
:104150000C0C0C0C0C0C0C0C0C0C0C0C0C0C0C0C9F
:104160000C0C0C0C0C0C0C0C0C0C0C0C0C0C0C0C8F
:104170000C0C0C0C0C0C0C0C0C0C0C0C0C0C0C0C7F
:1041800008080808080808080C0C0C0C0C0C0C0C8F
:104190000C0C0C0C0C0C0C0C0C0C0C0C0C0C0C0C5F
:1041A0000C0C0C0C0C0C0C0C0C0C0C0C0C0C0C0C4F
:1041B0000C0C0C0C0C0C0C0C0C0C0C0C0C0C0C0C3F
:1041C00008080808080808080C0C0C0C0C0C0C0C4F
:1041D0000C0C0C0C0C0C0C0C0C0C0C0C0C0C0C0C1F
:1041E0000C0C0C0C0C0C0C0C0C0C0C0C0C0C0C0C0F
:1041F0000C0C0C0C0C0C0C0C0C0C0C0C0C0C0C0CFF
:104200000C0C0C0C0C0C0C0C0C0C0C0C0C0C0C0CEE
:1050000008080808080808080C0C0C0C0C0C0C0C00
:105010000C0C0C0C0C0C0C0C0C0C0C0C0C0C0C0CD0
:105020000C0C0C0C0C0C0C0C0C0C0C0C0C0C0C0CC0
:105030000C0C0C0C0C0C0C0C0C0C0C0C0C0C0C0CB0
:1050400008080808080808080C0C0C0C0C0C0C0CC0
:105050000C0C0C0C0C0C0C0C0C0C0C0C0C0C0C0C90
:105060000C0C0C0C0C0C0C0C0C0C0C0C0C0C0C0C80
:105070000C0C0C0C0C0C0C0C0C0C0C0C0C0C0C0C70
:1050800008080808080808080C0C0C0C0C0C0C0C80
:105090000C0C0C0C0C0C0C0C0C0C0C0C0C0C0C0C50
:1050A0000C0C0C0C0C0C0C0C0C0C0C0C0C0C0C0C40
:1050B0000C0C0C0C0C0C0C0C0C0C0C0C0C0C0C0C30
:1050C00008080808080808080C0C0C0C0C0C0C0C40
:1050D0000C0C0C0C0C0C0C0C0C0C0C0C0C0C0C0C10
:1050E0000C0C0C0C0C0C0C0C0C0C0C0C0C0C0C0C00
:1050F0000C0C0C0C0C0C0C0C0C0C0C0C0C0C0C0CF0
:1051000008080808080808080C0C0C0C0C0C0C0CFF
:105110000C0C0C0C0C0C0C0C0C0C0C0C0C0C0C0CCF
:105120000C0C0C0C0C0C0C0C0C0C0C0C0C0C0C0CBF
:105130000C0C0C0C0C0C0C0C0C0C0C0C0C0C0C0CAF
:1051400008080808080808080C0C0C0C0C0C0C0CBF
:105150000C0C0C0C0C0C0C0C0C0C0C0C0C0C0C0C8F
:105160000C0C0C0C0C0C0C0C0C0C0C0C0C0C0C0C7F
:105170000C0C0C0C0C0C0C0C0C0C0C0C0C0C0C0C6F
:1051800008080808080808080C0C0C0C0C0C0C0C7F
:105190000C0C0C0C0C0C0C0C0C0C0C0C0C0C0C0C4F
:1051A0000C0C0C0C0C0C0C0C0C0C0C0C0C0C0C0C3F
:1051B0000C0C0C0C0C0C0C0C0C0C0C0C0C0C0C0C2F
:1051C00008080808080808080C0C0C0C0C0C0C0C3F
:1051D0000C0C0C0C0C0C0C0C0C0C0C0C0C0C0C0C0F
:1051E0000C0C0C0C0C0C0C0C0C0C0C0C0C0C0C0CFF
:1051F0000C0C0C0C0C0C0C0C0C0C0C0C0C0C0C0CEF
:105200000C0C0C0C0C0C0C0C0C0C0C0C0C0C0C0CDE
:1060000008080808080808080C0C0C0C0C0C0C0CF0
:106010000C0C0C0C0C0C0C0C0C0C0C0C0C0C0C0CC0
:106020000C0C0C0C0C0C0C0C0C0C0C0C0C0C0C0CB0
:106030000C0C0C0C0C0C0C0C0C0C0C0C0C0C0C0CA0
:1060400008080808080808080C0C0C0C0C0C0C0CB0
:106050000C0C0C0C0C0C0C0C0C0C0C0C0C0C0C0C80
:106060000C0C0C0C0C0C0C0C0C0C0C0C0C0C0C0C70
:106070000C0C0C0C0C0C0C0C0C0C0C0C0C0C0C0C60
:1060800008080808080808080C0C0C0C0C0C0C0C70
:106090000C0C0C0C0C0C0C0C0C0C0C0C0C0C0C0C40
:1060A0000C0C0C0C0C0C0C0C0C0C0C0C0C0C0C0C30
:1060B0000C0C0C0C0C0C0C0C0C0C0C0C0C0C0C0C20
:1060C00008080808080808080C0C0C0C0C0C0C0C30
:1060D0000C0C0C0C0C0C0C0C0C0C0C0C0C0C0C0C00
:1060E0000C0C0C0C0C0C0C0C0C0C0C0C0C0C0C0CF0
:1060F0000C0C0C0C0C0C0C0C0C0C0C0C0C0C0C0CE0
:1061000008080808080808080C0C0C0C0C0C0C0CEF
:106110000C0C0C0C0C0C0C0C0C0C0C0C0C0C0C0CBF
:106120000C0C0C0C0C0C0C0C0C0C0C0C0C0C0C0CAF
:106130000C0C0C0C0C0C0C0C0C0C0C0C0C0C0C0C9F
:1061400008080808080808080C0C0C0C0C0C0C0CAF
:106150000C0C0C0C0C0C0C0C0C0C0C0C0C0C0C0C7F
:106160000C0C0C0C0C0C0C0C0C0C0C0C0C0C0C0C6F
:106170000C0C0C0C0C0C0C0C0C0C0C0C0C0C0C0C5F
:1061800008080808080808080C0C0C0C0C0C0C0C6F
:106190000C0C0C0C0C0C0C0C0C0C0C0C0C0C0C0C3F
:1061A0000C0C0C0C0C0C0C0C0C0C0C0C0C0C0C0C2F
:1061B0000C0C0C0C0C0C0C0C0C0C0C0C0C0C0C0C1F
:1061C00008080808080808080C0C0C0C0C0C0C0C2F
:1061D0000C0C0C0C0C0C0C0C0C0C0C0C0C0C0C0CFF
:1061E0000C0C0C0C0C0C0C0C0C0C0C0C0C0C0C0CEF
:1061F0000C0C0C0C0C0C0C0C0C0C0C0C0C0C0C0CDF
:106200000C0C0C0C0C0C0C0C0C0C0C0C0C0C0C0CCE
:1090000008080808080808080C0C0C0C0C0C0C0CC0
:109010000C0C0C0C0C0C0C0C0C0C0C0C0C0C0C0C90
:109020000C0C0C0C0C0C0C0C0C0C0C0C0C0C0C0C80
:109030000C0C0C0C0C0C0C0C0C0C0C0C0C0C0C0C70
:1090400008080808080808080C0C0C0C0C0C0C0C80
:109050000C0C0C0C0C0C0C0C0C0C0C0C0C0C0C0C50
:109060000C0C0C0C0C0C0C0C0C0C0C0C0C0C0C0C40
:109070000C0C0C0C0C0C0C0C0C0C0C0C0C0C0C0C30
:1090800008080808080808080C0C0C0C0C0C0C0C40
:109090000C0C0C0C0C0C0C0C0C0C0C0C0C0C0C0C10
:1090A0000C0C0C0C0C0C0C0C0C0C0C0C0C0C0C0C00
:1090B0000C0C0C0C0C0C0C0C0C0C0C0C0C0C0C0CF0
:1090C00008080808080808080C0C0C0C0C0C0C0C00
:1090D0000C0C0C0C0C0C0C0C0C0C0C0C0C0C0C0CD0
:1090E0000C0C0C0C0C0C0C0C0C0C0C0C0C0C0C0CC0
:1090F0000C0C0C0C0C0C0C0C0C0C0C0C0C0C0C0CB0
:1091000008080808080808080C0C0C0C0C0C0C0CBF
:109110000C0C0C0C0C0C0C0C0C0C0C0C0C0C0C0C8F
:109120000C0C0C0C0C0C0C0C0C0C0C0C0C0C0C0C7F
:109130000C0C0C0C0C0C0C0C0C0C0C0C0C0C0C0C6F
:1091400008080808080808080C0C0C0C0C0C0C0C7F
:109150000C0C0C0C0C0C0C0C0C0C0C0C0C0C0C0C4F
:109160000C0C0C0C0C0C0C0C0C0C0C0C0C0C0C0C3F
:109170000C0C0C0C0C0C0C0C0C0C0C0C0C0C0C0C2F
:1091800008080808080808080C0C0C0C0C0C0C0C3F
:109190000C0C0C0C0C0C0C0C0C0C0C0C0C0C0C0C0F
:1091A0000C0C0C0C0C0C0C0C0C0C0C0C0C0C0C0CFF
:1091B0000C0C0C0C0C0C0C0C0C0C0C0C0C0C0C0CEF
:1091C00008080808080808080C0C0C0C0C0C0C0CFF
:1091D0000C0C0C0C0C0C0C0C0C0C0C0C0C0C0C0CCF
:1091E0000C0C0C0C0C0C0C0C0C0C0C0C0C0C0C0CBF
:1091F0000C0C0C0C0C0C0C0C0C0C0C0C0C0C0C0CAF
:109200000C0C0C0C0C0C0C0C0C0C0C0C0C0C0C0C9E
:10A0000008080808080808080C0C0C0C0C0C0C0CB0
:10A010000C0C0C0C0C0C0C0C0C0C0C0C0C0C0C0C80
:10A020000C0C0C0C0C0C0C0C0C0C0C0C0C0C0C0C70
:10A030000C0C0C0C0C0C0C0C0C0C0C0C0C0C0C0C60
:10A0400008080808080808080C0C0C0C0C0C0C0C70
:10A050000C0C0C0C0C0C0C0C0C0C0C0C0C0C0C0C40
:10A060000C0C0C0C0C0C0C0C0C0C0C0C0C0C0C0C30
:10A070000C0C0C0C0C0C0C0C0C0C0C0C0C0C0C0C20
:10A0800008080808080808080C0C0C0C0C0C0C0C30
:10A090000C0C0C0C0C0C0C0C0C0C0C0C0C0C0C0C00
:10A0A0000C0C0C0C0C0C0C0C0C0C0C0C0C0C0C0CF0
:10A0B0000C0C0C0C0C0C0C0C0C0C0C0C0C0C0C0CE0
:10A0C00008080808080808080C0C0C0C0C0C0C0CF0
:10A0D0000C0C0C0C0C0C0C0C0C0C0C0C0C0C0C0CC0
:10A0E0000C0C0C0C0C0C0C0C0C0C0C0C0C0C0C0CB0
:10A0F0000C0C0C0C0C0C0C0C0C0C0C0C0C0C0C0CA0
:10A1000008080808080808080C0C0C0C0C0C0C0CAF
:10A110000C0C0C0C0C0C0C0C0C0C0C0C0C0C0C0C7F
:10A120000C0C0C0C0C0C0C0C0C0C0C0C0C0C0C0C6F
:10A130000C0C0C0C0C0C0C0C0C0C0C0C0C0C0C0C5F
:10A1400008080808080808080C0C0C0C0C0C0C0C6F
:10A150000C0C0C0C0C0C0C0C0C0C0C0C0C0C0C0C3F
:10A160000C0C0C0C0C0C0C0C0C0C0C0C0C0C0C0C2F
:10A170000C0C0C0C0C0C0C0C0C0C0C0C0C0C0C0C1F
:10A1800008080808080808080C0C0C0C0C0C0C0C2F
:10A190000C0C0C0C0C0C0C0C0C0C0C0C0C0C0C0CFF
:10A1A0000C0C0C0C0C0C0C0C0C0C0C0C0C0C0C0CEF
:10A1B0000C0C0C0C0C0C0C0C0C0C0C0C0C0C0C0CDF
:10A1C00008080808080808080C0C0C0C0C0C0C0CEF
:10A1D0000C0C0C0C0C0C0C0C0C0C0C0C0C0C0C0CBF
:10A1E0000C0C0C0C0C0C0C0C0C0C0C0C0C0C0C0CAF
:10A1F0000C0C0C0C0C0C0C0C0C0C0C0C0C0C0C0C9F
:10A200000C0C0C0C0C0C0C0C0C0C0C0C0C0C0C0C8E
:10B0000008080808080808080C0C0C0C0C0C0C0CA0
:10B010000C0C0C0C0C0C0C0C0C0C0C0C0C0C0C0C70
:10B020000C0C0C0C0C0C0C0C0C0C0C0C0C0C0C0C60
:10B030000C0C0C0C0C0C0C0C0C0C0C0C0C0C0C0C50
:10B0400008080808080808080C0C0C0C0C0C0C0C60
:10B050000C0C0C0C0C0C0C0C0C0C0C0C0C0C0C0C30
:10B060000C0C0C0C0C0C0C0C0C0C0C0C0C0C0C0C20
:10B070000C0C0C0C0C0C0C0C0C0C0C0C0C0C0C0C10
:10B0800008080808080808080C0C0C0C0C0C0C0C20
:10B090000C0C0C0C0C0C0C0C0C0C0C0C0C0C0C0CF0
:10B0A0000C0C0C0C0C0C0C0C0C0C0C0C0C0C0C0CE0
:10B0B0000C0C0C0C0C0C0C0C0C0C0C0C0C0C0C0CD0
:10B0C00008080808080808080C0C0C0C0C0C0C0CE0
:10B0D0000C0C0C0C0C0C0C0C0C0C0C0C0C0C0C0CB0
:10B0E0000C0C0C0C0C0C0C0C0C0C0C0C0C0C0C0CA0
:10B0F0000C0C0C0C0C0C0C0C0C0C0C0C0C0C0C0C90
:10B1000008080808080808080C0C0C0C0C0C0C0C9F
:10B110000C0C0C0C0C0C0C0C0C0C0C0C0C0C0C0C6F
:10B120000C0C0C0C0C0C0C0C0C0C0C0C0C0C0C0C5F
:10B130000C0C0C0C0C0C0C0C0C0C0C0C0C0C0C0C4F
:10B1400008080808080808080C0C0C0C0C0C0C0C5F
:10B150000C0C0C0C0C0C0C0C0C0C0C0C0C0C0C0C2F
:10B160000C0C0C0C0C0C0C0C0C0C0C0C0C0C0C0C1F
:10B170000C0C0C0C0C0C0C0C0C0C0C0C0C0C0C0C0F
:10B1800008080808080808080C0C0C0C0C0C0C0C1F
:10B190000C0C0C0C0C0C0C0C0C0C0C0C0C0C0C0CEF
:10B1A0000C0C0C0C0C0C0C0C0C0C0C0C0C0C0C0CDF
:10B1B0000C0C0C0C0C0C0C0C0C0C0C0C0C0C0C0CCF
:10B1C00008080808080808080C0C0C0C0C0C0C0CDF
:10B1D0000C0C0C0C0C0C0C0C0C0C0C0C0C0C0C0CAF
:10B1E0000C0C0C0C0C0C0C0C0C0C0C0C0C0C0C0C9F
:10B1F0000C0C0C0C0C0C0C0C0C0C0C0C0C0C0C0C8F
:10B200000C0C0C0C0C0C0C0C0C0C0C0C0C0C0C0C7E
:10C0000008080808080808080C0C0C0C0C0C0C0C90
:10C010000C0C0C0C0C0C0C0C0C0C0C0C0C0C0C0C60
:10C020000C0C0C0C0C0C0C0C0C0C0C0C0C0C0C0C50
:10C030000C0C0C0C0C0C0C0C0C0C0C0C0C0C0C0C40
:10C0400008080808080808080C0C0C0C0C0C0C0C50
:10C050000C0C0C0C0C0C0C0C0C0C0C0C0C0C0C0C20
:10C060000C0C0C0C0C0C0C0C0C0C0C0C0C0C0C0C10
:10C070000C0C0C0C0C0C0C0C0C0C0C0C0C0C0C0C00
:10C0800008080808080808080C0C0C0C0C0C0C0C10
:10C090000C0C0C0C0C0C0C0C0C0C0C0C0C0C0C0CE0
:10C0A0000C0C0C0C0C0C0C0C0C0C0C0C0C0C0C0CD0
:10C0B0000C0C0C0C0C0C0C0C0C0C0C0C0C0C0C0CC0
:10C0C00008080808080808080C0C0C0C0C0C0C0CD0
:10C0D0000C0C0C0C0C0C0C0C0C0C0C0C0C0C0C0CA0
:10C0E0000C0C0C0C0C0C0C0C0C0C0C0C0C0C0C0C90
:10C0F0000C0C0C0C0C0C0C0C0C0C0C0C0C0C0C0C80
:10C1000008080808080808080C0C0C0C0C0C0C0C8F
:10C110000C0C0C0C0C0C0C0C0C0C0C0C0C0C0C0C5F
:10C120000C0C0C0C0C0C0C0C0C0C0C0C0C0C0C0C4F
:10C130000C0C0C0C0C0C0C0C0C0C0C0C0C0C0C0C3F
:10C1400008080808080808080C0C0C0C0C0C0C0C4F
:10C150000C0C0C0C0C0C0C0C0C0C0C0C0C0C0C0C1F
:10C160000C0C0C0C0C0C0C0C0C0C0C0C0C0C0C0C0F
:10C170000C0C0C0C0C0C0C0C0C0C0C0C0C0C0C0CFF
:10C1800008080808080808080C0C0C0C0C0C0C0C0F
:10C190000C0C0C0C0C0C0C0C0C0C0C0C0C0C0C0CDF
:10C1A0000C0C0C0C0C0C0C0C0C0C0C0C0C0C0C0CCF
:10C1B0000C0C0C0C0C0C0C0C0C0C0C0C0C0C0C0CBF
:10C1C00008080808080808080C0C0C0C0C0C0C0CCF
:10C1D0000C0C0C0C0C0C0C0C0C0C0C0C0C0C0C0C9F
:10C1E0000C0C0C0C0C0C0C0C0C0C0C0C0C0C0C0C8F
:10C1F0000C0C0C0C0C0C0C0C0C0C0C0C0C0C0C0C7F
:10C200000C0C0C0C0C0C0C0C0C0C0C0C0C0C0C0C6E
:10D0000008080808080808080C0C0C0C0C0C0C0C80
:10D010000C0C0C0C0C0C0C0C0C0C0C0C0C0C0C0C50
:10D020000C0C0C0C0C0C0C0C0C0C0C0C0C0C0C0C40
:10D030000C0C0C0C0C0C0C0C0C0C0C0C0C0C0C0C30
:10D0400008080808080808080C0C0C0C0C0C0C0C40
:10D050000C0C0C0C0C0C0C0C0C0C0C0C0C0C0C0C10
:10D060000C0C0C0C0C0C0C0C0C0C0C0C0C0C0C0C00
:10D070000C0C0C0C0C0C0C0C0C0C0C0C0C0C0C0CF0
:10D0800008080808080808080C0C0C0C0C0C0C0C00
:10D090000C0C0C0C0C0C0C0C0C0C0C0C0C0C0C0CD0
:10D0A0000C0C0C0C0C0C0C0C0C0C0C0C0C0C0C0CC0
:10D0B0000C0C0C0C0C0C0C0C0C0C0C0C0C0C0C0CB0
:10D0C00008080808080808080C0C0C0C0C0C0C0CC0
:10D0D0000C0C0C0C0C0C0C0C0C0C0C0C0C0C0C0C90
:10D0E0000C0C0C0C0C0C0C0C0C0C0C0C0C0C0C0C80
:10D0F0000C0C0C0C0C0C0C0C0C0C0C0C0C0C0C0C70
:10D1000008080808080808080C0C0C0C0C0C0C0C7F
:10D110000C0C0C0C0C0C0C0C0C0C0C0C0C0C0C0C4F
:10D120000C0C0C0C0C0C0C0C0C0C0C0C0C0C0C0C3F
:10D130000C0C0C0C0C0C0C0C0C0C0C0C0C0C0C0C2F
:10D1400008080808080808080C0C0C0C0C0C0C0C3F
:10D150000C0C0C0C0C0C0C0C0C0C0C0C0C0C0C0C0F
:10D160000C0C0C0C0C0C0C0C0C0C0C0C0C0C0C0CFF
:10D170000C0C0C0C0C0C0C0C0C0C0C0C0C0C0C0CEF
:10D1800008080808080808080C0C0C0C0C0C0C0CFF
:10D190000C0C0C0C0C0C0C0C0C0C0C0C0C0C0C0CCF
:10D1A0000C0C0C0C0C0C0C0C0C0C0C0C0C0C0C0CBF
:10D1B0000C0C0C0C0C0C0C0C0C0C0C0C0C0C0C0CAF
:10D1C00008080808080808080C0C0C0C0C0C0C0CBF
:10D1D0000C0C0C0C0C0C0C0C0C0C0C0C0C0C0C0C8F
:10D1E0000C0C0C0C0C0C0C0C0C0C0C0C0C0C0C0C7F
:10D1F0000C0C0C0C0C0C0C0C0C0C0C0C0C0C0C0C6F
:10D200000C0C0C0C0C0C0C0C0C0C0C0C0C0C0C0C5E
:10E0000008080808080808080C0C0C0C0C0C0C0C70
:10E010000C0C0C0C0C0C0C0C0C0C0C0C0C0C0C0C40
:10E020000C0C0C0C0C0C0C0C0C0C0C0C0C0C0C0C30
:10E030000C0C0C0C0C0C0C0C0C0C0C0C0C0C0C0C20
:10E0400008080808080808080C0C0C0C0C0C0C0C30
:10E050000C0C0C0C0C0C0C0C0C0C0C0C0C0C0C0C00
:10E060000C0C0C0C0C0C0C0C0C0C0C0C0C0C0C0CF0
:10E070000C0C0C0C0C0C0C0C0C0C0C0C0C0C0C0CE0
:10E0800008080808080808080C0C0C0C0C0C0C0CF0
:10E090000C0C0C0C0C0C0C0C0C0C0C0C0C0C0C0CC0
:10E0A0000C0C0C0C0C0C0C0C0C0C0C0C0C0C0C0CB0
:10E0B0000C0C0C0C0C0C0C0C0C0C0C0C0C0C0C0CA0
:10E0C00008080808080808080C0C0C0C0C0C0C0CB0
:10E0D0000C0C0C0C0C0C0C0C0C0C0C0C0C0C0C0C80
:10E0E0000C0C0C0C0C0C0C0C0C0C0C0C0C0C0C0C70
:10E0F0000C0C0C0C0C0C0C0C0C0C0C0C0C0C0C0C60
:10E1000008080808080808080C0C0C0C0C0C0C0C6F
:10E110000C0C0C0C0C0C0C0C0C0C0C0C0C0C0C0C3F
:10E120000C0C0C0C0C0C0C0C0C0C0C0C0C0C0C0C2F
:10E130000C0C0C0C0C0C0C0C0C0C0C0C0C0C0C0C1F
:10E1400008080808080808080C0C0C0C0C0C0C0C2F
:10E150000C0C0C0C0C0C0C0C0C0C0C0C0C0C0C0CFF
:10E160000C0C0C0C0C0C0C0C0C0C0C0C0C0C0C0CEF
:10E170000C0C0C0C0C0C0C0C0C0C0C0C0C0C0C0CDF
:10E1800008080808080808080C0C0C0C0C0C0C0CEF
:10E190000C0C0C0C0C0C0C0C0C0C0C0C0C0C0C0CBF
:10E1A0000C0C0C0C0C0C0C0C0C0C0C0C0C0C0C0CAF
:10E1B0000C0C0C0C0C0C0C0C0C0C0C0C0C0C0C0C9F
:10E1C00008080808080808080C0C0C0C0C0C0C0CAF
:10E1D0000C0C0C0C0C0C0C0C0C0C0C0C0C0C0C0C7F
:10E1E0000C0C0C0C0C0C0C0C0C0C0C0C0C0C0C0C6F
:10E1F0000C0C0C0C0C0C0C0C0C0C0C0C0C0C0C0C5F
:10E200000C0C0C0C0C0C0C0C0C0C0C0C0C0C0C0C4E
:020000040006F4
:1010000008080808080808080C0C0C0C0C0C0C0C40
:101010000C0C0C0C0C0C0C0C0C0C0C0C0C0C0C0C10
:101020000C0C0C0C0C0C0C0C0C0C0C0C0C0C0C0C00
:101030000C0C0C0C0C0C0C0C0C0C0C0C0C0C0C0CF0
:1010400008080808080808080C0C0C0C0C0C0C0C00
:101050000C0C0C0C0C0C0C0C0C0C0C0C0C0C0C0CD0
:101060000C0C0C0C0C0C0C0C0C0C0C0C0C0C0C0CC0
:101070000C0C0C0C0C0C0C0C0C0C0C0C0C0C0C0CB0
:1010800008080808080808080C0C0C0C0C0C0C0CC0
:101090000C0C0C0C0C0C0C0C0C0C0C0C0C0C0C0C90
:1010A0000C0C0C0C0C0C0C0C0C0C0C0C0C0C0C0C80
:1010B0000C0C0C0C0C0C0C0C0C0C0C0C0C0C0C0C70
:1010C00008080808080808080C0C0C0C0C0C0C0C80
:1010D0000C0C0C0C0C0C0C0C0C0C0C0C0C0C0C0C50
:1010E0000C0C0C0C0C0C0C0C0C0C0C0C0C0C0C0C40
:1010F0000C0C0C0C0C0C0C0C0C0C0C0C0C0C0C0C30
:1011000008080808080808080C0C0C0C0C0C0C0C3F
:101110000C0C0C0C0C0C0C0C0C0C0C0C0C0C0C0C0F
:101120000C0C0C0C0C0C0C0C0C0C0C0C0C0C0C0CFF
:101130000C0C0C0C0C0C0C0C0C0C0C0C0C0C0C0CEF
:1011400008080808080808080C0C0C0C0C0C0C0CFF
:101150000C0C0C0C0C0C0C0C0C0C0C0C0C0C0C0CCF
:101160000C0C0C0C0C0C0C0C0C0C0C0C0C0C0C0CBF
:101170000C0C0C0C0C0C0C0C0C0C0C0C0C0C0C0CAF
:1011800008080808080808080C0C0C0C0C0C0C0CBF
:101190000C0C0C0C0C0C0C0C0C0C0C0C0C0C0C0C8F
:1011A0000C0C0C0C0C0C0C0C0C0C0C0C0C0C0C0C7F
:1011B0000C0C0C0C0C0C0C0C0C0C0C0C0C0C0C0C6F
:1011C00008080808080808080C0C0C0C0C0C0C0C7F
:1011D0000C0C0C0C0C0C0C0C0C0C0C0C0C0C0C0C4F
:1011E0000C0C0C0C0C0C0C0C0C0C0C0C0C0C0C0C3F
:1011F0000C0C0C0C0C0C0C0C0C0C0C0C0C0C0C0C2F
:101200000E0E0E0E0E0E0E0E0E0E0E0E0E0E0E0EFE
:1020000008080808080808080C0C0C0C0C0C0C0C30
:102010000C0C0C0C0C0C0C0C0C0C0C0C0C0C0C0C00
:102020000C0C0C0C0C0C0C0C0C0C0C0C0C0C0C0CF0
:102030000C0C0C0C0C0C0C0C0C0C0C0C0C0C0C0CE0
:1020400008080808080808080C0C0C0C0C0C0C0CF0
:102050000C0C0C0C0C0C0C0C0C0C0C0C0C0C0C0CC0
:102060000C0C0C0C0C0C0C0C0C0C0C0C0C0C0C0CB0
:102070000C0C0C0C0C0C0C0C0C0C0C0C0C0C0C0CA0
:1020800008080808080808080C0C0C0C0C0C0C0CB0
:102090000C0C0C0C0C0C0C0C0C0C0C0C0C0C0C0C80
:1020A0000C0C0C0C0C0C0C0C0C0C0C0C0C0C0C0C70
:1020B0000C0C0C0C0C0C0C0C0C0C0C0C0C0C0C0C60
:1020C00008080808080808080C0C0C0C0C0C0C0C70
